:020000022000DC
:10600000000004207D860200915F07008B65070079
:10601000915F0700915F0700915F0700000000009B
:10602000000000000000000000000000915F070079
:10603000915F070000000000915F0700915F07007B
:1060400071850200915F0700D1890200AD880200CE
:10605000BD880200915F0700ED810200915F07009B
:10606000915F0700B1890200C18902004D860200DC
:10607000915F0700915F0700915F0700915F070044
:10608000218E02005D860200915F0700915F07008C
:10609000915F0700915F07001D890200915F070073
:1060A000915F0700915F0700915F0700915F070014
:1060B000915F0700915F07000000000000000000F2
:1060C000915F0700915F0700915F0700CD88020094
:1060D0006D860200915F0700915F0700F189020061
:1060E000E1890200915F0700915F0700F5880200D7
:0860F00000000000915F0700B1
:1070000040F8044B40F8045B40F8046B40F8047B04
:1070100040F8048B40F8049B40F804AB40F804BBF4
:1070200040F804CB40F804DB6846704781F000412B
:1070300002E000BF83F0004330B54FEA41044FEA5D
:10704000430594EA050F08BF90EA020F1FBF54EAF8
:10705000000C55EA020C7FEA645C7FEA655C00F094
:10706000E2804FEA5454D4EB5555B8BF6D420CDD65
:107070002C4480EA020281EA030382EA000083EAE8
:10708000010180EA020281EA0303362D88BF30BD88
:1070900011F0004F4FEA01314FF4801C4CEA1131DE
:1070A00002D0404261EB410113F0004F4FEA03333D
:1070B0004CEA133302D0524263EB430394EA050FC8
:1070C00000F0A780A4F10104D5F1200E0DDB02FA37
:1070D0000EFC22FA05F2801841F1000103FA0EF2CB
:1070E000801843FA05F359410EE0A5F120050EF191
:1070F000200E012A03FA0EFC28BF4CF0020C43FAC2
:1071000005F3C01851EBE37101F0004507D54FF0CE
:10711000000EDCF1000C7EEB00006EEB0101B1F51E
:10712000801F1BD3B1F5001F0CD349085FEA300064
:107130004FEA3C0C04F101044FEA445212F5800F6F
:1071400080F09A80BCF1004F08BF5FEA500C50F10C
:10715000000041EB045141EA050130BD5FEA4C0CEF
:10716000404141EB0101013C28BFB1F5801FE9D24C
:1071700091F0000F04BF01460020B1FA81F308BF6F
:107180002033A3F10B03B3F120020CDA0C3208DD3B
:1071900002F1140CC2F10C0201FA0CF021FA02F116
:1071A0000CE002F11402D8BFC2F1200C01FA02F186
:1071B00020FA0CFCDCBF41EA0C019040E41AA2BFAB
:1071C00001EB0451294330BD6FEA04041F3C1CDA73
:1071D0000C340EDC04F11404C4F1200220FA04F093
:1071E00001FA02F340EA030021FA04F345EA03013D
:1071F00030BDC4F10C04C4F1200220FA02F001FAFF
:1072000004F340EA0300294630BD21FA04F0294680
:1072100030BD94F0000F83F4801306BF81F4801119
:107220000134013D4EE77FEA645C18BF7FEA655C8C
:1072300029D094EA050F08BF90EA020F05D054EA5E
:10724000000C04BF1946104630BD91EA030F1EBF63
:107250000021002030BD5FEA545C05D14000494167
:1072600028BF41F0004130BD14F580043CBF01F55A
:10727000801130BD01F0004545F0FE4141F4700140
:107280004FF0000030BD7FEA645C1ABF194610461B
:107290007FEA655C1CBF0B46024650EA013406BF1C
:1072A00052EA033591EA030F41F4002130BD00BFDB
:1072B00090F0000F04BF0021704730B54FF4806498
:1072C00004F132044FF000054FF0000150E700BF19
:1072D00090F0000F04BF0021704730B54FF4806478
:1072E00004F1320410F0004548BF40424FF0000165
:1072F0003EE700BF42004FEAE2014FEA31014FEAA8
:1073000002701FBF12F07F4393F07F4F81F06051F6
:10731000704732F07F4208BF704793F07F4F04BF41
:1073200041F40021704730B54FF4607401F000451E
:1073300021F000411CE700BF50EA010208BF70477E
:1073400030B54FF000050AE050EA010208BF70476F
:1073500030B511F0004502D5404261EB41014FF4D8
:10736000806404F132045FEA915C3FF4D8AE4FF0E0
:1073700003025FEADC0C18BF03325FEADC0C18BFC3
:10738000033202EBDC02C2F1200300FA03FC20FA14
:1073900002F001FA03FE40EA0E0021FA02F1144461
:1073A000BDE600BF4FEA4102B2F1E04324BFB3F5AE
:1073B000001CDCF1FE5C0DD901F0004C4FEAC0026C
:1073C0004CEA5070B2F1004F40EB830008BF20F050
:1073D0000100704711F0804F21D113F13872BCBF0A
:1073E00001F00040704741F480114FEA5252C2F15F
:1073F0001802C2F1200C10FA0CF320FA02F018BFA8
:1074000040F001004FEAC1234FEAD32303FA0CFCFA
:1074100040EA0C0023FA02F34FEA4303CCE77FEA89
:10742000625307D150EA01331EBF4FF0FE4040F4D3
:107430004000704701F0004040F0FE4040F4000082
:10744000704700BF80F0004002E000BF81F00041C3
:1074500042001FBF5FEA410392EA030F7FEA226CFA
:107460007FEA236C6AD04FEA1262D2EB1363C1BF8A
:10747000D218414048404140B8BF5B42192B88BFF9
:10748000704710F0004F40F4000020F07F4018BF1C
:10749000404211F0004F41F4000121F07F4118BF3C
:1074A000494292EA030F3FD0A2F1010241FA03FCE4
:1074B00010EB0C00C3F1200301FA03F100F00043CC
:1074C00002D5494260EB4000B0F5000F13D3B0F194
:1074D000807F06D340084FEA310102F10102FE2A03
:1074E00051D2B1F1004F40EBC25008BF20F0010073
:1074F00040EA03007047490040EB0000013A28BF12
:10750000B0F5000FEDD2B0FA80FCACF1080CB2EB94
:107510000C0200FA0CF0AABF00EBC2505242184312
:10752000BCBFD0401843704792F0000F81F40001B7
:1075300006BF80F400000132013BB5E74FEA41038A
:107540007FEA226C18BF7FEA236C21D092EA030FF6
:1075500004D092F0000F08BF0846704790EA010F70
:107560001CBF0020704712F07F4F04D1400028BF9D
:1075700040F00040704712F100723CBF00F500007F
:10758000704700F0004343F0FE4040F400007047B5
:107590007FEA226216BF08467FEA23630146420261
:1075A00006BF5FEA412390EA010F40F48000704774
:1075B0004FF0000304E000BF10F0004348BF40421A
:1075C0005FEA000C08BF704743F0964301464FF056
:1075D00000001CE050EA010208BF70474FF00003B2
:1075E0000AE000BF50EA010208BF704711F00043F3
:1075F00002D5404261EB41015FEA010C02BF8446C3
:107600000146002043F0B64308BFA3F18053A3F521
:107610000003BCFA8CF2083AA3EBC25310DB01FA68
:1076200002FC634400FA02FCC2F12002BCF1004FEC
:1076300020FA02F243EB020008BF20F0010070477D
:1076400002F1200201FA02FCC2F1200250EA4C00D1
:1076500021FA02F243EB020008BF20EADC70704717
:107660007BB972B90029BEBF00204FF0004106E08F
:1076700008BF00281CBF6FF000414FF0FF3000F042
:1076800081B9ADF1080C6DE904CE002909DB002BAE
:107690001ADB02F045FDDDF804E0DDE9022304B069
:1076A0007047404261EB4101002B1BDB02F038FDCB
:1076B000DDF804E0DDE9022304B0404261EB410162
:1076C000524263EB43037047524263EB430302F0C1
:1076D00027FDDDF804E0DDE9022304B0404261EB60
:1076E00041017047524263EB430302F019FDDDF89C
:1076F00004E0DDE9022304B0524263EB4303704728
:1077000053B94AB9002908BF00281CBF4FF0FF3108
:107710004FF0FF3000F036B9ADF1080C6DE904CE42
:1077200002F0FEFCDDF804E0DDE9022304B070475E
:1077300070B54FF0FF0C4CF4E06C1CEA11541DBF07
:107740001CEA135594EA0C0F95EA0C0F00F0DEF8D2
:107750002C4481EA030621EA4C5123EA4C5350EAB7
:10776000013518BF52EA033541F4801143F4801308
:1077700038D0A0FB02CE4FF00005E1FB02E506F099
:107780000042E0FB03E54FF00006E1FB03569CF0EE
:10779000000F18BF4EF0010EA4F1FF04B6F5007FF4
:1077A00064F5407404D25FEA4E0E6D4146EB060666
:1077B00042EAC62141EA55514FEAC52040EA5E50EF
:1077C0004FEACE2EB4F1FD0C88BFBCF5E06F1ED899
:1077D000BEF1004F08BF5FEA500E50F1000041EBD0
:1077E000045170BD06F0004646EA010140EA02007D
:1077F00081EA0301B4EB5C04C2BFD4EB0C0541EA9F
:10780000045170BD41F480114FF0000E013C00F3B3
:10781000AB8014F1360FDEBF002001F0004170BDD7
:10782000C4F10004203C35DA0C341BDC04F11404F0
:10783000C4F1200500FA05F320FA04F001FA05F27C
:1078400040EA020001F0004221F0004110EBD37049
:1078500021FA04F642EB06015EEA430E08BF20EA75
:10786000D37070BDC4F10C04C4F1200500FA04F318
:1078700020FA05F001FA04F240EA020001F00041AA
:1078800010EBD37041F100015EEA430E08BF20EA1D
:10789000D37070BDC4F1200500FA05F24EEA020E65
:1078A00020FA04F301FA05F243EA020321FA04F094
:1078B00001F0004121FA04F220EA020000EBD3704B
:1078C0005EEA430E08BF20EAD37070BD94F0000F4B
:1078D0000FD101F00046400041EB010111F4801F7F
:1078E00008BF013CF7D041EA060195F0000F18BF30
:1078F000704703F00046520043EB030313F4801F6C
:1079000008BF013DF7D043EA0603704794EA0C0F25
:107910000CEA135518BF95EA0C0F0CD050EA41063B
:1079200018BF52EA4306D1D181EA030101F00041B8
:107930004FF0000070BD50EA410606BF10461946E0
:1079400052EA430619D094EA0C0F02D150EA0136EC
:1079500013D195EA0C0F05D152EA03361CBF10462D
:1079600019460AD181EA030101F0004141F0FE41CC
:1079700041F470014FF0000070BD41F0FE4141F450
:10798000780170BD704700BF4A0011D212F5001295
:1079900011D20DD56FF47873B3EB62520ED44FEA67
:1079A000C12343F0004343EA505323FA02F07047E7
:1079B0004FF00000704750EA013002D14FF0FF3025
:1079C00070474FF00000704730B5144685B017A3DC
:1079D000D3E90023FFF744FE054601A9284646F0F7
:1079E00079FF9DF807309DF806200F491B0443EAF4
:1079F00042539DF8082043EAC2239DF8092043EA38
:107A000042139DF80A2043EA5203BDF8042025F0F2
:107A10000105A2F2BC7243EA4263A5FB01012360A7
:107A200005B030BDAFF3008000CA9A3B00CA9A3B54
:107A300000000000182A2DE9F74F054621D0202A22
:107A400022D00A200423C5F8002185F8040185F816
:107A50000531284600F0A0FC0022034695F80541B8
:107A6000A24214D3DFF8DCC0DFF8DCE000EB8403D3
:107A700095F804210132B4EB820F1AD303B0BDE8AC
:107A8000F08F0C200623DEE70E200823DBE711F839
:107A9000044B03F8044B11F8034C03F8034C11F8A2
:107AA000024C03F8024C11F8014C03F8014C01326E
:107AB000D4E795F80521B4FBF2FA02FB1A4913F852
:107AC000041C13F8038C13F8027C13F8016C019268
:107AD000B9F1000F0BD11CF808B01CF807801CF896
:107AE00006701CF801601EF80A108BEA0101D5F837
:107AF0000021202A0CD1B9F1040F09D1DFF84490FC
:107B000019F8011019F8088019F8077019F80660BB
:107B1000019AA21A043310F8229000EB820281EA43
:107B2000090103F8041C517888EA010803F8038C62
:107B300091784F4003F8027CD278564003F8016CEC
:107B4000013495E7BB320A00B0320A002DE9F04F4C
:107B5000044685B0084600F01FFC89460246804670
:107B6000214600204EF0F1F9231D019304F110038A
:107B70000125029322462146002311F82300324EAC
:107B8000305C01F823000133042BF6D1019B013155
:107B90008B42F1D1617963786170617A6171617B47
:107BA0006172A17A6373A378A170A17BA372A37998
:107BB000A171E17BA373E378E170E17AE173E1798C
:107BC000E172E37199F80431AB4234D092F800B01D
:107BD0005678917892F803A08BEA060081EA0A03AE
:107BE00080EA0307039365F01CFE8BEA00007840EF
:107BF000107086EA010065F014FE46407E40567023
:107C0000039865F00EFE4140794091708BEA0A00BE
:107C100065F007FE8AEA000A029B87EA0A07D77026
:107C200004329342D2D128464246214601354EF0D5
:107C30008CF9EDB29EE742462146284605B0BDE8E4
:107C4000F04F4EF082B900BFBB320A002DE9F04F71
:107C5000504C904603F003029B101F2B04EB821440
:107C600089469E464C49A8BF4FF01F0E1C2B1D464F
:107C7000A8BF1C2551F822206168033587B025EA8A
:107C8000E575294101920391E268A1688446294182
:107C900000202A410290049105925CF8045B3F4A5F
:107CA000154225F0004111D106AA02EB810151F8DD
:107CB000102C002D40EA0200B8BF5242B8F1010872
:107CC00049F8042BE9D107B0BDE8F08F344A1542DA
:107CD00009D154F82120002BBABFCEF100018A400F
:107CE00042FA0EF2E5E72F4A154214D110392E4A16
:107CF000019E52F8212082FB0616AEF10302002AF3
:107D000044DA51426FF0004242FA01F7B742D0DB49
:107D100006FA01F2CDE74A04B2F1006FB6BF4A0598
:107D200000210421B2F1005FB8BF92001F4EB8BF1E
:107D30000231B2F1804FBCBF52000131B242C7BF25
:107D40001B4F1C4E1C4F1D4E924687FB0ABA77688C
:107D50005744924687FB0ABAB7685744924687FB56
:107D60000ABAF768BA448AFB027236691644144AA2
:107D700052F8212086FB0272019ED20082FB067619
:107D8000104A52F82120AEEB0202B8E746FA02F29E
:107D90008FE700BFB06C0A00A06C0A00FCFFFF7FF9
:107DA000F0FFFF7FC0FFFF7FE06B0A009979825AE6
:107DB00063218510786B0A00A9BDA0298C6B0A008D
:107DC000C06B0A00A06B0A002DE9F74F00F5A04830
:107DD0004FF0000A476D88F8B4AD88F8AEADB1F148
:107DE000000B816DC0F820A04FF0FF3304464362C2
:107DF0000CBFFF220C22CB1BD019013B04F5DA7615
:107E00008842C8BF1A46236C0092314604F15400E0
:107E10009847009A8242054613D1002F68D1A549A0
:107E20000522304658F09EFF78B1A349052230461E
:107E300058F098FF48B10823E361002003B0BDE883
:107E4000F08F0623F8E70123F6E7B4F8BA31236090
:107E5000A360B4F8BC316360E36094F8BE31C3F34F
:107E600002120132A261BBF1000F40F0BB8194F815
:107E7000BF2188F8B02D180688F8AFBD4BD503F0A8
:107E8000070B0BF1010B4FF0030A05F5DA710AFA43
:107E90000BFA236C5246214404F1540098470544E0
:107EA00098F8B50D01282DD804F58D520221123213
:107EB00001FA0BF1A44611449CF8C1319CF8C2E1CF
:107EC000DB084FEA9E0EDB0243EA4E139CF8C3E147
:107ED00043EADE0300B15BBA22F8023F91420CF1A3
:107EE000030CE9D14FF0030A0AFA0BFA0AF10D0A62
:107EF00016F80A302C2B00F0E3803B2B0ED1072321
:107F0000E3616FE104F58D50524604F2C111143063
:107F100058F03CFFEAE74FF00D0AE9E7212B40F06B
:107F20009B8006EB0A020AF102015378FE2B68D00F
:107F3000FF2B21D0012B5ED0F92B84D1735C042B55
:107F400013D1D17888F8AF1D5079137903EB002352
:107F50000A204343012BD8BF64232362C90744BFCF
:107F6000937988F8B13D0AF108018A46C0E70AEB27
:107F70000301BAF1000FF8D016F801A04B1CA5EBD5
:107F8000030B0AF11F025A4515DB01F2B5115A46DF
:107F900021443046009358F024FF009B0BF5DA7122
:107FA0001F440AF12002236C214404F15400984735
:107FB00000230BEB0005BAF10B0FD8D106EB030B36
:107FC0003E4900935246584658F0CCFE009B03F1C0
:107FD0000B010028D0D19BF80B30032BCCD19BF8A0
:107FE0000C30012BC8D19BF80E209BF80D3003EB11
:107FF00002236362C0E7735C4A1C9918002BFAD114
:10800000B3E716F801A04B1CA5EB030B0AF11F0206
:108010005A4515DB01F2B5115A462144304600930A
:1080200058F0DFFE009B0BF5DA711F440AF12002C5
:10803000236C214404F15400984700230BEB000506
:10804000A26B1AB9DA19A263A4F83CA00AEB0301E7
:10805000BAF1000FD5D188E7A36DDB1B202BB4BF8D
:1080600007230123E8E604F5A55006EB0B011430C5
:10807000009258F08BFE009A93447EE0009258F0F4
:1080800085FE009A616B236C114461635144ABEB34
:108090000202214404F1540000929847636B009A55
:1080A00029461A4494E0636C394404F1540098471B
:1080B00098E000BF8C1C0900921C0900841A09007A
:1080C00006EB0A030AF10A0B99785A7802EB0122AF
:1080D00022611979DA7802EB0122626199795A7981
:1080E00002EB01222260197ADA7902EB0122626046
:1080F0005B7A88F8B33D1A0644D503F007030133D1
:1081000005F5DA7103229A4001932144236C009211
:1081100004F15400984798F8B51D009A01290544C8
:10812000A1D8019B04F5A5524FF0020C12324FF07A
:10813000010B0CFA03FC04EB0A000BFA03FB94445A
:1081400090F8BE3190F8BFE1DB084FEA9E0EDB02EB
:1081500043EA4E1390F8C0E143EADE0301B15BBA93
:1081600022F8023F944500F10300E9D10BF1FF3BF7
:108170000BEB4B0B0AF10D0AD34404F5A04301228B
:1081800083F8B42D16F80B30174A04F5A0480BF10C
:10819000010188F8B23DD35CA3610023636341F21F
:1081A000B47A8D421EDD16F801B0606B4B1CEA1AE2
:1081B00050449345204406EB03013FF75FAF5A4616
:1081C000009358F0E3FD626B009B5A440BEB0301F4
:1081D0006263BBF1000FE4D101238D4288F8AE3D0C
:1081E0003FF761AF012029E6C0680A002DE9F0479A
:1081F000002486B0CDE90044614A624E624D0121FF
:1082000013684BB1D6F804330B4205D0A2F5C04039
:1082100080B25FF0CCFF0C430432AA424FEA410126
:10822000EED1584BD3F87C3173B14FF4BE705FF090
:10823000BEFF4FF0A04344F00044D3F81035009344
:10824000524BD3F810350193E3B2D3B1504F01260E
:108250000025344210D0AB0003F1804303F5C04346
:10826000D3F81005D3F8101557F8253023B1C1F312
:108270000141C0F3052098470135082D4FEA460615
:10828000E7D1002C78DA04AE0023049373604FF03A
:10829000FF33029300253F4F0393A84617F9012FA0
:1082A000531C4ED002F03F0402A920465FFA82F927
:1082B0005FF06CFF002844D0354B19194FEA99192B
:1082C00091F9281053F821A0BAF1000F0BD1B9F1A0
:1082D000030F36D1E10802F0070001238340705CF0
:1082E0000343735402E0B9F1030FF3D01F2C8BBF8B
:1082F00002F01F022246254B4FF0A04302F5E07228
:10830000694653F822202046C2F301425FF03EFF47
:1083100030B1022A15D1B9F1030F0CD1494605E05D
:10832000032A0ED1B9F1030F05D10221204637F0FF
:1083300091F90135EDB2BAF1000F02D0494620465D
:10834000D04708F10103022B4FF00108A6D19DB1DF
:108350004FF0A0430099D3F8102503F540739142E4
:10836000D3F8103502D10199994205D00092049AB0
:10837000CDE90132059B8DE706B0BDE8F08700BF6F
:108380000061004000600040206100400003005098
:10839000585B0120AF5B0120D0F80031103B102B5F
:1083A00007D8054A22FA03F313F0010F08BF002093
:1083B00070470020704700BF010101002DE9F04F18
:1083C00004468DB00846FFF7E7FF0D4601900246D0
:1083D000214695F804014DF0B8FD95F80461231D80
:1083E000013E099304F11003F6B20A93627A637BAB
:1083F00062736279627262786271A27A6370A37842
:10840000A270A27BA372A379A271E279A373E3782D
:10841000E270E27AE271E27BE272E3732546224681
:10842000002312F823105148415C02F82310013355
:10843000042BF6D1099B01329342F1D1019A2146D6
:1084400030464DF082FD002E00F08C8095F80080C3
:10845000AB780093404665F0E4F9029065F0E1F9ED
:10846000039065F0DEF96F780B90384665F0D9F926
:10847000024665F0D6F9049065F0D3F9824600987B
:1084800095F803B065F0CDF9059065F0CAF906904E
:1084900065F0C7F98146584665F0C3F9079065F065
:1084A000C0F9089065F0BDF9DDE9023183EA010CFD
:1084B0000B9B069983EA0C0C82EA0C0C8AEA0C0CE2
:1084C00081EA0C0C89EA0C0C009980EA0C0C87EA12
:1084D0000C0C81EA0C0C04995A404A4005998AEA2E
:1084E00002024A40089989EA02024A404240009941
:1084F00088EA02024A408BEA02026A70039A0599EE
:108500005A408AEA02024A4006994A40079989EA93
:1085100002024A40424088EA02027A408BEA0C0C8E
:108520008BEA020B85F800C085F802B0029A53402E
:10853000049A53408AEA030A089A89EA0A0981EAF6
:1085400009035340584000990A9B88EA000887EACB
:1085500008077940E9700435AB427FF477AF013EFC
:10856000F6B243E70DB0BDE8F08F00BFB0310A00AE
:1085700010B54FF08043D3F80443620707D54FF49A
:1085800084705FF020FE10B11E4B1B689847A30655
:1085900008D54FF48A705FF016FE18B11A4B002010
:1085A0001B689847600608D54FF48C705FF00BFE8F
:1085B00018B1154B01201B689847210608D54FF4C8
:1085C0008E705FF000FE18B1104B00201B689847BA
:1085D000E20508D54FF490705FF0F5FD18B10B4B34
:1085E00001201B689847A3050AD54FF492705FF0ED
:1085F000EAFD28B1054BBDE810401B680220184772
:1086000010BD00BFE85C0120EC5C0120F05C0120A3
:10861000DFED0A7A9FED0A7ADFED0A6AA0EE277A8B
:10862000DFED097AE7EE007AB7EE007AA0EE267A5F
:1086300067EE807A87EE870A704700BF6BD30DBC68
:10864000BA132FBDAEE534BF75AA2A3E02480322F5
:10865000002122F05FB900BF00B0004002480422B0
:10866000012122F057B900BF001001400248042246
:10867000022122F04FB900BF0040024008B57E4AF7
:108680007E4B7F498B42C0F0BF807E4B7E4A0021EB
:108690009342C0F0BE804FF08053D3F83021082AB7
:1086A0004ED14FF080420021C2F80C11C2F81011D7
:1086B000C2F8381502F54042D3F80414C2F8201568
:1086C000D3F80814C2F82415D3F80C14C2F82815EE
:1086D000D3F81014C2F82C15D3F81414C2F83015BE
:1086E000D3F81814C2F83415D3F81C14C2F8401586
:1086F000D3F82014C2F84415D3F82414C2F848154E
:10870000D3F82814C2F84C15D3F82C14C2F850151D
:10871000D3F83014C2F85415D3F83414C2F86015E5
:10872000D3F83814C2F86415D3F83C14C2F86815AD
:10873000D3F84014C2F86C15D3F84434C2F870353D
:1087400055F062FB18B1514B514AC3F88C2655F0D5
:108750005BFB18B14F4BFB22C3F8182555F054FBB7
:1087600058B14FF080424FF08051D2F8E43ED1F83A
:10877000581261F30303C2F8E43E55F045FB20B103
:10878000454B4FF40072C3F840264FF08053D3F8A6
:108790003031082B09D14FF08043D3F80024D107A2
:1087A00044BF6FF00102C3F800243C4AD2F888307D
:1087B00043F47003C2F88830BFF34F8FBFF36F8F5D
:1087C0004FF01023D3F80C22D20725D5344B0122C9
:1087D000C3F80425D3F80024002AFBD04FF0102260
:1087E000D2F80C3223F00103C2F80C322C4BD3F830
:1087F0000024002AFBD00022C3F80425D3F800246B
:10880000002AFBD000F0ACFC52F8040B43F8040B38
:1088100038E743F8041B3BE7D3F80022002A03DBC8
:10882000D3F80432002B22DA1D4B0122C3F80425B1
:10883000D3F80024002AFBD04FF010221221C2F8F6
:108840000012D3F80024002AFBD04FF0102312228C
:10885000C3F80422124BD3F80024002AFBD00022D4
:10886000C3F80425D3F80024002AFBD0CAE70D4B37
:108870000D4A1A6040F0D4FD7C760A000000012009
:10888000E40501200006012050690120005000404D
:108890004881030000F000400090024000ED00E03D
:1088A00000E00140000001200090D003014902488F
:1088B00047F070B91C5C01200030004002494FF0C5
:1088C000402047F067B900BF505C012008B5074859
:1088D000D0F8183143B14FF48C715FF060FCBDE803
:1088E0000840034856F043BE08BD00BF00300240B8
:1088F000BC5B012008B50748D0F8183143B14FF4EC
:108900008C715FF04CFCBDE80840034856F02FBE68
:1089100008BD00BF00F00240E05B012073B51F4CB2
:10892000022501A861F0F7F9052812D11C4D4FF47A
:108930000C741C48ADF802400DF1020161F077F9AA
:1089400008B30C2803D1184918485AF029F902B085
:1089500070BD019B032B14D004D8022BE1D100235E
:108960002370DEE7A3F10902022ADAD80A2B06D027
:10897000092B14BF0120022046F0BCFFD1E70020E4
:10898000FAE72570CDE7D5F8B030002BD1D01E68BE
:108990000448D3E9011290473346F6E730690120D5
:1089A000F85C01202859012094180900005C090096
:1089B0000149024857F072BD045C0120009000405C
:1089C0000149024857F06ABD105C012000A0004038
:1089D0000149024863F089BE845C01200020004008
:1089E0000149024863F081BEA85C0120008002407A
:1089F0002DE9F04FBC4BBD4AD3F80013002385B0DE
:108A00001C4601201D4621FA03F6F6070BD552F845
:108A1000236046B100FA03F6344342F82350BFF313
:108A20006F8FBFF34F8F0133192BECD1E10738D58E
:108A3000AD4B0122C3F81425C3F8102500221546BA
:108A4000930003F1804303F51C330132082A5D6073
:108A50009D62F5D1A44BA6485D629D64C3F8585150
:108A6000D3F80024D3F800140A43C3F80024D3F841
:108A70000023C3F808239F4AC3F8042300214FF4BE
:108A8000927258F0C4F99A4A8DF808504023138323
:108A9000138101214FF4807301A8ADF8043017F061
:108AA00015FE14F4006F924D07D08F4BD3F8A83603
:108AB000A5F81631012385F81C31A20204F48006C2
:108AC00035D5894AD2F8143513F4807308D01EB115
:108AD000D2F80034DB0702D408204BF071F90123EF
:108AE000814AD2F81015CF0540F14A8195F81C3122
:108AF0008BB1002385F81C31B5F816319BB24FF4C9
:108B0000E06203930121882301A8ADF80420ADF8A9
:108B1000083017F0DBFD744B4FF44072D3F820356A
:108B20000293012101A8ADF8042017F0CFFD7EB318
:108B30006D4BD3F8006440F201723240F005C3F887
:108B4000002409D50121C3F82C1501A84FF4806336
:108B5000ADF8043017F0BAFD71050FD5624B012254
:108B6000C3F808259A65D3F8002312F4001208BF51
:108B7000C3F854214FF40012C3F80423B20507D5FB
:108B80004FF4A063012101A8ADF8043017F09EFD59
:108B900023022ED5544BD3F88014D3F88424D3F871
:108BA00088E4D3F88CC4D3F89074D3F89464D3F8E1
:108BB0009804D3F89C3411F07F0FD2B201D1052A6A
:108BC00017D04FF4C0688DF808108DF80E00012101
:108BD00001A8ADF804808DF809208DF80AE08DF821
:108BE0000BC08DF80C708DF80D608DF80F3017F0FC
:108BF0006DFD414B23403BB1BFF35B8F3F4B4FF0CB
:108C000000021A70BFF35B8F394FDFF8DCB000262B
:108C1000B8464FF0140AB14606F10C0324FA03F3E8
:108C2000D80726D50AFB06B305EB4611D3F808276B
:108C3000D8F8003013FA82F3C8F80030B1F806C053
:108C400090B2082E1CFA82F24FEA4613CA8000F056
:108C5000A480B8F80820824240F09F80CA88B8F803
:108C6000041092B2914240F2988016B924481AF04A
:108C70001DFD0136092E08F12008CDD1214B2340DE
:108C8000002B00F09480184BD3F86C84C3F86C84EC
:108C9000BFF36F8FBFF34F8F14F480641CBFD3F802
:108CA0008044D3F88064DFF848A01DBFC6F3C01627
:108CB000C4F3C01486F0010626464FF000094FF4B5
:108CC000E06B28FA09F1CA0703D4B9F1000F31D1DA
:108CD00084B3054B142202FB09315FFA89F0D1F805
:108CE0000836DAF810100FE0007002400071024000
:108CF000D42101200514C001FCFB1F00F422012037
:108D00004C7002400004000151FA83F1CAF81010BF
:108D100005EB4911B1F816E05EFA83FCA1F816C024
:108D2000B1F816C0BAF814E01FFA8CFCE6455ED91B
:108D30004BF026F809F10109B9F1080F0AF1200AF0
:108D4000BFD100244FF0010904F1100328FA03F306
:108D5000DB0701D474B96EB105EB44126301D17A1B
:108D6000002955D0D288B98892B2914250D9E0B248
:108D70004BF026F80134082C07F12007E4D116E067
:108D8000002B7FF4C8AE95F82131002B7FF4C3AEE1
:108D90004FF40013C2F80833BDE62B44DA7A8AB9DF
:108DA0004FF0E023D3F8F03DD90700D500BE1A4AB2
:108DB0001A4B136010460023536005B0BDE8F04F16
:108DC00007F088BDDA88A8F8042083F80B90DB88C8
:108DD0008DF808609BB24FF4E062012101A8ADF864
:108DE000042003938DF8099017F070FC41E7C98ABD
:108DF000ADF804B089B260F07F00039100218DF8D6
:108E000008008DF8091001A8012117F05FFC91E717
:108E10002B4483F80A90ADE7BC62012097C9080093
:108E200010B5074CD4F800314BB1064B5B6898473E
:108E300020464FF48071BDE810405FF0B0B910BD1E
:108E400000000140CC5C0120022A2DE9F04159D1FB
:108E50003B4B826883FB02423A4D846985FB046484
:108E600022440A60DFF8F0C042688CFB0242364EB2
:108E7000C46986FB047422444A60026883FB024290
:108E8000046A85FB046422448A60304E026886FBD3
:108E900002422F4C056A84FB05752A44CA604FF0D4
:108EA0006045426885FB0272C76985FB07E73A4463
:108EB0000A61826884FB0272876986FB07E73A448D
:108EC0004A61426983FB02728A6102698CFB027209
:108ED000CA61C26883FB02720A62C36886FB03230D
:108EE0004B62036985FB03238B62436984FB032385
:108EF000CB620023C1E91033C1E90E33C1E90C3361
:108F0000BDE8F081134B902404FB023202F1480EBD
:108F100002F18C0501F14406683250F8043B55F823
:108F200004795EF804CB1C468CFB048441F8044BA6
:108F300087FB0343AA4246F80439EED1E0E700BFBD
:108F4000D8E3CEB8281C3107CD3C410D9A615FC9EA
:108F5000669EA0F638690A0033C3BEB22DE9F84315
:108F60001C4E04468846914600254FF4004746F0C3
:108F70000106B4F85E20ABB29A4205D894F83400EA
:108F8000BDE8F84336F07ABB03F00F0347FA03F36A
:108F900013EA090F14BF0121002120464DF038FECD
:108FA000B4F85E30AAB2A3EB08039A4203DD94F84A
:108FB000340036F091FB94F8610036F08DFB4020D0
:108FC000B04794F8610036F059FB4020B0470135B6
:108FD000CFE700BF90180A00F8B590F86530013B64
:108FE00080F86B3090F866305A1E80F86C20012BA8
:108FF00088BF90F86C304FF000058CBF03F1FF3351
:10900000012380F86D30044680F86E500127856595
:1090100040F2033694F86330EAB293423CD82368B6
:10902000314A934257D002F58052934255D002F50F
:109030008052934253D002F58032934251D002F5D0
:10904000805293421ED10423284850F8332000EB6D
:10905000C300002590F9043001215160002BC2F8B3
:109060000455D160C2F80855C2F810554FF4803548
:10907000C2F8045306DB5A0903F01F0399401C4B46
:1090800043F82210236801224FF47A715A60DA60A3
:10909000C3F840151A60F8BDA36C03EB02131B7BE9
:1090A0001F2B86BF03F01F0312494FF0A04103F5A9
:1090B000E07341F82360A36C94F86D1003EB021386
:1090C0003942187B04D036F007FB7F000135A1E759
:1090D00036F0D4FAF9E70023B6E70123B4E7022318
:1090E000B2E70323B0E700BF0080004094630A00AA
:1090F00000E100E00003005000280CDB43090649B2
:1091000000F01F0020330122824041F82320BFF3EA
:109110004F8FBFF36F8F704700E100E043090649AE
:1091200000F01F0020330122824041F82320BFF3CA
:109130004F8FBFF36F8F704700E100E00028ABBF97
:1091400000F16040054B00F5614000F00F004FEA70
:109150004111B4BF195480F80013704714ED00E0BA
:10916000BFF34F8F0549064BCA6802F4E062134310
:10917000CB60BFF34F8F00BFFDE700BF00ED00E005
:109180000400FA05014B1868704700BF5400012025
:1091900007EE900AF5EEC07AF1EE10FA01D400F075
:1091A00009B808B580F0004000F004F8404261EBD7
:1091B000410108BD70B5FEF79DF80C4B0022044636
:1091C0000D46FEF7B5FAFEF7DFFB0646FEF770F830
:1091D000074B0022FEF7ACFA02460B462046294612
:1091E000FDF728FFFEF7D0FB314670BD0000F03DD3
:1091F0000000F04170B510EE105A25F00044012334
:10920000B4F1FF4FB0EE403A0646036004D320EEBF
:10921000003AB0EE430A70BD34B9DFEDD07AB7EE54
:10922000007A87EE273AF4E7B4F1E45F0BD2002D21
:10923000BEBF4FF0FF330360B1EE400A24F006F8E2
:10924000B1EE403AE5E7002D80F2C682B4F1964FC8
:10925000E3D2B4F17A5F9FEDC25A78D2DFEDBF0A54
:1092600020EE050A002000F015FEF0EE402AF5EE93
:10927000402AF1EE10FAD0D023EE220AB0EEC00A56
:1092800085EE000A23F0E2FFF5EEC02AF1EE10FAB7
:10929000B0EE402A40F1B9804FF0FF33B4F17E5F69
:1092A000336000F09382B4F1804F00F08F82B1EE12
:1092B000433A6B0000F1DE81AA4B9C4200F2F5803C
:1092C000B0EE430A23F0C2FFA74B9C42B1EE400A26
:1092D00040F29D80B7EE007A37EE437A67EE077A68
:1092E000DFEDA26A9FEDA26A9FEDA23AA7EEA66A01
:1092F000DFEDA16AE6EE276A9FEDA06AA6EEA76AF7
:10930000DFED9F6AE6EE276A9FED9E6AA6EEA73A1A
:10931000DFED9D6AE7EE866A9FED9C6AA6EEA76A7E
:10932000DFED9B6AE6EE276A9FED9A6AA6EEA76AD2
:10933000DFED996AE6EE276A23EE073AA6EEA73A32
:10934000F6EE007AA7EE673A33EE003AFFE0B1EEB0
:10935000407AB0EE470A1DF0CFF8B4EE407AF1EE55
:1093600010FA19D0F6EE007A27EE277AB0EE470A07
:109370001DF0C2F837EE400A30EE000AF0EE407AF7
:10938000FEEECF7A17EE903A062B39D8DFE803F0DD
:109390002312121F1F2B2B00DFED807A77EEC37A8A
:1093A00017EE903A03F0010307EE903A9B00B8EEF7
:1093B000E70AE9E7F6EE007A37EEC00ADFED670A62
:1093C00020EE050A00F036FBF1EE402A4FE7F7EEFB
:1093D000007A37EEC00ADFED610A20EE050A0020B0
:1093E00000F058FDF0E7F7EE087A30EE670ADFED9F
:1093F0005B0A20EE050A00F01DFBB1EE400AE3E730
:10940000F0EE007A30EE670AE5E7012346E7644BA9
:109410009C4264D99FED637A33EE477A67EE074A40
:109420009FED616ADFED616ADFED615A9FED615A80
:109430009FED613A64EE877AE7EE866A9FED5F6A98
:10944000A6EEA76ADFED5E6AE6EE276A9FED5D6A2B
:10945000A6EEA76ADFED5C6AE7EEA65ADFED5B6A6F
:10946000E5EEA76ADFED5A5AE6EEA75ADFED596A34
:10947000E5EEA76ADFED585AA7EEA55ADFED575A79
:10948000E5EE275A9FED565AA5EEA75ADFED555A3D
:10949000E5EE275AE5EE876AA6EEE73ADFED527A67
:1094A00094EE863A33EE673A4EE7504B9C4206D92B
:1094B000B0EE007A37EE437A9FED280A0EE74C4B68
:1094C0009C4206D99FED4B7A9FED240A33EE477AF2
:1094D000A4E7F7EE007A33EE673A9FED200A9FED9E
:1094E000467ADFED467ADFED466AE3EE077A9FEDD6
:1094F000457AA7EE837ADFED447AE7EE037A9FEDB3
:10950000437AA7EE837ADFED4D7AE7EE037A9FED9B
:10951000407AE3EE076A9FED3F7AA6EE837ADFEDAD
:109520003E6AE7EE036A9FED3D7AA6EE837AF7EE98
:10953000006AE7EE036A67EE837A87EEA67AFEEEAC
:10954000006AF0EE477AE3EE267A37EE803A002D95
:10955000BFF65FAE32EE433A5BE600BF00000000AC
:10956000DB0F49406666663F1F4A3B3FA283D33705
:10957000679767393F239E3DA1549C3A7E02F23B98
:1095800001F0893D752C3C384584E23834B6053A03
:10959000C66E3D3B1599A83C661AA53E0000004BDF
:1095A00007336D3E0C5BEC3E6B7BA53976F4B7BAA6
:1095B00067F8663A85300DBA521CE63107E7C73BBB
:1095C000474D06BD5EB9F73E27F9A3B9FE7771BBDB
:1095D0003D37933C3C2117BEF7E9AF399916143B50
:1095E000FEFC28BC155A843DCDCDF83D17A6DD3FC5
:1095F0001FA69D3FC316BB3F5E3C5B3C78756A3E31
:10960000AF72D53DB24B7A3FE73ABA3FF400223F02
:10961000DBD5523BDFEF443F2D390840BE2E1D40C5
:1096200067FF0538B435F13ABDD7F536E440DA3C8A
:10963000E6DC153E7ACCA63E5A245C3E3F239EBD16
:10964000D6EE4B3A54BF983C6E0F303EC5D0383FF3
:109650003B2DB23FE8C4D5BAD23D5B3A5C061CBA9A
:10966000FD0C503A610B36BBABAAAA3D1D7FD63E1E
:1096700000000000B4F1824FF7EE002A75D2FDEE33
:10968000C35A1FED197A5FED196A1FED196AF8EEDA
:10969000E57A15EE903A73EE677A033BE7EE876A58
:1096A0001FED1E7AA6EEA77A5FED1F6AE7EE276A26
:1096B0001FED207AA6EEA77A5FED216AE7EE276A12
:1096C0001FED227AA6EEA77A5FED236AE7EE866A9F
:1096D0001FED246AA6EEA76A5FED256AE6EE276A0B
:1096E0001FED266AA6EEA76A5FED276AE6EE276AF7
:1096F00027EE277AE6EEA72A87EE223AB6EE007A20
:10970000A7EE873A042B3FF622AFDFE803F02B28C1
:1097100025220300B1EE087A37EE877AF1EE046A6B
:1097200077EEA66A66EE876AB1EE007A37EE877A40
:1097300027EE267AB0EE080A37EE800A20EE070AF6
:10974000B0EE007A77EE877A27EE800A23F07EFD6E
:10975000FAE5B7EE007AE1E7F7EE006AE4E7B7EE84
:10976000007AE7E7B7EE000AEAE7B0EE430A23F033
:109770006DFDB4F1B94F30EE620A24D2C2EE836AB5
:109780005FED4C5A1FED4C6A66EEA67AB6EE007A93
:10979000A7EEA56A5FED4F5AE6EE275A1FED506A15
:1097A000A5EEA76A5FED515AE6EE275A1FED526A01
:1097B000A5EEA76A33EE477A1FED543AA6EE263A95
:1097C000A7EE003AC3E623EE003AC0E61FED583A92
:1097D000C0E61FED593A1CE5B4F17E5FF9D0B4F153
:1097E000804FF6D01FED5E2A63E500BF7FB510EE17
:1097F000105A834A25F000439342044605D80023BB
:1098000080ED000A4360002022E07E4A93423AD86D
:1098100025F00043002DDFED7C7A7C4A23F00F0316
:1098200018DD934230EE670A09BFDFED797A9FEDCC
:10983000797A9FED797A30EE670A70EE477A30EEEA
:10984000670AC0ED007A30EE470A80ED010A012078
:1098500004B070BD934230EE270A09BFDFED6C7A89
:109860009FED6C7A9FED6C7A30EE270A70EE077AE6
:1098700030EE670AC0ED007A30EE070A80ED010A8B
:109880004FF0FF30E4E7654A93426DD89FED647A6C
:10989000B0EEC00AF6EE007AE0EE077AFDEEE77A67
:1098A000F8EEE76A17EE900ADFED577AA6EEE70AC0
:1098B0001F28DFED587A66EEA77A30EE677A09DC6A
:1098C0005849461E25F0004251F8261022F0FF02AA
:1098D0008A4207D117EE102AC2F3C752C2EBD35205
:1098E000082A02DC84ED007A1BE09FED497AB0EE95
:1098F000406AA6EEC76A70EE467AE6EEC77A9FED3A
:10990000467AD6EE877A36EE677A17EE102AC2F3D9
:10991000C752C2EBE353192B15DC84ED007AB0EE8D
:10992000460A30EE470A002D30EE670A84ED010A40
:109930008EDAB1EE477AB1EE400A84ED007A84ED1A
:10994000010A404284E79FED387AB0EE460AA6EE5F
:10995000C70A76EE407AE6EEC77A9FED347AD6EE05
:10996000877A30EE677ABDE7B3F1FF4F06D330EE6A
:10997000400A80ED010A80ED000A44E7DA15863AD4
:10998000A3EBC25307EE903ABDEEE77ADFED286A0B
:10999000B8EEC77A77EEC77A8DED017A67EEA67AD0
:1099A000BDEEE77AB8EEC77A77EEC77A8DED027A28
:1099B00067EEA67AF5EE407AF1EE10FACDED037A75
:1099C00019D1B5EE407AF1EE10FA16D002232146F5
:1099D00001A800F089F8002DBFF63AAFD4ED007A67
:1099E000F1EE677AC4ED007AD4ED017AF1EE677A90
:1099F000C4ED017AA5E70323E9E70123E7E700BF08
:109A0000D80F493FE3CB1640800FC93FD00FC93F65
:109A1000004435374344353708A3852E800F49432A
:109A200084F9223F645D0A0000A3852E32318D2423
:109A30000000804310EE103A23F00043B3F1485F7A
:109A4000B7EE007A04D2FDEEC07A17EE902ABAB3D0
:109A500060EE006ADFED1C5A9FED1C6A1C4AA6EE00
:109A6000A56A9342DFED1B5AE6EE265A9FED1A6A6D
:109A7000A5EEA66ADFED195AE6EE265A9FED186AA2
:109A8000A5EEA66A60EEC00A26EE266AF6EE007A19
:109A9000E6EE860A66EEA77A04D877EEE07A37EE2D
:109AA000670A70470F4A93429ABF03F17F4306EE5D
:109AB000903AF5EE026A37EE667A77EEE67AECE7F0
:109AC000B0EE470A704700BF4ED747ADF6740F316E
:109AD0009999993E7CF293B4010DD037610BB6BAD7
:109AE000ABAA2A3D0000483F2DE9F04F9246033AC9
:109AF00048BF0AF10402D7B0D2109B46551C2DB2C4
:109B000002910BF1FF31EB0080460DF16809501A0C
:109B10000BF1090CC24F0393AAEBC50500EB0C0631
:109B20004C460028AABF3B5CDFEDC17A07EE903AB5
:109B300000F10100A8BFF8EE677AB042E4EC017AC8
:109B4000EFD142AF08EB8B0309EB8B040193BE46C8
:109B5000DFEDB77A26464046F0EC016A019B36ED10
:109B6000017A9842E6EE877AF6D101318C45EEEC27
:109B7000017A04F10404EBD1A949DFEDAA6A9FED53
:109B8000AA6A531809240593A300049356AB03EB68
:109B9000840212ED140A07EB840006A92246002A6B
:109BA00045DC28463DF05CFDB0EE407AB4EE000A9C
:109BB00027EE000A1CF0A0FCF2EE007AA0EE677A15
:109BC000002DFDEEC77A17EE906AF8EEE77A37EED1
:109BD000677A3EDD06AA601EC5F1080E52F82030F5
:109BE00043FA0EF10E4401FA0EF1591A42F8201010
:109BF000C5F10702114100293ADD002201360DF1BD
:109C0000180E1346944255DC002D03DD012D62D061
:109C1000022D6AD002292BD1B7EE000A30EE477A26
:109C200033B328463DF01CFD37EE407A20E060EE6D
:109C3000267A013AFDEEE77AF8EEE77AA7EEC60A51
:109C4000BDEEC00AA1EC010A30ED010A37EE800A30
:109C5000A5E705D1621E06A951F822100912CAE72C
:109C6000F6EE007AB4EEE77AF1EE10FA20DA00218F
:109C7000B5EE407AF1EE10FA40F08480601E0023C9
:109C80000DF1180E082838DC002B56D10FA901223F
:109C900051F8040DB0B3049B3E1D04EB0B01601C96
:109CA0001E4409EB8101224490422DDD14466BE7EE
:109CB0000221A2E7DEF8000053B920B1C0F58070A0
:109CC000CEF80000012001320EF1040E034699E7A0
:109CD000C0F1FF00F4E704F1FF3E06A850F82E2083
:109CE00002F07F0240F82E2094E704F1FF3E06A820
:109CF00050F82E2002F03F02F4E75EF820200138F1
:109D00001343BFE70132C3E7059B1B5C07EE903AA4
:109D1000F8EE677A4446E1EC017ADFED457A8C464D
:109D2000F4EC015A019B3CED017A9C42E5EE877A06
:109D3000F6D1E6EC017A0130B6E7013C083D06AA0F
:109D400052F82430DBB12846B7EE000A3DF088FC1B
:109D50009FED347A381D4FEA840800EB84002346D7
:109D600006AD002B3CDA2346002B63DBDFF8BCE0BA
:109D7000DFED2F7A07EB830C0025E01A47E0013C6A
:109D8000083DDDE7039BB0EE470AA3EB0A003DF078
:109D900067FC9FED257AB4EEC70AF1EE10FA19DBE5
:109DA000DFED207A60EE277A06AAFDEEE77A083525
:109DB000F8EEE77AA7EEC70AFDEEE77ABDEEC00A35
:109DC00010EE103A42F8243017EE903A013442F87F
:109DD0002430B8E7BDEEC00A06AA10EE103AF6E746
:109DE00055F8232007EE902AF8EEE77A013B67EE5C
:109DF000807A20EE070A60ED017AB2E7FEEC016A94
:109E0000BCEC017A01350A2DE6EE877A01D0854255
:109E1000F4DD56AA02EB800040ED287A013BA3E76F
:109E2000E45D0A000000803B00008043AC5E0A0055
:109E3000000000002FA81FED027A00EB0803224665
:109E4000002A17DAE1B1F1EE477A029BC3ED007AFE
:109E5000DDED2E7A77EEC77A01239C4213DA09B141
:109E6000F1EE677A029B06F00700C3ED017A57B066
:109E7000BDE8F08F73ED017A013A37EE277ADFE71C
:109E8000F0EE477AE1E7B0EC017A013377EE877ABA
:109E9000E3E700BF10EE103A23F00043B3F1485F50
:109EA00004D2FDEEC07A17EE903A5BB320EE007A52
:109EB000DFED157A9FED156AA7EE276ADFED147ABC
:109EC000E6EE077A9FED136AA7EE876ADFED127A56
:109ED00060EE076AE6EE077A30B99FED106AA7EEEA
:109EE000276AA6EE260A704767EEE67AB6EE006AA3
:109EF000E0EE867AD7EE870ADFED097AE6EEA70A6A
:109F000030EE600A704700BFD3C92E2F342FD7B26E
:109F10001BEF3836010D50B98988083CABAA2ABE20
:109F2000ABAA2A3E10EE103A23F00042B2F1465F8F
:109F3000F0EE407A14D2BDEEC07A17EE101A29BBAB
:109F4000431C134306D1F0EEC07AB7EE007A87EED9
:109F5000270A7047012800F09B80BFEE007AF6E7E1
:109F60004C498A4212D3002B9FED4B7AB8BFF1EED9
:109F7000407A37EE677ADFED497AB8BFF1EE600AD2
:109F800077EEE07ADFED460A77EE877A67EEA76A2A
:109F9000DFED445A9FED446A9FED445A3D4926EE59
:109FA000A67A67EEA64AA7EE256A8A42DFED405AF6
:109FB000E6EE075A9FED3F6AA5EE876ADFED3E5A4F
:109FC000E6EE075A9FED3D6AA5EE876ADFED3C5A43
:109FD000E7EE055A9FED3B5AA5EE875ADFED3A5A58
:109FE000E5EE075A9FED395AA5EE875ADFED385A4C
:109FF000E5EE075AB0EE467AA5EEA67AB0EE606AB4
:10A00000A7EE246A9FED337AE6EE260AE4EE870A8D
:10A0100037EEA00A1DD307EE100AF8EEC76A60EE0D
:10A02000005A30EE260A9B1785EE806A03F0020381
:10A03000C3F1010307EE103A36EE606AB8EEC77A54
:10A0400077EEC67AB0EE006AE7EEC66A26EE870AB9
:10A05000704701281CD010EE103A6FF30B0306EE88
:10A06000903A76EEE77A70EEE70AFFEE007A87EE36
:10A07000807AF7EE007A17EE103A6FF30B0300EEDA
:10A08000103AE6EE807AE0EE807AA7EE870A704713
:10A09000704700BF40A12C3FDA0F493F68212233AF
:10A0A000000000005FAE9BB745F4A3388453D93756
:10A0B000C8261A3A16696B3BA427B33C8988083E28
:10A0C0007AC09538B937813948DEBE3A1F37113C1E
:10A0D000D10D5D3DABAAAA3E42084B0802F05532B5
:10A0E00003F05533801AC91A8A08830801F0333106
:10A0F00000F0333002F0333203F033330344881876
:10A1000003EB131300EB101003F00F3300F00F30CC
:10A11000184400EB002000EB0040000E704700BF29
:10A120002DE9F04782B00646DDF828E00846B4463F
:10A130000D46002B4ED18A4214466DD9B2FA82F2F6
:10A1400042B1C2F12003954026FA03F394401D4327
:10A1500006FA02FC260CA7B2B5FBF6F14FEA1C4347
:10A1600006FB115543EA054301FB07F0984209D964
:10A17000E31801F1FF3580F00381984240F200813D
:10A18000023923441B1A1FFA8CFCB3FBF6F006FBC2
:10A1900010334CEA034C00FB07F363450AD914EB78
:10A1A0000C0C00F1FF3580F0ED80634540F2EA8051
:10A1B000A444023840EA0140ACEB030C0021BEF19C
:10A1C000000F04D02CFA02F30022CEE9003202B0D4
:10A1D000BDE8F0878B4209D9BEF1000F01D0CEE96E
:10A1E00000610021084602B0BDE8F087B3FA83F1B0
:10A1F000174600294DD1834202D3B24200F20F81AB
:10A20000B6EB070C60EB030301201D46BEF1000F07
:10A21000DDD0CEE900C5DAE7002A00F098801A46C2
:10A22000B4FA84F3002B40F0AF800B1B270CA6B2CE
:10A230000121B3FBF7F54FEA1C4007FB153340EA59
:10A24000034306FB05F8984507D9E31805F1FF30ED
:10A2500002D2984500F2E8800546A3EB08031FFAF6
:10A260008CFCB3FBF7F007FB10334CEA034C06FB06
:10A2700000F3634508D914EB0C0C00F1FF3602D251
:10A28000634500F2CE803046ACEB030C40EA05405B
:10A2900095E7C1F120058B4022FA05FC4CEA030C3E
:10A2A00000FA01F426FA05F3E84002FA01F943EA5C
:10A2B00004084FEA1C4206FA01FAB0FBF2F71FFA53
:10A2C0008CF602FB17004FEA184444EA004407FBEF
:10A2D00006F0A0420AD91CEB040407F1FF3380F01A
:10A2E0009C80A04240F29980023F6444241A1FFAE5
:10A2F00088F3B4FBF2F002FB104443EA044300FB92
:10A3000006F69E4209D91CEB030300F1FF3480F0EE
:10A3100082809E427FD90238634440EA0740A0FB16
:10A3200009749B1BA3423E46A04664D361D0BEF194
:10A33000000F0AD0BAEB060263EB080303FA05F537
:10A34000CA401543CB40CEE9005300213FE77308D4
:10A3500043EAC1734A08190C41EA02414FEAC67C3C
:10A360009BB2B2FBF4F02646A04627461F2243EAE2
:10A370000143B1FBF4F1A3EB080341EA004158E7C4
:10A380002946FFE6284615E71A46C3F120019C40FE
:10A3900026FA01F320FA01F190400343270C06FA54
:10A3A00002FCB1FBF7F0A6B207FB1015190C41EA4D
:10A3B000054100FB06F58D423BD9611801D28D4263
:10A3C00020D8491B0138B1FBF7F5019505FB06F8CC
:10A3D000019D9BB207FB151143EA0143434526D279
:10A3E000E31805F1FF31C6D24345C4D2A91E234468
:10A3F000C1E7BA459BD2B7EB090664EB0C04013800
:10A40000A04694E7651B29440238B1FBF7F5019596
:10A4100005FB06F8DCE720467FE71F4666E70846AF
:10A42000F4E6A44402382FE7023D234415E70199DE
:10A43000A1E7491BB1FBF7F5019505FB06F8C7E756
:10A440002DE9F0410D4606464EF001FF294640F247
:10A45000FC4058F0B2FB06F10807044690B143688F
:10A4600028469847A36801219B690546984710B183
:10A47000284845F087FFA368394628469B68BDE811
:10A48000F04118472449284657F0D1FC18B390F8FA
:10A490005030D906ECD443F0100380F850303946E0
:10A4A00053F0ACFA96F82A3003F00C03002B90F826
:10A4B000513014BF0122002223F0060343EA420375
:10A4C00080F8513005D190F8503043F0020380F805
:10A4D0005030BDE8F0811149284657F0A8FC0446E9
:10A4E000B0B190F82A309A07C2D443F0020339463B
:10A4F00080F82A3053F025F896F82A1001F00C0164
:10A500000039204618BF0121BDE8F04153F000B8E2
:10A510000348AEE7514209005CBD0900C0BD090017
:10A52000434209002DE9F7430746002608466A46DC
:10A5300001A9019658F0C5F80199022902D82348CB
:10A5400045F00CFF7868012289001DF025FB7E6034
:10A5500080463E81019BB4B2A34206D85B00C7F897
:10A5600004803B8103B0BDE8F083009B184953F899
:10A57000245040F2E742284625F0E4FA686840F2A9
:10A58000E742022125F09CFAA86840F2776125F0A5
:10A5900007FB40F2776347F6FF720E49814656F09B
:10A5A000B5FDE86840F27D6125F0FAFA094940F20C
:10A5B0007D6347F6FF72054656F0A8FD28F8249003
:10A5C00008EB840401366580C4E700BF144009002D
:10A5D000202109000080FFFF2DE9F04F2DED028BB7
:10A5E00091468DB0C268BDF864B0DDF86880BDF8F2
:10A5F0006C501D9C07468A461E46B0EE408A2AB122
:10A6000043689A4200F0B8800FF038FC4BEA05032B
:10A610001F2B09D8BAF1000F7BD1002D00F0A580C7
:10A6200054464FF0040A09E0BAF1000F40F092805E
:10A63000002D00F0938054464FF0080AB9F1000F46
:10A6400000F0978040F20122ADF81820721CADF89E
:10A650001A200022079206A85FF015FB8146002809
:10A6600051D1182201460DEB020056F0D0FBDFED70
:10A67000447A9FED447A444B8DF818A028EE278A3F
:10A680005E43C8EE077A42F210734D4508BFC846D4
:10A69000B6FBF3F64846189BADF8246001260794F4
:10A6A0008DF82D600293ADF80CB0CDF81080ADF8A8
:10A6B0001450B6EE007A77EE877AFCEEE77ACDEDAD
:10A6C000087A4DF0BBF88146E8B9304C06AA02A9D9
:10A6D00020465FF0B2FA8146A8B92D493A4607F103
:10A6E00028000AF065FE9DF97020217830465FF061
:10A6F000D4FA814638B9207831465FF0A0FA814615
:10A7000008B9189BFB6048460DB0BDEC028BBDE854
:10A71000F08F3CB3F0EE0C7AB4EEE78AF1EE10FA6B
:10A720006946204610D807EE906A9FED1A7AF8EE37
:10A73000677AF4EEC77AF1EE10FA05D84CF03AFDDC
:10A740006C464FF0020A79E74CF034FD6C464FF04E
:10A75000030A73E700244FF0060A6FE72C464FF018
:10A760000A0A6BE74FF0010A68E72C464FF0050A2A
:10A7700064E7CDE906996EE74FF01109C3E700BF22
:10A780000024744900401C4440420F00B3050120DE
:10A79000397907006666A63F2DE9F843416099467E
:10A7A0004B680B9F90469A790A9B80F82C20038572
:10A7B0008D7D044605F0300605F0060572B34B6842
:10A7C000D8684EF058F8E0842DB10023C4E902891E
:10A7D000C4E90433A361002384F82D3084F82A30BF
:10A7E000A384089BE361099B23621AB3EFB11B4961
:10A7F000224638460AF0DCFD5DB115F0040118BFB1
:10A80000012160681ABF84F82B10002201220FF08A
:10A81000CFFCDEB1B20616D4012315E04FF6FF736C
:10A82000C3842B4635461E46CEE70C4821460AF027
:10A83000A3FDE1E767B10A49224638460AF0B8FDB0
:10A8400026B17307E8D4022384F82B30BDE8F883DF
:10A85000034821460AF090FDF2E700BF2B8508006F
:10A86000958508002DE9F04F89B081469DF8486034
:10A8700015465FFA81F81C46002B36D043681A79DA
:10A880001B680621C3F800151D4B342101FB023360
:10A8900086F00106022283F82D207201194E4FF036
:10A8A000000AB4F5806F274603A928BF4FF48067DC
:10A8B0004846CDE9047ACDE9065A8DF80CA08DF80A
:10A8C0000D80019200F01AFEB042834603D1E41BD2
:10A8D000019A3D44E5D1D9F8040035F031FA5846E3
:10A8E00009B0BDE8F04F45F033B941460FF0A6FE80
:10A8F000A0420CBF6FF01200204609B0BDE8F08FF7
:10A900001C5C01200000AD0B074A00231168814246
:10A9100001D1184670470133082B02F10402F5D12A
:10A920004FF0FF30704700BFE04601200C4B187815
:10A9300001280DD10B4B1B78FF2B0BD10A4B18684C
:10A94000C20708D4C30308D4800C00F00400704789
:10A950000228F3D17047052070470120FAE700BFB5
:10A96000746901207C690120006101202DE9F0411A
:10A97000094D0746884600244FF6FF7635F8140047
:10A98000B04203D0424639465FF0A9F94434B4F5E9
:10A99000AA7FF3D1BDE8F081A0090120034B53F851
:10A9A000203013B19A6801329A607047BC200120B0
:10A9B00038B5144B53F82040ECB1207934F07CFECC
:10A9C0000546607934F078FEA2790F49E37940EAD0
:10A9D000450000F0030040EA8202A0718A5C134443
:10A9E00094F908205BB29342E37105DBE36801331D
:10A9F000E3600023E37138BD52429342FBDCE3681D
:10AA0000013BF5E70047012079180A002DE9F04FD6
:10AA10000546A7B08A460146002058F0CEF809AC9A
:10AA2000002841D1CDE913000CAA7E21284629F047
:10AA300085FBA94B0F9301224023CDE9102316ABD0
:10AA400012930FAB0E93A54B09940A93002608208E
:10AA5000CDE9050656F0E2F807902046CDE90366F9
:10AA60008DF8206055F081FDDFF880B2374635461D
:10AA70009DF85490B9F1000F13D0204655F075FDA4
:10AA8000B9F15D0F00F092804AD8B9F13A0F3BD886
:10AA9000B9F11F0F14D8B9F10A0F31D8B9F1080F65
:10AAA000E6D88F4845F06EFC0121284628F03AFD93
:10AAB00043680A93002309950B938DF85430C5E73A
:10AAC000A9F12002D2B20123934013EA0B0F40F008
:10AAD0000F81844A1340CBD1B9F1220FE1D1069303
:10AAE0009DF854100029DCD0222940F0A480204693
:10AAF00055F03BFDDDE906102BF002FF81462CE00E
:10AB0000B9F10D0FB4D0CCE7B9F15B0FC9D100207A
:10AB100022F0EEF88146002D3AD04FF0010821E0F6
:10AB2000B9F1740F70D039D8B9F1660F4FD0B9F1BF
:10AB30006E0FB6D19DF85430752BB2D1204655F02A
:10AB400014FD6C28ADD1204655F00FFD6C28A8D11E
:10AB5000204655F00AFD4FF00E09002D00F00E8141
:10AB60004FF00008604B9F4240F0F5804946284670
:10AB700057F071FDB8F1000F3FF47AAF049B002B42
:10AB800040F0F780012101A82BF08EFC049B1D6092
:10AB900048462AF0C1FD4D46074669E7B9F17B0FEB
:10ABA00000F0D580B9F17D0F7FF47BAF002D3FF42D
:10ABB00078AF039B002B00F00081013B049A0393C4
:10ABC00052F8235028462AF0A7FD074650E79DF883
:10ABD0005430612B7FF465AF204655F0C6FC6C28DD
:10ABE0007FF45FAF204655F0C0FC73287FF459AF67
:10ABF000204655F0BAFC65287FF453AF204655F047
:10AC0000B4FC4FF01E09A8E79DF85430722B7FF476
:10AC100048AF204655F0A9FC75287FF442AF204686
:10AC200055F0A3FC65287FF43CAF204655F09DFC11
:10AC30004FF03E0991E75C290CD1204655F095FC78
:10AC40007528014606D86D2808D8622840D06628A5
:10AC500008BF0C2105A862F0FBF935E0A0F16E03F6
:10AC6000072BF7D801A252F823F000BF8DAC0200E9
:10AC700055AC020055AC020055AC0200D5AC020048
:10AC800055AC020091AC020095AC02000A21E1E74C
:10AC90000921DFE74FF000084FF00409204655F086
:10ACA00064FC40F02000A0F130025738D2B2C0B2AC
:10ACB000092A88BF0246B9F1010942EA0818EDD114
:10ACC000414605A862F0D6F9204655F04EFC07E74C
:10ACD0000821BFE70D21BDE7E45509001D05080067
:10ACE0006D2D090001100004505509000020FF03DC
:10ACF000002306939846494605A862F0A9F99DF8F5
:10AD00005490B9F12E0F17D009F0DF03452B13D063
:10AD1000B9F12B0F12D0B9F12D0F0FD0484645F0E5
:10AD200069FA024650B9DDE90610B8F1000F09D002
:10AD3000134657F0B0FEE1E64FF00108204655F00B
:10AD400014FCD8E743460A222DF090FCD6E60020FA
:10AD50002BF07CFCDEE62EB9B8F1000F7FF4A1AE3B
:10AD60004E4685E631464A46284657F0B9F8002651
:10AD700000E7294601A857F06EFC09E7BAF1000F79
:10AD800011D0B9F1000F3FF48CAE039B002B7FF480
:10AD900088AE05A862F0D3F9484627B0BDE8F08F29
:10ADA000204655F0E2FB9DF85450284645F036FA0F
:10ADB0000028F5D1002DE4D073E6A946BAF1000FC2
:10ADC000F1D0E2E7C20713B5044603D5C0F347004C
:10ADD00002B010BD830707D102680E4B9A4203D11F
:10ADE0002AF088FCC0B2F3E7204657F001FC48B1D6
:10ADF00020462AF007FCFCEEC07ACDED017A9DF8E2
:10AE00000400E5E720462AF087FC5E22C18802485C
:10AE100045F0ACFAE42A0900E038090010B50E4804
:10AE200061F013FB3F2815D90C4CA07847F0F6F8D9
:10AE300080B104F1100061F008FB3F28A07805D92B
:10AE4000BDE810400649402247F01CBABDE810405A
:10AE500047F0CAB910BD00BF883501207835012000
:10AE60003835012070B5164B5A78064632B31B7838
:10AE70005B0723D4134B40F6280444431D19EA789A
:10AE8000E2B110341C44204661F0DFFA3F2815D9A6
:10AE9000E87847F0C3F888B1204661F0D6FA3F2839
:10AEA000E87807D90849402201EBC611BDE8704097
:10AEB00047F0E8B9BDE8704047F096B970BD00BFF3
:10AEC000666701205C1001205C0F01202DE9F04F26
:10AED0000546E3B058484EF0C5FC061E09DB574C4A
:10AEE0006388B3F57F7F08D340F2512323803DF080
:10AEF00033F8002063B0BDE8F08F1A1DAA4200F2BB
:10AF00009880591E251D4E486A5C2F2A4FF000027A
:10AF10000CBF6A54EA5405A954F055F9494B074649
:10AF2000186010B11AF09CFF20B940F25133238011
:10AF30003046DCE707F18000059A06A953F0DAFAFB
:10AF400040F2511345F8043C0023C4E9013307469D
:10AF5000E36010B103236370EAE71AAD294606A83F
:10AF600053F0B4FB08B9AB7E93B9002106A853F0A7
:10AF7000ADFB4FF00009A7604F450FD106A852F076
:10AF8000BAFF0023A26863806260E360A361CFE739
:10AF9000294606A853F09AFB0137E3E7294606A89D
:10AFA00053F094FB6B892989C4F8049003F01F02C5
:10AFB0005200480A0192C3F344120092DB0A01F0E6
:10AFC0001F0200F2BC70C1F3431160F08EFF1E4BF4
:10AFD000A0FB0303C4E904032B7B13F0100318BF89
:10AFE00001230DF1820B15BFE360E36000232B68A2
:10AFF000A361584660F0F3F86080824630463CF02A
:10B00000ABFF4FF00008C24502D809F10109B3E7D0
:10B01000AAEB0802042A4FF0000328BF04220BEB1E
:10B0200008010548009303920FF0A0F9039A904499
:10B03000E9E701205EE700BFEC4F012058510120F5
:10B040005C5101206050012000CA9A3BF8B5284BA2
:10B050001D68284B1B681A68012151641B68264A29
:10B06000D3F844650023146814B12179814230D0AB
:10B070000133082B02F10402F5D1F8BD6369A06920
:10B08000E289218AEB1A89B211FA82F2301AA18977
:10B09000B2FBF1F7C3EB034303444FF6FF7001FB30
:10B0A00017228342A16828BF034621F81230238A61
:10B0B000A2899BB2934203D2238A0133238214E0F4
:10B0C000E3899BB20133B3FBF2F102FB1133E3815D
:10B0D0000BE0E379002BD1D034F0EEFA637900F085
:10B0E0000100834201D00023E3716561A661C4E7DA
:10B0F000F0600120A0620120E04601202DE9FF411F
:10B1000004460F464EF0A3F86368DB6853F82750F7
:10B1100040F2FC40294657F050FD064600285CD01E
:10B12000436828469847B36801A95B6880469847FA
:10B13000B36800219B68054640469847B3680021E4
:10B140009B694046984763682849DB6853F82700A5
:10B1500056F06DFEC0B190F85030B0F9382023F0B1
:10B16000100380F85030B0F93C309A421FBFADF860
:10B170000830C38F826BADF80A304FF000031ABF5E
:10B18000019201250025836263681949DB6853F841
:10B19000270056F04CFE064668B190F82A3023F09E
:10B1A000020301A980F82A3017F01AFC0021054695
:10B1B000304652F0C6F96DB194F82A30DB070ED450
:10B1C000019BA361029BE36194F82A3043F00103E1
:10B1D00084F82A3004B0BDE8F0810546B3E704F1F5
:10B1E000180201A9104651F078FBEDE75CBD09009B
:10B1F000C0BD09002DE9F74F404B019000201870A9
:10B200003F4BDFF820A1DFF820C1FF2002EB8109CE
:10B2100018703C493C48144615464FF001084FF061
:10B22000FF32A94520D1013204D0019B002B51D11E
:10B2300014F090FA354E364800220023C6E9002368
:10B2400000231A46A5424BD15AB193ED017ADFEDA6
:10B25000317A67EE277A17EE900AFDF799FFC6E973
:10B26000000103B0BDE8F08F55F8047BBB07D8D1CF
:10B270003B685345D5D17B681A79A2F12003C2F10E
:10B28000200628FA06F608FA03F333433E7A08FA52
:10B2900002FEAEB1DCF804600096DCF8006046EA1D
:10B2A0000E0B009E1E43CCE900B67E7A002EB8D06D
:10B2B000D1E9007647EA0E071E43C1E90076B0E700
:10B2C00046680096066846EA0E0B009E1E43C0E9DB
:10B2D00000B6EAE7104A00231360104A1370A9E78A
:10B2E00021688F0708D10F68874205D112B10C4839
:10B2F00045F048F80B4601220434A3E774690120A5
:10B300007C690120200D0120100D0120280D012055
:10B310004886090000007A44006101202B69012061
:10B320006740090064860900000D0120242B2DE9E7
:10B33000F047884601D8012B06D1FDF723FF1623DD
:10B3400003600020BDE8F087344E0D46294615F80D
:10B35000014B375D17F00807F8D12D2C10D12C7850
:10B3600001278D1C33F0100115D1302C0DD1297817
:10B3700001F0DF01582908D16C78023510230AE06A
:10B380002B2C04BF2C788D1CECE7002BF6D1302C35
:10B3900014BF0A23082307F1004E0EF1FF3E0021DF
:10B3A000BEFBF3F90E4603FB19EAA4F1300CBCF125
:10B3B000090F10D86446A3421EDDB1F1FF3F07D04C
:10B3C000B14516D301D1A24513DB06FB034601218B
:10B3D00015F8014BE9E7A4F1410CBCF1190F01D8B4
:10B3E000373CE8E7A4F1610CBCF1190F04D8573CD5
:10B3F000E1E74FF0FF31EBE74B1C05D1222303605F
:10B40000764632B930469DE707B17642002AF9D038
:10B4100009B105F1FF38C2F80080F3E779750A0039
:10B420002DE9F043344E86460D46284615F8014B6B
:10B43000375D17F00807F8D12D2C10D12C78012793
:10B44000851C33F0100015D1302C0DD1287800F078
:10B45000DF00582808D16C78023510230AE02B2C25
:10B4600004BF2C78851CECE7002BF6D1302C14BFE0
:10B470000A2308234FF0FF380026B8FBF3F803FB3C
:10B4800008F96FEA09093046A4F1300CBCF1090F44
:10B4900010D86446A3421EDDB6F1FF3F07D08045B9
:10B4A00016D301D1A14513DB00FB0340012615F89B
:10B4B000014BE9E7A4F1410CBCF1190F01D8373C6D
:10B4C000E8E7A4F1610CBCF1190F04D8573CE1E79F
:10B4D0004FF0FF36EBE7731C06D12223CEF8003085
:10B4E000304632B9BDE8F08307B14042002AF9D0B6
:10B4F00006B1691E1160F5E779750A002DE9F74F6D
:10B5000080460D4601925FF057FFD8F80430AC4FEB
:10B5100001225A72D8F804301E791C68342303FBC8
:10B520000677002387F82E30EB6803F06043B3F111
:10B53000005F81468B4607D0A248D8F8043000222D
:10B540005A7203B0BDE8F08F9F4BC4F8083397F8E8
:10B550002F3003F0FF0A23B1BB689C48C4F80433C2
:10B56000EBE787F82F20AE46BEE80F0007F10C0C82
:10B57000ACE80F00DEF80030CCF8003087F830A0DF
:10B580006B78C4F888354FF4827120465CF007FE72
:10B590004FF4927120465CF002FEC4F850A5C4F846
:10B5A00040A52B78032B00F2B380DFE803F0729AFA
:10B5B00052022B6903F06043B3F1005FBCD14FF43A
:10B5C0008073C4F800326B68EA68C4F844254FF40D
:10B5D000A871C4F8483520465CF0E1FD4FF4B07125
:10B5E00020465CF0DCFD4FF4A47120465CF0D7FDF2
:10B5F00001232362A360D4F85031002BFBD04FF419
:10B60000A87120465CF0CBFDAB682A69C4F84425DC
:10B61000C4F848356A4B342202FB06336C4A9A6000
:10B620004FF4827308226B4F2978654D03291CBFA4
:10B630000121A15034227243A918AA58002A79D0B6
:10B640008B68C4F80433634B9F4200F0A8806248C3
:10B6500073E76B68EA68C4F84425C4F848352B6979
:10B6600003F06042B2F1005F7FF466AFAA68C4F8ED
:10B6700034354FF48453C4F83825C4F80032504BA5
:10B68000342202FB063340F202229A600123236235
:10B69000C6E701996B68EA68C4F84425C4F84835E0
:10B6A0003422474B89B102FB06334FF48071C4F852
:10B6B0000012474A9A604FF4A47120465CF06FFD77
:10B6C0004FF4A47301222262ACE702FB06334FF46D
:10B6D000007140F20222C4F800129A604FF48273A3
:10B6E000F0E76B68EA68C4F83425C4F838354FF4DD
:10B6F0008053C4F80032324B342202FB063340F24E
:10B7000002229A600123236200224FF482738AE7A7
:10B71000314F4FF48273082286E7D4F8242152B1C6
:10B720004FF4927120465CF03AFD0123236263617D
:10B730004FF4827323441A68002AEED03422D4F8DE
:10B74000C434C4F8C43402FB0651002281F82F200F
:10B750008BB1224A224813F0010F08BF104613F0A4
:10B76000020F02F5803218BF104613F0040F1D4B74
:10B7700018BF1846E1E6204648F086FB00287FF413
:10B7800062AF1648D9E65FF017FE814574EB010100
:10B7900009D2D8F80430144800225A72D1E619F5BB
:10B7A0007A794BF10004D8F804305A7A002AEAD1A9
:10B7B0009B7A042B96BF0D4A084852F82300C0E636
:10B7C0001C5C01200A00AD0B02029C010B00AD0BBA
:10B7D000000204000000AD0B0400AD0B0100AD0B36
:10B7E0000000AE0B0200AE0B0700AD0BC0190A0043
:10B7F000F8B590F82A309B0704462DD4F8BDDB68D5
:10B8000053F8256040F2FC40314657F0D6F9074620
:10B8100068B1436830469847BB6804F108019B68EB
:10B820009847013563689A689542E8D3E6E70B4983
:10B83000304656F0FCFA20B104F1080152F0DEF86F
:10B84000EFE70749304656F0F2FA0028E9D004F154
:10B85000080151F076FEE4E70025E3E75CBD09004E
:10B86000C0BD090090F950301F4A10B5002B836A03
:10B87000B4BF418A018AB0F90C40002B08BF1346BF
:10B880000C44997B8289B9B193F9051011FB02F13F
:10B890005A88114409B2A0F8461093F905205B8834
:10B8A00012FB04331BB29942D2BFA0F84A30A0F871
:10B8B0004A10A0F8463010BD93F9041011FB02F1B4
:10B8C0001A88114409B2A0F8441093F904201B8887
:10B8D00012FB04331BB29942D2BFA0F84830A0F843
:10B8E0004810A0F84430E6E79C05012090F950305C
:10B8F0001F4A10B5002B836AB4BF018A418AB0F990
:10B900000E40002B08BF13460C44997BC289B9B185
:10B9100093F9041011FB02F11A88114409B2A0F83E
:10B92000441093F904201B8812FB04331BB2994284
:10B93000D2BFA0F84830A0F84810A0F8443010BD9D
:10B9400093F9051011FB02F15A88114409B2A0F8CD
:10B95000461093F905205B8812FB04331BB2994211
:10B96000D2BFA0F84A30A0F84A10A0F84630E6E767
:10B970009C05012008B510EE103A23F00042B2F108
:10B980007E5FF0EE405A10D308D19FED2F0ADFED15
:10B990002F7A002BB8BFB0EE670A08BD70EE405A90
:10B9A000DFED297A87EEA50AF7E7B2F17C5F11D2C5
:10B9B000B2F14A5F9FED266A42D920EE000AFCF7F9
:10B9C00027FEDFED247AE0EE657A75EEE75A36EE73
:10B9D000650AE2E7002BB7EE000AF6EE007A14DA09
:10B9E00075EE805A25EEA70AB1EEC06AFCF710FE8C
:10B9F000DFED197AE0EE067A9FED150A77EE867A8A
:10BA000030EE670A30EE000AC7E730EE650A20EE36
:10BA1000270AB1EEC05AB0EE407A15EE103A6FF335
:10BA20000B0305EE903AA5EEE57A75EE257A87EEE2
:10BA3000276AFCF7EDFDA0EE056A36EE250AE1E780
:10BA4000B0EE460AA9E700BF00000000DA0F494047
:10BA5000DA0FC93F6821A2336821A2B308B510EEFE
:10BA6000103A5A00F0EE407A0FD4B7EE007A70EE3A
:10BA7000477ABDE8084037EEA77AA7EEA77AB1EE7D
:10BA8000C70A37EE800A21F035BB23F00043B3F13B
:10BA90008B4F13D2FFEE006AE0EE006ABDE808406B
:10BAA000B1EEE67AF7EE006A37EE007A86EE870AA4
:10BAB000B0EE007A97EE870A21F0C8BB21F0C6FBF2
:10BAC000DFED027A30EE270A08BD00BF1872313F61
:10BAD00030B589B0084611461A4602AB0193194B9E
:10BAE0000093032355F0DFFA1749029D0C2056F00E
:10BAF0003FFE9DF80C30037245609DF810300446FF
:10BB0000EBB128460DF0A6FD606805AA40F2F541AC
:10BB100028F014FB237A5B0043F0010305AA0021FF
:10BB20000120079355F008FC56F06EFD054660684D
:10BB30004DF027FD1DB9217A044844F02BFC204626
:10BB400009B030BDD41B0A0098C409009041090017
:10BB500010B58EB003AB51F8044B0193194B009311
:10BB60000138032323F008FF40F21951606806AA48
:10BB700028F0E4FA237A5B0043F001030893039B67
:10BB8000099340F626130A93049B5B0043F00103DC
:10BB90000B93059B6FF0004293421FBF40F2E642B9
:10BBA0005B000C9243F0010314BF0221012106AA9D
:10BBB0004FF0020018BF0D9355F0BEFB0E200EB0E3
:10BBC00010BD00BFBC1B0A0010B58EB003AB51F80E
:10BBD000044B0193194B00930138032323F0CCFE4F
:10BBE00040F27561606806AA28F0A8FA237A5B0023
:10BBF00043F001030893039B099340F626130A932D
:10BC0000049B5B0043F001030B93059B6FF0004224
:10BC100093421FBF40F2E6425B000C9243F00103E7
:10BC200014BF0221012106AA4FF0020018BF0D9394
:10BC300055F082FB0E200EB010BD00BFA41B0A0001
:10BC400010B596B003AB51F8044B01932D4B009304
:10BC50000138062323F090FE09AA606840F276615D
:10BC600028F06CFA237A5B0043F001030B93039BEB
:10BC70000C93049B0D9344F616430E93059B5B00B7
:10BC800043F001030F93069B6FF00042934235D0BF
:10BC90005B0043F0010344F6E6321193109209234E
:10BCA000032116AA02EB830244F2D60042F8340CB8
:10BCB00016AA02EB8300079A520042F0010240F8F4
:10BCC000302C089A6FF00040824210D016A800EB8A
:10BCD000830044F2A60440F82C4C16A800EB830322
:10BCE000520042F00102013143F8282CC9B209AADE
:10BCF000032055F021FB0E2016B010BD07230221B2
:10BD0000CFE700BF741B0A00F0B58BB008461146A0
:10BD10001A4603AB01931B4B0093072355F0C3F95D
:10BD2000DDE903600E2816D010F0030203D101688C
:10BD3000154B99420CD029F0EFFCC38800931348AF
:10BD400040F28F134FF4917240F2FD2144F00EFB4C
:10BD500001214DF09CFE0E49182056F009FD9DF87A
:10BD600020409DF824109DF81C50069F049A9DF8D1
:10BD700014300573C0E90167447381730261037570
:10BD80000BB0F0BD741C0A0098BE09003D490900C3
:10BD90007CC4090030B58BB004466A464068244D27
:10BDA0004FF4C46128F0CAF900216A46084655F0EC
:10BDB000C3FA56F029FC002831D060686A4640F288
:10BDC0001D3128F0BBF942F6B6330293A3685B003D
:10BDD00043F00103039344F696630493237B5B00D3
:10BDE00043F00103059344F696530693637B5B008F
:10BDF00043F00103079342F6A6421123CDE908233D
:10BE000004216A46002055F097FA23690E2B03D0CF
:10BE1000217D58684DF027FE60680BB030BD04F0FE
:10BE200095FDAB6A002BBFD0012027F0A1FCBBE73A
:10BE3000F85C01202DE9F341054601F134000E467E
:10BE400004F048FD2B88102B05D0112B41D0002089
:10BE500002B0BDE8F081314C002388224FF6FF711B
:10BE600002FB03F7E05B884205D00133052BF7D1D5
:10BE70004FF40877042388225343A988E152E2183B
:10BE80004FF000080E2307F16000D36520442449D9
:10BE900082F85A80A2F87680E21909F089FAC6F889
:10BEA0001880286969696C373C4403C468465DF0B2
:10BEB000E6FEBDF800302A8A9A4202D86A8A9A427F
:10BEC00003D2A88869465DF0C2FE0023F36001201A
:10BED000BEE7AB88114F0024882202FB04F1785A98
:10BEE000984205D00134052CF7D14FF40871042491
:10BEF00039440B4809F072FA88235C433A194FF62B
:10BF0000FF733B53002382F85A30D26D0E2A1EBFB6
:10BF10005360297A1172B361D9E700BFA0090120EB
:10BF20007DF803002DE9F0418AB0084611461A4613
:10BF300005AB0193234B0093052355F0B4F805227C
:10BF4000059802A927F09CFA039EA6F11002102A78
:10BF500003D81D4BD340DB0702D41C4844F012FA2F
:10BF6000069C022C04DC002C04DC194844F0AEF9D9
:10BF7000062CFAD10798DDF80880A0B907461549C4
:10BF80004FF48A7056F0F4FB089B80F80C41C0F81F
:10BF9000103132463B46414605464DF0AAFB284645
:10BFA0000AB0BDE8F081012202A927F069FA002851
:10BFB000E4D0039840F26512102123F081FD029F26
:10BFC000DDE700BF1C1C0A000101010069420900F5
:10BFD0004C3F090038C4090070B588B003AB51F874
:10BFE000045B0193184B00930138022323F0C4FC37
:10BFF0000522039805A927F043FA069CA4F1100234
:10C00000102A03D8114BD340DB0702D4104844F068
:10C01000B9F9DDE9040640B903462846224631460F
:10C020004DF067FB0E2008B070BD012205A927F076
:10C0300027FA0028F0D0069840F26512102123F06C
:10C040003FFD059BE9E700BF0C1C0A000101010050
:10C050006942090010B50446084655F0B6FF0228AB
:10C0600004DC002804DC044844F030F90628FAD146
:10C0700084F80C010E2010BD4C3F090080B584B03F
:10C0800002AF3B1D01931F4B0093054601230E4653
:10C09000002023F071FC3146284646F093FBD7F888
:10C0A000048040462AF0D2F94FEA60094FEA89033A
:10C0B000073323F00703ADEB030D0DF1080A00244D
:10C0C0004C4505D1A4B1104840F2F14144F006F9C5
:10C0D0006100042241F0010140462BF021FD0B4993
:10C0E00040F28E2223F02EFD4AF824000134E7E7C7
:10C0F000294601203246FFF77DF80548214660F0C9
:10C10000DAFB00BF081D0A00184A090098BE0900A2
:10C11000E41C0A0070B505460E46002844D046F0DF
:10C1200051FB324629460020FFF764F800F0A4F9DD
:10C1300000231A4641F0F6FB1C4B9C6A94BB4DF061
:10C14000F7FA78B3FEF7F2FB012818D002280BD1DA
:10C15000174A234656F82340A10702D1216891428D
:10C1600003D001339D42F5D10E2420463CF0FCFA69
:10C1700000F060F820463CF0F7FA204670BD0D4B09
:10C180000D491A78234656F82340A00706D12068A7
:10C19000884203D1606800799042E6D001339D4225
:10C1A000F1D1E1E70E24E3E70E24E6E7F85C012095
:10C1B000488609007C6901206486090010B586B0B4
:10C1C000084611461A4602AB0193114B0093042313
:10C1D00054F069FF40F2DD41029846F0BBFA0D4988
:10C1E00004460C2056F0C4FA9DF8102012B10A48FB
:10C1F00044F0C8F822792F2A01D95CF04FFF9DF84E
:10C2000014209DF80C1001724460427206B010BDFB
:10C21000C41C0A0064860900AE45090010B5044C30
:10C2200023781BB913F096FA0123237010BD00BFC9
:10C230002B690120F8B5344C344A23686FF3172377
:10C2400093421CD04FF480720021314854F0DFFD3E
:10C25000304A00231370304A4FF4403113701A01F2
:10C2600002F180420133082BC2F80419F7D14FF0D4
:10C2700080434FF47C12C3F88429244B2360274E5B
:10C28000274D0024D5E90001D6E90032C4F120078A
:10C2900003430A430120A4F1200100FA01F120FA2E
:10C2A00007F73943A04003400A40134308D0E0B2E7
:10C2B00039F048FE204633F015FB204633F0FAFBF8
:10C2C0000134402CDED11749174800220023C6E96B
:10C2D0000023C5E90023C1E900234FF40033C0F86F
:10C2E0004833D0F80423920308D5C0F80833D0F8B7
:10C2F00044311BB14FF4A2715BF051FF0B4B002096
:10C300000021C3E90001F8BD78690120AF0000AD4C
:10C310007D690120746901207C690120000D0120E4
:10C32000100D0120200D012000400240280D0120A9
:10C33000F0B50E4687B000251446002A5ED08A0765
:10C340005FD10A68414B9A425BD16A464FF48070D4
:10C3500056F070FD10B93E4843F0B8FFDDE90035F6
:10C36000042CA5EB030536D0A30732D12368394A44
:10C37000934208D0384A934205D0384A934202D0BB
:10C38000374A934225D1052203A9204627F078F8A1
:10C39000049BAB4202D0334843F0F4FF9DF81410E5
:10C3A000039C0022402023F02BFC012801D02E48C2
:10C3B000F2E7009B5A19B2F5807F07D82B482A462E
:10C3C0002146184454F0E2FC0E2417E0284843F0BC
:10C3D000A7FF2848C0E7284654F020FC009B5A19C4
:10C3E000B2F5807F044604D820492A46194454F007
:10C3F000CDFC214628462AF0D9F80446204607B04D
:10C40000F0BD3246006800234FF4807127F056F8E3
:10C41000042C064600F1010708D1B7F5807F9CBFC8
:10C42000124B1D5C6D0045F00104E7E7204655F016
:10C43000CCFD4223FF220021044654F067FEB7F5ED
:10C44000807FC3D8094B9C55BEE700BF3454090018
:10C45000FD2F0900A85D0900E455090004550900F5
:10C46000B0590900F73E0900454709007D690120E0
:10C47000B43C0900223A090038B5084BD3E900451D
:10C4800054EA050305D05EF097FF201A65EB010121
:10C4900038BD4FF0FF300146FAE700BF280D0120FC
:10C4A00010B52DED028B88B0084611461A4603AB35
:10C4B00001932D4B0093022354F0F5FDDDE90304B5
:10C4C000B0F10E0218BF0122B4F10E0318BF012310
:10C4D0009A4202D1254843F055FF0E2836D029F064
:10C4E00091F8B0EE408A5EF067FFFBF773F8DFED7E
:10C4F000207A07EE100A0E2CC7EE278A1FD0049868
:10C5000055F004FF04463AF099FC05A93EF090FC72
:10C510009DF81A3001939DF8193000939DF817206B
:10C520009DF818309DF81610BDF8140042F0AAF9D5
:10C53000231A08EE103AB8EEC88A38EE288AB4EE0C
:10C54000E88AF1EE10FA04D50A48C4E79FED0A8A9A
:10C55000C9E70A49082056F00BF980ED018A08B0B6
:10C56000BDEC028B10BD00BFB41C0A00A53E090043
:10C5700000007A44BE3D0900000000004886090022
:10C580001FB5084611461A4603AB0193084B0093AA
:10C59000012354F088FD40F2DD41039846F0DAF8BB
:10C5A0000449082056F0E4F8002043F08FFE00BF55
:10C5B000AC1C0A002C86090010B5094B094C1B68FD
:10C5C00023B1A34202D0084843F0AAFEC0220021B2
:10C5D000064854F01CFC054B43F8044C181F10BDD2
:10C5E0007C550120085C09008D3D09008055012023
:10C5F00010B5084C20681EF0DFF9014610B106485E
:10C6000043F08EFEB422201D54F001FC034B236046
:10C61000204610BD480C0120863D0900085C090039
:10C6200038B51C46084611464FF0021223F06CF94B
:10C63000206840F2DD4146F08DF8094904460820A3
:10C6400056F096F8637905460BB95CF027FD207922
:10C6500032F0D0FF20790CF0EBFD6C60284638BD3D
:10C66000B4C3090008B540684CF0C2FDBDE80840FD
:10C670009FED010A2AF054B83333534037B50546CD
:10C6800040684CF0B5FD304A00230321ADF8063078
:10C69000C2F8F0150121C2F8F435C2F800151946A8
:10C6A0001A0102F1804202F5E0420133082BC2F880
:10C6B0001415C2F81015F3D1234C4FF49053C4F85D
:10C6C00018356B685B79C4F81435C4F810350DF172
:10C6D0000603C4F82C360123C4F830362360D4F89E
:10C6E0000031002BFBD018484FF480715BF057FDF0
:10C6F00001236360144CD4F80431002BFBD01248A2
:10C700004FF482715BF04BFD0123A360D4F8143128
:10C71000002BFBD00C484FF48A715BF040FD0023E6
:10C72000C4F80035C4F81435C4F81035BDF9063026
:10C7300023EAE373181340EA830080B2400040F01C
:10C74000010003B030BD00BF007000401C4608B5BA
:10C75000084611464FF0021223F0D6F840F2DD41B0
:10C76000206845F0F7FF0449042056F001F803481B
:10C77000F02143F0B3FD00BF98C30900184A090037
:10C780002DE9F04F2DED088B8FB009AB01936D4B68
:10C790000093052323F0F0F80021099830F0A8FB5E
:10C7A000002180460A9830F0A3FB044600210B9834
:10C7B00030F09EFBE379012B05460AD1C379012BAA
:10C7C00007D1A268012A04D98368012B01D99A42B2
:10C7D00002D05D4843F0D6FD6621D8F808005BF032
:10C7E000B8FBE66927790590394630465BF040FB97
:10C7F000A368A069013B00FB03603946B0EE40AA84
:10C800005BF036FB0C98EE690E28F0EE40AA28D1BA
:10C81000297930465BF02CFB0D980E28F0EE408A0B
:10C8200022D1A868AB692979013803FB00605BF06D
:10C830001FFBEB690493D8F81C300293059BD4F8D6
:10C840001CB0DB690393B0EE409A4FF00009D8F8B2
:10C8500008304B450BD805980FB0BDEC088BBDE8F0
:10C86000F08F28F0CFFED7E728F0CCFEE1E7029862
:10C8700098F804105BF0FCFA029AD8F81830B4EE7D
:10C88000C0AA1A44F1EE10FAB0EE408A029252DCCD
:10C89000F4EEC0AAF1EE10FA50D4A668D4F818A0AD
:10C8A0002179013E0027F31B012B32D80AFB07B088
:10C8B00006915BF0DDFA069906FB0AB0F0EE40BA8D
:10C8C0005BF0D6FAAB69049A2979079103FB07203C
:10C8D000F0EE409A06935BF0CBFA049A069B079918
:10C8E00006FB0320B0EE40BA5BF0C2FA38EE6B8A6A
:10C8F00030EE4B0A79EEEB9A28EE008A88EE290A90
:10C9000030EE0B0A039BA3EC010A039309F1010922
:10C910009DE707EB530303FB0AB0079106935BF017
:10C92000A7FA069B0799B4EEC80AF1EE10FAB4BF55
:10C930001F461E46B7E7B0EE680AE3E7B0EE490AC5
:10C94000E0E700BF40610A00683309002DE9F04FBD
:10C950002DED048B87B003AB0193504B0093032361
:10C9600023F00AF80398002130F0C2FA8368012B03
:10C97000044640F28C80C679012E02D0484843F02C
:10C9800001FD007930F038FB81460498E5690E28F6
:10C9900057D0002130F0ACFAC779012F834603D17C
:10C9A000A26883689A4201D03E48E8E700799FED8B
:10C9B0003E8A30F021FB82462846DBF81C80C847BF
:10C9C000A3694046EE18F0EE408AD047DBF81830F5
:10C9D000B0EE409A9844A568BD4211D86B1E00EE97
:10C9E000103AF6EE007A28EE278AB8EE400A20EEDA
:10C9F000080A07B0BDEC048BBDE8F04F29F090BEEB
:10CA00003046C847A3694046F0EE409A1E44D047DE
:10CA100078EEA98A30EE499AF0EE486AD9EE286A93
:10CA2000DBF8183007EE907AB8EE677A9844C6EED5
:10CA3000877A0137B0EE409A38EE278AF0EE698A9D
:10CA4000C9E705989FED188A28F0DCFD2846B0EE6E
:10CA5000409AC847A568F0EE408AB54202D828EE51
:10CA6000098ABBE732462179E0695BF0C8F907EE35
:10CA7000906A78EE808AB8EE677A78EEC88A0136D6
:10CA8000C8EE877AF0EE408A38EE278AE5E7074855
:10CA900007B0BDEC048BBDE8F08F00BFD0610A0089
:10CAA000D22C0900DC2C090000000000020080806C
:10CAB0001E280CD03E280AD010F0010307D18207AF
:10CAC00007D10068044BC31A5842584170470120EF
:10CAD00070471846704700BFE42A0900F0B51B28CC
:10CAE0008DB006460C46154672D03CD80E2800F094
:10CAF0009C8004D8042840F2B580002430E010283F
:10CB0000FBD115F0010206D115F00303F5D1296818
:10CB1000704A9142F1D1284655F057FA0122054654
:10CB200009A9204600F024F9102E0A9F3DD1217951
:10CB30000022402023F064F8A3686B4300FB03F15C
:10CB4000E06854F08CF8A368E0606B43A36063680E
:10CB500003F0FF0363601DB1013DC319002F34D101
:10CB600020460DB0F0BD1D28CBD02428C5D1012210
:10CB700003A9284626F084FC002860D0A10712D122
:10CB80002268554B9A420ED1012209A9204600F095
:10CB9000EFF801230093DDE90901DDE9032352F0F9
:10CBA000C5FC00285CD11E24DAE7A1689DF82C00A2
:10CBB000694300F035F9C3680446CFE71846099980
:10CBC0003A4654F0E3F8013DC319002DF6D1C7E70A
:10CBD0000A68424B9A4290D009A90122204600F0EF
:10CBE000C7F806A90522284626F04AFC9DF82C1015
:10CBF0000022402023F004F8A168079DB5FBF0F562
:10CC0000064629449DF82C0000F00AF90446DDE9A7
:10CC10000912C06854F0BAF8E0680A9B069905FB4F
:10CC200006F2184454F0B2F89AE70A682B4B9A427D
:10CC30003FF463AF294620464AF0FCFF90E7EA073D
:10CC400002D5002043F042FBAB0703D12A68214BF9
:10CC50009A42F6D0284655F0CBFC0028A3D0F0E746
:10CC60003E247DE7012209A9204600F081F8012237
:10CC700006A9284626F004FC002894D00B9A012A25
:10CC800021D05A2A21DC20320146089B012B1ED0DC
:10CC90005A2B01DC203301469342D2D123F0020308
:10CCA000642BCED0022E01D00029CAD0079B00935E
:10CCB000DDE90912069B304656F02EF8002814BF15
:10CCC0003E241E244CE74222DDE70021DDE742231B
:10CCD000E0E700BFE42A0900E45509000455090013
:10CCE000F0B5012885B007460E4608D08B0727D13E
:10CCF0000B681C4A934202D01B4A934220D1012266
:10CD000001A9304626F0BCFBD0B1394600224020B4
:10CD100022F076FF029BB3FBF0F100FB01F5AB4282
:10CD200002D0124843F02EFB384600F079F8019902
:10CD300004462A46C06854F029F8204605B0F0BDE4
:10CD4000304629F093FB58B145102946384600F08B
:10CD500067F82B463A46314604464AF0B1FFECE705
:10CD60000546F2E7B0590900E45509002E390900DB
:10CD700070B50D460179044601F07F01164640204A
:10CD8000002222F03DFFE3682B60A26842436A6004
:10CD9000227902F07F02AA602168094A91420BD1F0
:10CDA00094F90420002A01DBB20707D46268C2F3B9
:10CDB000172200FB02332B60002070BD0120FCE72E
:10CDC00004550900074BC1E900300023C1E90233D3
:10CDD000054B02689A4202BF4368C3F317238B6076
:10CDE00008467047185E09000455090038B50D461D
:10CDF0001C4611462846094A22F086FD20682AF082
:10CE00006BFD012D007804D1BDE83840002100F011
:10CE100007B86168BDE83840FFF762BF0400020050
:10CE20007828F8B505460E4602D10F4843F0AAFA15
:10CE300000220146402022F0E3FE0C4B0C4907463D
:10CE4000012D18BF1946102055F092FC057143685A
:10CE500003F0FF030446C0E9013606FB07F053F078
:10CE6000FBFEE0602046F8BD9C390900A85D090082
:10CE7000E455090070B50A79012A05460C460DD122
:10CE8000184955F07EFED4E9022128462CF0F2FA2A
:10CE900028461549BDE8704055F073BE134955F05A
:10CEA0007FFEA368002BF3D01149284655F069FE98
:10CEB0000026A368B34204D80E49284655F061FE07
:10CEC000E6E71EB10C49284655F05BFE3246E168A4
:10CED000207922F06DFF01220146284629F07CFED0
:10CEE0000136E6E744DA0800531A090050DA080070
:10CEF0005BDA080073180900911B09002DE9F04F57
:10CF0000044687B00D4616460AB90025D0E011F058
:10CF100003078068DFF82CA240F0DF800B68814AAD
:10CF2000934240F0DA806A4655F084FF10B97E489B
:10CF300043F0CCF92179042E01F07F013A464FF0FD
:10CF4000400000F0968022F05BFE16F003020546DA
:10CF500055D131688B7B002B42D001EB83031869DC
:10CF6000724B98423CD13179402001F07F0122F090
:10CF700047FEA84202D06E4843F004FA3368534596
:10CF8000D6E9028B38D17368C3F3172905FB09F979
:10CF9000DDE900062368E768361A5345A8EB060664
:10CFA0002FD194F90430002BAFDA002EE3D163685F
:10CFB000C3F3172305FB037705FB08F20BEB09010D
:10CFC00005FB007053F00DFF0199A268009B521AF7
:10CFD00008EB03006A4305FB017105FB007039E0B3
:10CFE000544B99420BD1012DC5D1052203A93046DE
:10CFF00026F046FADDE903B84FF00009C8E74E48CD
:10D0000096E7002ED8DD6368B6EB132F2FD9A16801
:10D0100031446943384653F022FE6368E06066F3AA
:10D020001F2382466360BB4508BF83460098A26801
:10D03000019940443244121A6A4301FB05A105FBE1
:10D0400000A053F0CEFE009805FB08F20BEB09019F
:10D0500000FB05A053F0C5FE6368C6EB132262F324
:10D060001F236360A3683344A3600E2520E0BA4603
:10D07000DCE722F0C5FD2168009B514506461BD127
:10D08000B3F1807F03DB2D492D485FF014FC1020A5
:10D0900055F06EFB054694E80F0085E80F00009AF6
:10D0A00002EB112363F31F216960019B9B1AAB60A4
:10D0B000284607B0BDE8F08F01992079C91AFFF71B
:10D0C000AFFEDDE90032E168D21A0546724306FB85
:10D0D0000311C06853F05AFEEAE700232A460146CE
:10D0E000206826F0EBF923685345024620790ED1DB
:10D0F0006368042E02EB13220BD003067FF505AF05
:10D10000E168334600F07F0023F04AF9ADE7042ED2
:10D11000F6D1E16800F07F0007B0BDE8F04F22F0E3
:10D1200047BE00BF34540900FD2F0900FDCE0200A8
:10D1300083320900B0590900223A0900D7310900A9
:10D14000085009000455090010EE102A08B522F015
:10D150000043B3F17E5FB0EE406A12D319BF76EEA2
:10D16000467A9FED1F7ADFED1F7A9FED1F7A12BF7F
:10D1700087EE276AE0EE077AB0EE676AB0EE460AFD
:10D1800008BDB3F17C5F0BD2A3F50003B3F1645F7C
:10D19000F4D320EE000AFBF73BFAA0EE066AEDE7B7
:10D1A000B0EEC06AB7EE000A30EE460AF6EE007A3C
:10D1B00020EE270AB1EEC06AFBF72AFA002ADFED5B
:10D1C0000B7AA0EE066AB0EE007AE6EE077A9FEDE3
:10D1D000066A36EE676AB8BFB1EE466ACEE700BFB0
:10D1E0000000000000008003DA0FC93F6821A2B3ED
:10D1F0001FB58DED010A019B23F00042B2F18B4F68
:10D2000000EE102A4FEAD3700AD320F01FF8DFEDAA
:10D210001E7A30EE270A08B1B1EE400A05B000BD13
:10D220005B0014D5B7EE007AF0EE476AE0EE006AD4
:10D23000F1EEE67A77EE807AC7EE276AF0EE007AB2
:10D24000E0EE276AB0EE660A20F000F8E3E7B2F1FC
:10D25000665F10D320EE007AF7EE006A37EE266A9A
:10D26000F1EEC67A77EEA67AC7EE276A36EE800A26
:10D270001FF040FFCFE7DFED057A70EE277ACDEDA6
:10D28000037A039BC7E700BF1872313F0000807B21
:10D2900008B5044B1A68044B9A4202D00D2038F0AE
:10D2A0003BFE08BD009C0320EF2978011FB5044612
:10D2B00090B10E2810D000794CF07BFE60B94FF48D
:10D2C000F773039301A9204603AB02AA1AF09EFF4D
:10D2D0000399024843F05EF804B010BDDA49090032
:10D2E000F4EE400AF1EE10FA10B5F0EE407A04D7F1
:10D2F00070EE207AB0EE670A10BD10EE902AB2F1FF
:10D300007E5F03D1BDE8104000F082B810EE103A05
:10D31000940F04F0020444EAD37433F0004308D1BC
:10D32000022C59D09FED317A032C08BFF0EE477ADA
:10D33000E0E732F0004209D1DFED2D7A9FED2D7A42
:10D3400014F0010F08BFF0EE477AD3E7B2F1FF4FB8
:10D3500010D1B3F1FF4F04F1FF3407D1022C3ED8B6
:10D36000254B03EB8403D3ED007AC3E7022C39D8B5
:10D37000224BF6E702F150619942DDD3B3F1FF4F42
:10D38000DAD0A10703D503F1506393420CD387EEA3
:10D39000A00AB0EEC00A00F03BF8012CF0EE407A93
:10D3A00004D1F1EE407AA5E7DFED157A022C0AD020
:10D3B000002C9FD09FED137A77EE877A9FED127A3B
:10D3C00077EEC77A96E79FED0F7A77EE877A9FED33
:10D3D0000E7A77EE677A8DE7DFED0B7A8AE7DFED7D
:10D3E0000B7A87E7DFED067A84E700BFDB0F49C0E1
:10D3F000DB0FC9BFDB0FC93F385D0A002C5D0A0097
:10D40000000000002EBDBB33DB0F4940DB0F493F5E
:10D4100010EE102A22F00043B3F1994F82B04FEA88
:10D42000D2700ED3B4EE400AF1EE10FA07D69FED9B
:10D43000410ADFED417A002818BFB0EE670A02B05A
:10D4400070473E498B420BD8B3F1665F5AD212F057
:10D45000FF4FF4D160EE007ACDED017A019BEEE74B
:10D46000374A9342F0EEC07A37D8A2F5D002934201
:10D4700029D8F0EE006ABFEE007AA7EEA67A002364
:10D4800077EEA67A87EE270A5A1C60EE006A9FEDB7
:10D490002D6ADFED2D7ADFED2D5A26EEA67AE7EE26
:10D4A000067A9FED2B6AA7EE876ADFED2A7AE7EE10
:10D4B000257A67EE877AE6EE267A67EE807A24D1BF
:10D4C00030EE670ABBE7B7EE007A77EEC76A77EE11
:10D4D000877A012386EEA70AD6E71F4A93420BD824
:10D4E000F7EE086AB7EE007AA7EEA67A022337EEC7
:10D4F000E66A86EE070AC7E7BFEE007A87EE270ADC
:10D500000323C1E74FF0FF33BEE7144A144902EB8F
:10D51000830201EB830393ED007A77EEC77A37EE4F
:10D52000C00AD2ED007A37EEC00A002887D0B1EEEB
:10D53000400A84E7DA0FC93FDA0FC9BFFFFFDF3EB9
:10D54000FFFF973F25AC7C3D0DF5113E4712DABD3C
:10D55000A9AAAA3E98CA4CBEFFFF1B40545D0A0010
:10D56000445D0A002DE9F84FD1F8008001280646F5
:10D5700040468CBF01F1040B4FF0000B0F46914663
:10D5800028F0A4FE30B9404628F0C6F8C1882748E4
:10D5900042F0ECFE06F1FF3AB9F1000F2DD0D9F8B8
:10D5A0000050C5F3DC051AEB050404D02C44A000A0
:10D5B00053F034FB04460022924520D804EB860049
:10D5C0000022954221D11A4EDFF868903168D9F8CF
:10D5D00000000131090153F042FB3368C9F8000033
:10D5E0005A1C32601A0100EB031340F802A0C3E991
:10D5F0000158DC603868BDE8F88F4D46D3E75BF82A
:10D60000223044F822300132D6E7D9F80830083009
:10D6100053F8323040F80C3CD9F8083003EBC20321
:10D6200001325B6840F8083CCBE700BFB548090011
:10D63000845001207C500120F0B50023DFF838E051
:10D640000C4E19460E27DEF80020934201D30E201F
:10D65000F0BD346804EB03124FEA031C9568854261
:10D6600008BF44F80C1003F1010304BFC2E901171D
:10D67000D160E8E77C5001208450012070B590F81B
:10D680002330FF2B04461CD00F4B012200265A608A
:10D69000C3F80065FF2590F8210038F053FC94F89A
:10D6A000220084F8215038F04DFC94F8230084F8CF
:10D6B000225038F047FC054B84F823501E603EF0A2
:10D6C000A1F90E2070BD00BF005002401C5901207E
:10D6D0002DE9F04389B0084611461A4603AB019381
:10D6E000304B0093052353F0DEFC40F2C321039836
:10D6F00045F030F840F269618046049845F02AF818
:10D700004FF44E710746059845F024F840F25C410D
:10D710000646069845F02AF823490546282055F084
:10D720002EF8044625B1214840F25C4142F0D6FD76
:10D730001F4B1D6815B11F4842F0F2FD186098F8A4
:10D7400004009DF81C900BF073FD38790BF070FD10
:10D7500030790BF06DFD184B98F8042084F82120E7
:10D76000C3F864253A7984F82220C3F86825327911
:10D7700084F82320C3F870250122C3F80455C3F8A8
:10D780000855C3F80C25C3F81025C3F81C25C3F8A9
:10D790002055C3F824953EF04FF9204609B0BDE866
:10D7A000F08300BFF81D0A0068C30900184A090089
:10D7B0001C590120BA4409000050024010B504462B
:10D7C00090F823004BF00EFD0A4AD2F8083143B11D
:10D7D00094F8263023F0020384F826300023C2F8A0
:10D7E000083194F8263013F0020F0CBF1E203E20A3
:10D7F00010BD00BF0050024010B5044690F8230051
:10D800004BF0F0FC0C4AD2F8083143B194F82630C2
:10D8100023F0020384F826300023C2F8083194F87C
:10D8200026309A0701D400F009F843F0080384F881
:10D8300026300E2010BD00BF0050024008B5014840
:10D8400042F06EFDDE4009002DE9F04F0D4685B037
:10D8500055F8044B064694F8230017464BF0C2FCDB
:10D8600002AB0193684B0093294602233A46701E8F
:10D8700022F082F8654A0299D2F808319DF80C50DE
:10D8800043B194F8263023F0020384F826300023B5
:10D89000C2F8083194F8263098070BD55B4A01236B
:10D8A000536094F8263043F0040384F82630202394
:10D8B000C2F8083394F82600616065F3041084F818
:10D8C00026000A7BD1F804B0504EDFF84C81D20814
:10D8D00084F825208B7BCD7B497B84F82410003B8A
:10D8E00018BF01235B0143EA8513013A03F060038B
:10D8F00020F0600018BF0122034384F82630C6F8E8
:10D900001C2594F8243042495A1E534253410022A8
:10D91000C6F82835B7EE007A944696461546D6F8EE
:10D920001C35012B01D18B793BB307EE90BA394BF3
:10D93000D1F800A0B1F9047098FBF7F7F8EE676A28
:10D9400003F15809586897FBF0F007EE900AF8EEDB
:10D95000E77A76EEE77AF0EEE77A87EEA66AB4EE3B
:10D96000C76AF1EE10FA05D5D3F800C0B0EE467ADA
:10D970000246D64608339945E4D10135092D01F117
:10D980000801CCD1214DC5F818E5C5F814C594F8A7
:10D99000250094F8243062830BFB00F0584300010B
:10D9A0004FF47A73B0FBF3F0033020F0030080B241
:10D9B000208353F051F9A060208B53F04DF9E060C3
:10D9C00060684AF04FFC0023C4E9043384F8203037
:10D9D00094F8263023F00E0343F00203204684F827
:10D9E00026301BF02FFE238B9B08C5F850352023D3
:10D9F000C5F804330123C5F800352B601BF004FE85
:10DA00000E2005B0BDE8F08FE81D0A00005002406E
:10DA1000A01D0A00481D0A000048E80110B5044690
:10DA200090F823004BF0DEFB064A0123536094F884
:10DA3000263043F0040384F826302023C2F808334C
:10DA40000E2010BD0050024038B5084B1B68002264
:10DA50000446C3F80025FF25007938F073FA607991
:10DA6000257138F06FFA65710E2038BD4002012033
:10DA70002DE9F0432DED028B8BB0084611461A4676
:10DA800003AB01933E4B0093072353F00CFB4FF481
:10DA90004171039844F05EFE40F23B310746049822
:10DAA00044F058FE9DF818506A07064604D04FF41B
:10DAB0003171344842F06EFC9DF820305B0702D093
:10DAC00040F2C641F5E70998DDF814809DF81C90F6
:10DAD00010B327F097FDB0EE408A40F2CF520121FB
:10DAE0000020B0EE480A53F0F3FA2749082054F01A
:10DAF00046FE044638790BF09BFB30790BF098FB1F
:10DB000084F806903A79227133796371B8F57A5FB7
:10DB100005D01E4842F036FC9FED1D8ADDE7102D32
:10DB200001D01C48F6E71C4BDFED1C7A1B681C4932
:10DB3000C3F840256279C3F8442528EE278A4FF0C0
:10DB40000462C3F804250022C3F82025FCEEC87A3D
:10DB50002822C3F81825C3F81C250122C3F8002584
:10DB600017EE900AC3F86015C3F864251A6025F013
:10DB700043FD20460BB0BDEC028BBDE8F08300BF37
:10DB8000101D0A00484909004CC309001130090062
:10DB9000AE47E13D283009004002012000007A44F0
:10DBA000405601202DE9FF411446074600790D46F5
:10DBB0004BF012FB40F24541204621F0F1FF40F2CC
:10DBC00045420021044653F0ADFAAB0706D12A685E
:10DBD0002D4B9A4202D12D4842F078FB062201A932
:10DBE000284625F04DFC9DF80C10029D0022402097
:10DBF00022F006F8B5FBF0F5A54202D2244842F027
:10DC0000C1FB039B482B01D02248F8E7DFF8908046
:10DC1000019DD8F800300122C3F80825C3F86055EB
:10DC2000C3F864451C4B4FF4485043F00103984738
:10DC3000D8F800300022C3F80821184AC3F860253C
:10DC400001222E46C3F86425D8F80030D3F80831F5
:10DC50006BB105EB4405B5420CD1BB7983B124F01F
:10DC60000104640044F0010004B0BDE8F08102F05A
:10DC70006DFEE9E73388A3F5004326F8023BEAE7A7
:10DC800024F00304EDE700BFB00F0A00E9450900E6
:10DC9000CF440900AB360900401E0A00405601205F
:10DCA0004002012070B58AB0084611461A4606ABFC
:10DCB0000193264B0093042353F0F5F906980522AF
:10DCC00003A925F0DDFB059C622C0ED0682C0FD03B
:10DCD000482C1FD0422C01D1002507E0012C1BD07D
:10DCE0001B4840F2E32142F055FB0125012401E0ED
:10DCF000012502249DF8243083B9079B049A6343CD
:10DD00005B00B2FBF3F103FB11223AB1114840F280
:10DD1000E321E8E70025ECE70025EBE70E491820B2
:10DD200054F026FDE4009DF824309DF81C10089A5C
:10DD3000039E0473049CC37300230661857384608F
:10DD40004173426003750AB070BD00BF201E0A0017
:10DD5000624909002D4209002CC309002DE9F04158
:10DD60001C460D4692B0114628467F4A21F0CCFD54
:10DD700026687E4B3340062B05D0B20710D132689F
:10DD80007B4B9A4208D131467A4845F2461253F00D
:10DD9000C9FA8307064603D13268774B9A4202D00C
:10DDA000764842F0DBFA012D26D9062208A96068E0
:10DDB00025F066FB0998089F40F2E3234FF4806248
:10DDC000082121F09DFE05466D49402054F0D0FC0D
:10DDD000044606630022002306F1080050F094F880
:10DDE000206B10226B460DEB0201083050F0BDFB9A
:10DDF00028B1052042F07EFA00252F46E4E7009B7B
:10DE0000102B0BD15F49042204A852F0ABFF28B9B4
:10DE10005D49082206A852F0A5FF18B14FF46B70B7
:10DE200021F09CFD206B04226B460DEB02010830B3
:10DE300050F09BFB0028DCD1009B042B02D1019AFF
:10DE4000282A02D9514842F09DFA206B6B4608A956
:10DE5000083050F08AFB0028CBD1019A282A03D041
:10DE6000BDF82030012B0CD1BDF82210022908D8B2
:10DE7000BDF82E30102B04D8122A04D1BDF8302062
:10DE80008AB14348DFE7282A0DD1BDF820004FF6BC
:10DE9000FE729042F5D1BDF83820012AF1D1BDF8CB
:10DEA00032209A42EDD1082B099A237394BF0023A4
:10DEB0000123A3734FF40073A360002362606173B6
:10DEC000E373206B6B46042202A9083050F04DFB2F
:10DED00000288ED1009E042E8BD12E49324602A8F6
:10DEE00052F040FF8046206B6B46324603A9083053
:10DEF00050F03BFB00287FF47CAF009B042B7FF4A9
:10DF000078AF206B039AB8F1000F0AD0D0E9101354
:10DF1000521843F1000308304FF0F6FF0028D0D02C
:10DF200067E72262036CA38465B94FF48070E062F6
:10DF300052F092FE03462061E06A63B9A561657301
:10DF400042F08AF96D0827612F44E562A7612046F7
:10DF500012B0BDE8F08152F07FFEA0610028F6D13A
:10DF6000E06A25616573EBE7040002000F0080FFA3
:10DF700058290900B8520900B00F0A00D03509002D
:10DF80000CC30900551A09005A1A09008A420900EF
:10DF900079430900AEF708002DE9F04F2DED028B13
:10DFA0008BB0044606920393426A002943D0069B35
:10DFB000012B00D1826A169BA1691960216A237F17
:10DFC000914240F06383D4E90421002B18BF11462D
:10DFD000039B01911960237F83F001032377A369D9
:10DFE0009B08059304F130030893002307930093E3
:10DFF00094F82C30079A93421FDC009B3BB9019A9E
:10E000000599009B02EB8101914240F01F83A37BA5
:10E01000002B00F01E83236A01332362069B002B32
:10E0200040F03B83636A0133636201200BB0BDECB7
:10E03000028BBDE8F08F0691BDE7089B53F8047F83
:10E040000893BB680493002B40F0F282079B0133D6
:10E050000793CDE7BB60009B002B00F0F08201230B
:10E060000093F3E776008E42029A28BF0E4696424E
:10E0700028BF164653E00A469CE055F82C000904D8
:10E08000120431FB00F332FB10F023F3CF3320F303
:10E09000CF30C3EA00434BF82C300CF1010C66453D
:10E0A000EBD10499029B607B497B9B1B88420293C6
:10E0B0000BEB860BD7E9042300D0760802EB86022F
:10E0C0009B1BC7E90423029B002BC8D07B69B3B913
:10E0D0007B7B2BB93B7B002BBCD0B8684AF0C2F8E5
:10E0E000B86860B107F1140207F110014AF075F841
:10E0F0007B699B087B61431E584258417873049AA0
:10E10000637B507B3D697E6998424FEA0321A9D128
:10E11000B14228BF3146029E8E4228BF0E46D4ED42
:10E12000017AB6FBF3F3F8EE677AF7EE000A80EEB9
:10E13000A77ACC4A07F1180007EE903AF8EEE77A92
:10E14000C94B9FEDCA0A67EE877A27EE287AC3ED9E
:10E15000007AC74B83ED007A1378013313705DF0BA
:10E16000FFF9DFEDC40AB0EE408A07F11C009FED15
:10E17000C20A5DF011FADFEDC17A637B28EE278ACF
:10E18000022BBCEEC88A18EE102A91B27FF473AF4E
:10E1900010F4004F47F6FF7209BF121A801892B2AE
:10E1A0004FF400401CBF80B24FF400424A43484342
:10E1B000D213C113049894F80CE090F80DC00098A5
:10E1C000002840F0EF80BEF1100F40F08780A07B68
:10E1D00098B363452ED000980BF10408864686421A
:10E1E0007FF65FAF55F810304FEA034C1CFA83FC02
:10E1F000090431FB0CF1120432FB1CF221F3CF3184
:10E2000022F3CF32C1EA02416FF30F034BF8201023
:10E2100043EA13433EFB03F23EFB13F322F3CF32F8
:10E2200023F3CF33C2EA034248F820200022023011
:10E230001146D4E7DDF800C031E763454AD00098C5
:10E2400026F0010E4FF0802884460BF10409864524
:10E250003FF427AF55F8103093FA48F34FEA034ADA
:10E260001AFA83FA090431FB0AF1120432FB1AF29A
:10E2700021F3CF3122F3CF32C1EA02416FF30F0312
:10E280004BF8201043EA13433CFB03F23CFB13F32F
:10E2900022F3CF3223F3CF33C2EA034249F82020DE
:10E2A000002202301146D2E755F8203093FA4CF3A1
:10E2B0000904120431FB03FE32FB13F32EF3CF3EAD
:10E2C00023F3CF33CEEA03434BF8203001308642AC
:10E2D000EAD1E6E600984FF0802CF8E763454FEA74
:10E2E000460821D1DDF800A04FF08029C245BFF4D7
:10E2F000D8AE35F81A005EF0FFFAA37B0BB990FA9E
:10E3000049F00904120431FB00F332FB10F023F34F
:10E31000CF3320F3CF30C3EA00405AF0DEF82BF8B9
:10E320001A000AF1010AE1E7DDF800A00BF1020989
:10E33000A844A8453FF4B5AE35F8020B5EF0DCFA10
:10E340000346A07B18B94FF0802093FA40F34FEAC0
:10E35000034C1CFA83FC0993080430FB0CF01204F4
:10E3600032FB1CF220F3CF3022F3CF32C0EA02405E
:10E370005AF0B3F8099B29F8020C6FF30F0343EA34
:10E3800013433AFB03F03AFB13F320F3CF3023F3AC
:10E39000CF33C0EA03405AF0A0F8002229F8040B5A
:10E3A0001146C6E7BEF1100F40F0C980A07B0028DF
:10E3B00068D0634539D0043D58464FF0010C4FF00A
:10E3C000000EB445BFF46DAE55F8043F4FEA034864
:10E3D00018FA83F8090431FB08F1120432FB18F231
:10E3E00021F3CF3122F3CF32C1EA024250F8081BA9
:10E3F00092FA11F26FF30F0340F8082C43EA13432B
:10E400003EFB03F13EFB13F321F3CF3123F3CF3374
:10E41000C1EA034250F8043C92FA13F240F8042C8B
:10E4200000220CF1020C1146CBE7ABF1040C0020EA
:10E4300086423FF436AE55F820300904120431FB11
:10E4400003FE32FB13F32EF3CF3E23F3CF33CEEA9A
:10E4500003435CF804EF93FA1EF3CCF8003001306C
:10E46000E6E700BF4469012084620120000000004B
:10E470008062012000FE7F3F00FE7FBF000000475A
:10E48000DB0FC94063453BD0043DDC464FF0010E35
:10E490004FF0802876457FF604AE55F8043F93FA96
:10E4A00048F34FEA034919FA83F9090431FB09F1EA
:10E4B000120432FB19F221F3CF3122F3CF32C1EA39
:10E4C00002425CF8081B92FA11F26FF30F034CF84A
:10E4D000082C43EA134330FB03F130FB13F321F321
:10E4E000CF3123F3CF33C1EA03425CF8043C92FA04
:10E4F00013F24CF8042C00220EF1020E1146C9E76B
:10E50000ABF1040C4FF0802E86423FF4CAAD55F8B3
:10E51000203093FA4EF30904120431FB03F832FB66
:10E5200013F328F3CF3823F3CF33C8EA03435CF85F
:10E53000048F93FA18F3CCF800300130E4E7700050
:10E540006345099049D043190BF1020A09934FF032
:10E550000009099B9D423FF4A4AD35F8020B5EF023
:10E56000CBF98046A07B18B94FF0802398FA43F886
:10E570004FEA084010FA88F0090431FB00F1120458
:10E5800032FB10F221F3CF3122F3CF32C1EA024144
:10E590003AF8020C5EF0B0F991FA10F059F09DFFD4
:10E5A0006FF30F082AF8020C48EA184839FB08F202
:10E5B00039FB18F822F3CF3228F3CF38C2EA0842E9
:10E5C000BAF800005EF098F992FA10F059F085FF61
:10E5D00000222AF8040B1146BBE7ABF102094FF009
:10E5E000000A099B9A45BFF45CAD35F81A005EF04D
:10E5F00083F9A37B1BB94FF0802390FA43F0090401
:10E60000120431FB00F832FB10F028F3CF3820F36E
:10E61000CF30C8EA004839F8020F5EF06DF998FA79
:10E6200010F059F05AFF0AF1010AA9F80000D8E7E2
:10E63000059BDDF804B05FED6E8A029343E5029B13
:10E6400000999A00584652F0E2FB08E542F8043B74
:10E65000DAE4237B059A102B019B03EB82020AD09C
:10E660004FF080309A423FF4D6AC196881FA40F1FD
:10E6700043F8041BF6E74FF080209A423FF4CBACFE
:10E68000196891FA40F143F8041BF6E71BB92369B6
:10E69000039A1360C2E46369FAE7069B012B7FF4D7
:10E6A000C4ACA36A227B0133A362039B1B6803EB08
:10E6B000D203039A1360B8E42DE9F04788B0084606
:10E6C00011461A4602AB0193364B0093062352F0D3
:10E6D000EAFC40F25963FF220121029852F016FD34
:10E6E00040F2F923064602220498012152F00EFD61
:10E6F000079D002D804604DC40F26E51012021F080
:10E70000CDF9DDF814A0BAF1080F05D0BAF1100F59
:10E7100002D0254841F036FE06F10D002349800065
:10E7200054F026F8039F9DF818900446F8088000DE
:10E73000A06152F091FA03462061A0691BB963738E
:10E74000636141F089FD52F087FA606118B9607326
:10E750002061A069F5E765600025A76084F80CA03A
:10E7600084F80E9084F80D80E57384F82C6004F131
:10E770003007B5420ADB94F82C0004F1340128F08C
:10E780005BF92063204608B0BDE8F0870023084805
:10E790001A46194600F062F8013547F8040F446044
:10E7A000E7E700BF7C1F0A007E390900ECC20900C0
:10E7B000601F0A00F0B50C4687B054F8045B0646AB
:10E7C000687B174649F004FD03AB01930E4B0093A1
:10E7D0003A4603232146701E21F0CEF895F82C20EE
:10E7E0009DF810309A4203D84FF4CB6021F0B6F870
:10E7F00005EB83039DF81420586B03990BF04AF83E
:10E80000284607B0F0BD00BF481F0A00F0B50D460E
:10E8100085B055F8044B0646607B174649F0D8FC96
:10E8200003AB01930C4B00933A4601232946701E1B
:10E8300021F0A2F894F82C209DF80C309A4203D8CD
:10E840004FF4CB6021F08AF804EB83040022636B61
:10E850000E209A6005B0F0BD401F0A0010B50846B2
:10E860001146002221F050F80B49202053F080FF80
:10E8700000230446836000F1180140F24642074835
:10E880003EF04CF8064840F2CF4204F11C013EF045
:10E8900045F8204610BD00BF601F0A00020000C0FE
:10E8A000020080801FB502AB51F8044B0193074B67
:10E8B00000930138022321F05FF820469DF80C20D8
:10E8C00002990AF0E7FF0E2004B010BD301F0A00C5
:10E8D0001FB503AB0193064B51F8044B009301386D
:10E8E000012321F049F800230E20A36004B010BDDD
:10E8F000281F0A002DE9F04FAFB0446A04901CB9FC
:10E90000389B1C60022021E0002904998968149139
:10E910003899149C0C60049991F9541008BF002296
:10E920008A42049915D1049891F9551000EB8101A0
:10E93000496B01EB42021A60FF2380F85430389B88
:10E940001A68836D03EB5203836501202FB0BDE885
:10E95000F08F91F84410049CB1FA81F1490984F8D0
:10E96000441084F85510C2F1010204EB810184F8CF
:10E9700054204A6B1A60069252F0DEFA0498002185
:10E9800052F0B5FA049B044670B99A68014606989D
:10E9900052F03DFA389B1C60049B93F8450080F0D0
:10E9A00001004000C0B2D1E7049ADB6A126BD21AB0
:10E9B0000992049A12690392002A01F01685049ABA
:10E9C0000398576A1F44394646F080FE421C0646AB
:10E9D00001F00F85039BD3F80090B9F1000F00F010
:10E9E0003D81D3F80480B8F1000F00F0378199F829
:10E9F00000B099F81C303C18BBF1000F3ED1032B3E
:10EA00004FF0090114BF4FF0200A4FF0110A2AA855
:10EA1000CDE92A4BCDE92CBA5EF09BFEC8F8000088
:10EA200099F81C30032B14BF032105212AA85EF09E
:10EA300090FE454645F8040F039BD3F8BC379B4531
:10EA40000DDB4FF0000B039BD3F8C4379B4580F2DE
:10EA5000C880902303FB0B850023059392E005F10A
:10EA6000100301212AA805935EF073FE059B45F86B
:10EA7000040F9D42F5D10BF1010BDDE7032B4FF0A5
:10EA8000080114BF4FF0110A4FF0090A00232AA809
:10EA9000CDE92B332A94CDF8B4A05EF05AFEC8F825
:10EAA000000099F81C30032B14BF022101212AA871
:10EAB0005EF04FFEC8F80400C3E70C212AA85EF000
:10EAC00048FE0921A8622AA85EF043FE0821E862F8
:10EAD0002AA85EF03EFE286399F80030002B14BF90
:10EAE000092104212AA85EF034FE012168632AA8C6
:10EAF0005EF02FFEA863002856D002212AA85EF0FF
:10EB000028FE0121E8632AA85EF023FE052128647F
:10EB10002AA85EF01EFE052168642AA85EF019FE90
:10EB20000023EB64A86403212AA85EF012FE0321EF
:10EB300028652AA85EF00DFE032168652AA85EF00C
:10EB400008FEEB6BA86533BBC5E90A336B63E86D60
:10EB5000C0F11400286699F80030002B3FD1012144
:10EB60002AA85EF0F6FD686601212AA85EF0F1FD94
:10EB70000121A8662AA85EF0ECFD059BE86601333A
:10EB800005934835039B059AD3F8BC379A4294DB2A
:10EB90000BF1010B57E7022B04D12B6C13B908239F
:10EBA000EB65D4E70723FBE7C5E90F0005212AA899
:10EBB0005EF0CFFD052168642AA85EF0CAFD05213C
:10EBC000A8642AA85EF0C5FD0421E8642AA85EF0C6
:10EBD000C0FD0321E8652AA85EF0BBFDBAE700206E
:10EBE000C1E7039A0999D8F80080C2F8D88706EBE4
:10EBF0000A028A1A03990992D1F8B817039A04EB0A
:10EC00000A05D2F8B02700295AD0002A40F0A48083
:10EC1000039BD3F8CC27099B934280F2AE800699E0
:10EC2000039847F0B6FC4FF0FF34149A0698002181
:10EC300052F0EDF8049B93F845300BB903341BD820
:10EC4000049B06989A68002152F0E1F8389A002354
:10EC50001360049A012382F8453053E6069903981D
:10EC600047F097FC6FF00604049B099A1B6B9B1AF4
:10EC7000049AD362002CD8D1049B149A9B6D03EBA9
:10EC80005203049A9365104652F056F904980021F5
:10EC900052F02DF9049B049A1B6BD26A9A1A049BBA
:10ECA0009B6A9B1AB3F5007F044607DD049AAE4BBE
:10ECB00002F11400C2E9053201F00CFE204645E6DF
:10ECC000002A49D10399DDF824B00122C1F8B02708
:10ECD000A94659464846059347F06FFC431C059BDF
:10ECE00018D019F800C039788C4509EB00021DD105
:10ECF00092F801C079788C4518D197F802C09178C4
:10ED00008CEA0101032911D81CF0020F18BF02F18F
:10ED1000FF32501B039A0028C2F8B4070CDA069998
:10ED2000104647F036FC6FF002049DE7033002F115
:10ED30000309ABEB000BCCE7039A0644D2F8C027DB
:10ED400056445643039AD2F8C8275343039AF60011
:10ED500096FBF3F3C2F8B837039BD3F8B4271B68CC
:10ED600043B15B69003B18BF01231344039AC2F807
:10ED7000CC374DE74FF0FF33F7E7039B0399D3F808
:10ED8000DC37434501F11C003DDBA3EB08014246A3
:10ED900041180A9052F025F8039BD3F8D807D3F80E
:10EDA000CC270A9B2946184451F0F0FF039B039996
:10EDB000D3F8CC27D3F8D8371344C1F8DC37DB00BD
:10EDC0001093039B099903F2DC738A1A1A930023A8
:10EDD00009920C930593039B059AD3F8C4379A4282
:10EDE00081F21E837C235343119390235343199341
:10EDF000119B013B1F93119B08931A9B18930023AF
:10EE00000D939B46FEE32946184451F0BFFF039B38
:10EE10000399D3F8CC27D3F8DC3703981344C1F80F
:10EE2000DC37099B06999B1A09936FF0010447F0A0
:10EE3000B0FB19E7039B1E68002E00F0D4805B68CE
:10EE40000793002B00F0CF80039B9D68002D00F0FE
:10EE5000CA800A9B22930023CDE923330C9A109B8E
:10EE60009A18D31D48BF02F10E03DB1025930C9BAB
:10EE70001BB1194622A85EF06CFC059B31789022EC
:10EE80005A43482303FB0B22079B1A44536BD2F8C7
:10EE90003CC0002940F04E81344810F8136000EB6C
:10EEA0004300BCF1020F477862D1D2F84090B9F12B
:10EEB000000F10D0089B884605EB0309314622A8B5
:10EEC0005EF047FC08F10108B8F1080F09F8010BE2
:10EED000F4D14FF00309119B05EB03080D9B9844F7
:10EEE00009EB49039844314622A85EF032FC3146D2
:10EEF00088F8170022A85EF02CFC314688F818002C
:10EF000022A85EF026FC09F10109B9F1060F88F884
:10EF1000190008F10308E6D1089BEE18394622A82B
:10EF20005EF017FC394686F8290022A85EF011FC35
:10EF3000394686F82A0022A85EF00BFC09F1010987
:10EF4000B9F10C0F86F82B0006F10306E6D1059AFD
:10EF50007C2353433E2202FB0B332B44002283F8D5
:10EF60003B209A8724E000BFA5F80400BC5B0A00A0
:10EF7000059B002B3ED10D9BDDF8148005EB0309AA
:10EF8000314622A85EF0E5FB08F10108B8F10B0F4D
:10EF900009F8010BF4D10D9B1D44394622A85EF0FF
:10EFA000D8FB05F8080008F10108B8F1150FF4D1F5
:10EFB000059B189A90265E434820079B00FB0B6632
:10EFC00033449B6A5360229B0A9A9B1A249AC2EB91
:10EFD000C302D71007D4189B53F804CF1893109B83
:10EFE000634580F2ED810699039847F0D2FA6FF0FD
:10EFF000070439E64FEA0B13079A083302EB0309BB
:10F0000052F80380B8F1000F1FD00D9B8846EB1813
:10F010001F9913F8012B5A5408F10108B8F1060F93
:10F02000F6D1D9F80430FBB9089B4FF0060805EB80
:10F03000030A314622A85EF08CFB0AF8080008F1AA
:10F040000108B8F10B0FF4D121E0089B05EB030A8E
:10F05000314622A85EF07DFB08F10108B8F1060FE9
:10F060000AF8010BF4D1DCE7059C3E2303FB0BF30C
:10F070007C20EA1800FB04332B4491799971D179F3
:10F08000D971117A1972517A5972927A9A72D9F8A1
:10F0900008306BB9089B0B2605EB0308394622A8FC
:10F0A0005EF057FB08F806000136102EF6D112E08C
:10F0B000059C3E2303FB0BF37C20EA1800FB043382
:10F0C0002B44D17AD972117B1973517B5973917B7F
:10F0D0009973D27BDA73D9F80C306BB9089B102680
:10F0E00005EB0308394622A85EF033FB08F806005A
:10F0F0000136152EF6D112E0059C3E2303FB0BF3DF
:10F100007C20EA1800FB04332B44117C1974517CD9
:10F110005974917C9974D17CD974127D1A75059AB1
:10F120007C2353433E2202FB0B332B4400225A75AF
:10F130009A753DE7366A16F0010603D0BBF1010F60
:10F1400000F0B280B3F5C87F7BDA1911052291FB7C
:10F15000F2F2269202EB8202891AC3F3810228920C
:10F1600003F0030300222791299311461346BCF1B3
:10F17000020F40F0CE80059C902060434827079CFA
:10F1800007FB0B002044006C002808BF4FF0010C67
:10F1900001EB41018948614410F821702A9700EB86
:10F1A000810148782B908878C9782C902D910EB3E6
:10F1B000BBF1010F1ED10DF1980C05F1FC070DF10B
:10F1C000A80E664603CE764538607960B44607F1EE
:10F1D0000807F6D10DF1A80C05F58677664603CE33
:10F1E00079602EA98E423860B44607F10807F5D140
:10F1F000C5F8F820059990224A43482101FB0B22CB
:10F2000007990A445366D36B022B40F0C580176CF4
:10F21000002F00F0A880089B0026EF18269922A84E
:10F220005EF097FA0136062E07F8010BF6D14FF083
:10F2300001080327119B05EB030A0D9B0AEB03044E
:10F240008BE0B3F5FA7F12DAA3F5C87399100522A3
:10F25000B1FBF2F2269202EB8202891A03F0030359
:10F260000022279128932992134601217FE7A3F5D5
:10F27000FA730321B3FBF1F101EB410205982691EA
:10F280009B1A0022CDE9282290224243482000FB0D
:10F290000B22079827930244126C0AB1CDE9271379
:10F2A00000220123022162E7B3F5B47F03F00102DB
:10F2B0004FEA630110DA242091FBF0F3269300FB60
:10F2C0001313062093FBF0F100FB11332893002366
:10F2D0002791299303214AE7F3290CDCB4390B1158
:10F2E0002693C1F38103279301F0030100232891A2
:10F2F000299304213BE7F4390323B1FBF3F326936D
:10F3000003EB4303C91A00232791CDE928330521D4
:10F310002DE74FF0000C3BE726AB22A853F828A0BE
:10F3200051465EF016FA5146F07522A85EF011FAC9
:10F330005146307622A85EF00CFA033609F1010935
:10F34000B0752AAB53F828209145E5DB08F1010898
:10F35000B8F1040F3FF4FBAD4F4407EB47062644DA
:10F360004FF00009EDE7B84664E753F8261022A8ED
:10F370005EF0EFF909F8010B013726AB5AF82620A9
:10F380009742F2DB0136042E0DD0B84404EB080995
:10F3900000270DF1A80AF1E7089B4FF00008EC18D0
:10F3A000464626ABF2E7059A7C2353433E2202FBF6
:10F3B0000B331D440023AB756B75F9E5DC5B0A006C
:10F3C000039B1D68002D00F0C2815B680B93002B2E
:10F3D00000F0BD81039B9B68002B00F0B881039B6C
:10F3E000D968002900F0B38102F0070313930C9B46
:10F3F000139AC3EBC70313441C93BCEB030307939B
:10F4000000F1A5810A9B6A6B3B441D930B9B1E4434
:10F41000B36B002B00F02381F36B022B40F01F81B4
:10F42000336C002B40F00381059C9023634300FB69
:10F430000B330B9803440320DB6D013393FBF0F394
:10F4400002EB4303B3F92E0000EB40004FF41072BF
:10F45000059C9023634348250B9C05FB0B332344F9
:10F46000DB6A5B00B3F5107FA8BF4FF410739342C3
:10F47000D4BF2C932C920A932D938342D4BF2B9309
:10F480002B9001EB8B03209303F580530A9AC3F86A
:10F4900000224FF4106303FB0B131593139B0F9380
:10F4A0001D9B0C93002316930E93199B4033E31876
:10F4B00021930E9B169F01332AAA0E9352F82330F4
:10F4C0001693A3EB070EBEF1000F23DD159B0E9ADA
:10F4D0000C9903EB8707219B53F82250B14B03EBA8
:10F4E000C5031E790F9B5A4202F0070213462AB148
:10F4F00011F8010BC2F1200200FA02F2002E40F0D6
:10F50000C08033463A1D47F8263042F8263002368E
:10F51000B645F8DC00230F9A0C991A4401EBE2017E
:10F5200002F007020F92079A0C91D31A07930E9BD1
:10F53000032BBED1109B1C9A9B1A0E93079B002B8A
:10F5400000F09F82159B0A9A0C9803EB8205059A9E
:10F5500090235343482202FB0B330B9AD318924A51
:10F56000DB6E52F823200B92904A52F823100F9B27
:10F570005B4203F007031A462BB110F8016BC3F18D
:10F58000200306FA03F3079CA61A0A9C4FF0000911
:10F59000C4F50F7AC1F120014F460AF1010A0A9120
:10F5A000BA4500F3F081209B03F58052D2F8003277
:10F5B0003B44C2F800320022B3F5107FC0F26382F0
:10F5C000079A0F9B13440C9A02EBE30203F0070324
:10F5D0000C93089B0A923E3308930D9B3E330D9388
:10F5E000199B4833199313461D9A9B1A00F1AF805B
:10F5F000139AC2EBC3030C9A13440E9AD31A1093B6
:10F600000BF1010B039BD3F8BC379B45FFF612AC03
:10F610000599039844F06EFC013040F05785069937
:10F62000039846F0B6FF6FF00904FFF71DBB2B7877
:10F630005BB9059C9023634300FB0B330B98034499
:10F64000DB6D013332F9130000E7B2F93600B2F98D
:10F650003430C31AB2F90C0000EB4300F6E6059B08
:10F6600090255D43482303FB0B550B9B1D44EB6D1D
:10F670002D6E013332F913002B44013332F913207C
:10F68000E6E64B4850F825C04A4800EB4C0017907E
:10F690000798012EA0EB030040F08E80454C34F813
:10F6A0001C6006F00F064FF000094FF0004AC6F14B
:10F6B00020060F2853DD8C46C3F118081CF8025BA6
:10F6C000497805FA08F5C3F1100801FA08F10D436D
:10F6D0002A431033103861460A2BEADD22FA06F578
:10F6E000179C013534F815504FEA153C15F0F00F12
:10F6F00002FA0CF218BF02F0004CA3EB1533C5F36D
:10F7000003181EBF520003F1FF334CEA080815F43A
:10F71000706FC5F3032C1FBF03F1FF3302F00045E8
:10F7200045EA0C0C52004B4511DB47F8088BAEF153
:10F73000020EBEF1000F47F804CCCDDCA3EB0903A9
:10F74000079A0344D31A079A93427FF6E4AE0699C8
:10F75000039846F01EFF6FF00804FFF785BA1D18E6
:10F76000002DF4DD002812DD082891F800C0C8BF84
:10F770004878C3F118080CFA08FCC8BFC3F110039D
:10F7800042EA0C02C9BF98400131024302316B1EAC
:10F790004AFA03F31A404FF00B0905F10B0300205E
:10F7A0009AE700BFB8380A00B45B0A00AC5B0A00F5
:10F7B000DC5A0A00B8390A00A6F1020CBCF1010FAC
:10F7C000C5D8DFF8F0C25CF83580DDF85CC00024F5
:10F7D000129408F101041B94C8F120041E940F2810
:10F7E00027DD8946C3F1180A19F8025B497805FA42
:10F7F0000AF5C3F1100A01FA0AF10D432A43103346
:10F80000103849460A2BEADDBCF8009009F00F09D0
:10F81000C9F1200522FA05F501353CF815505FEADB
:10F82000153A2AD1A3EB090302FA09F20CEB450CB5
:10F83000E8E7C518002D8ADD002812DD082891F8B8
:10F840000090C8BF4878C3F1180A09FA0AF9C8BF7E
:10F85000C3F1100342EA0902C9BF984001310243D3
:10F8600002314FF000406B1E40FA03F30B201A40A8
:10F87000129005F10B030020C4E7C5F30319B9F199
:10F880000F0FA3EB0A0302FA0AF2C5F3032523D1F3
:10F89000032E24D11B9C03EB000C002D0CBFA246B1
:10F8A00004F1010AE2453FF752AF9C46E24552DCC3
:10F8B0000344B3EB0C0006D5581E9C464FF00043A2
:10F8C00003411A4000201E9B22FA03F909F10F0997
:10F8D000ACEB080302FA08F2B9F1000F05D002F010
:10F8E000004C49EA0C095200013B0F2D1DD1032E9B
:10F8F0001CD11B9C1D18AC423FF729AF9C461B9C9A
:10F90000644533DC0344B3EB0C0006D5581E9C461B
:10F910004FF0004303411A4000201E9B22FA03F5DA
:10F920000F35ACEB080302FA08F22DB102F0004CDF
:10F9300045EA0C055200013B129CA342FFF607AFBB
:10F94000AEF1020EBEF1000FC7E9009518DDDDF83B
:10F950005CC0083756E711F8019BCCF1180409FA8E
:10F9600004F942EA09020CF1080C9FE711F8015B67
:10F97000CCF1180A05FA0AF52A430CF1080CBEE787
:10F98000129A9B1ADCE60F2E56DD8446C2F1180E41
:10F990001CF8021B407801FA0EF1C2F1100E00FAB9
:10F9A0000EF001430B431032103E60465745BFF640
:10F9B000F7AD092A7FF7F4AD0A990B9C23FA01F100
:10F9C00021443B4C615C4FEA111C03FA0CF311F02B
:10F9D0000808A2EB11121FBF03F0004802F1FF322A
:10F9E0005B0048F0010811F0040E1FBF03F0004E49
:10F9F00002F1FF325B004EF0010E11F0020C1FBF4E
:10FA000003F0004C02F1FF325B004CF0010C11F0EE
:10FA100001011FBF03F0004102F1FF3241F001017B
:10FA20005B004A45FFF6BFAD45F8108B043745E94A
:10FA300003EC45F8041CB9E7B11800297FF7B3AD12
:10FA4000002E12DD082E90F800C0C8BF4678C2F123
:10FA5000180E0CFA0EFCC8BFC2F1100243EA0C03E8
:10FA6000C9BF96400130334302304A1E4FF0004474
:10FA700044FA02F213404FF00A0901F10A0200268B
:10FA800094E7079F8FE5159941F82320013393E50B
:10FA9000059903982A4645F0EDF901300CD10699F5
:10FAA000039846F076FD6FF00A04FFF7DDB800BF5B
:10FAB0005C5B0A00B8380A000135039BD3F8BC37F9
:10FAC0009D42E5DB039AD268002A00F08684039AFF
:10FAD00052690B92002A00F08084039A926907927F
:10FAE000002A00F07A84039AD2F8C867059A564330
:10FAF000069A5E43022B02EB460640F0E9820B9B1E
:10FB00001193331D089300230E93079B03F50053B5
:10FB10000D930E9B0D9A0799119803F001030F9313
:10FB20000B9B03F580554FF00077D5F8183B0093F9
:10FB3000D2F800220F9B44F07DFED5F81C3B0D9AB5
:10FB4000079911980093D2F800220F9B803100F59D
:10FB5000106044F06FFE0F9B0D9A5B42D2F80022BA
:10FB600003F488631344079A02EB830B4FF0000CF5
:10FB700052F82320DBF85C306046C2FB007C6FF05B
:10FB80007301C3FB017C4FF00076DBF88020DBF8CB
:10FB9000DC300546C2FB0065C3FB01654FF45579B7
:10FBA000DBF80430DBF85820C3FB097C834BC2FB35
:10FBB000037CDBF88410DBF8D820C1FB0965C2FBAD
:10FBC000036541F6D478DBF80830DBF85420C3FB3A
:10FBD000087C7B4BC2FB037CDBF88810DBF8D4206D
:10FBE000C1FB0865C2FB036546F2B86EDBF80C305A
:10FBF000DBF85020C3FB0E7C724BC2FB037CDBF8AE
:10FC00008C10DBF8D020C1FB0E65C2FB03656E4A89
:10FC1000DBF81030DBF84C10C3FB027C6B4BC1FBF4
:10FC2000037CDBF89000DBF8CC10C0FB0265C1FB65
:10FC30000365DBF81420DBF84830C2FB0E7C45F28C
:10FC40008401C3FB017CDBF89420DBF8C830C2FBE5
:10FC50000E65C3FB0165DBF81820DBF84430C2FBFE
:10FC6000087C40F22C71C3FB017CDBF89820DBF8A8
:10FC7000C430C2FB0865C3FB0165DBF81C20DBF860
:10FC80004030C2FB097C7421C3FB017CDBF89C2063
:10FC9000DBF8C030C2FB0965C3FB01650C243846A4
:10FCA0004FF014080CFA04F34CFA08FC20FA08F0A0
:10FCB00040EA030046F060F9089B23F8040C304644
:10FCC00005FA04F345FA08F520FA08F040EA0300C3
:10FCD00046F052F9089B0BF5805723F8020C3B685D
:10FCE0004FF4D0704FF000724FF0000CC3FB002CAB
:10FCF0004FF00073D7F880100026C1FB003641F6A4
:10FD00007C007968C1FB002CD7F88410C1FB003659
:10FD100049F2FC70B968C1FB002CD7F88810C1FB10
:10FD200000362B49F868C0FB012CD7F88C00C0FBCB
:10FD3000013628493D69C5FB012CD7F89050C5FB19
:10FD400001366FF0B3057969C1FB052CD7F8941023
:10FD5000C1FB05364FF41275B969C1FB052CD7F804
:10FD60009810C1FB05366FF0130EF969C1FB0E2C1C
:10FD7000D7F89C101D46C1FB0E5610460CFA04F332
:10FD80004CFA08FC20FA08F040EA030046F0F4F8C8
:10FD9000089B9887284606FA04F346FA08F620FAE4
:10FDA00008F040EA030046F0E7F8089B0A49D887C4
:10FDB00004331293089B043B13930FE0D4F8FFFF26
:10FDC0007CAFFFFF3CB6FDFF78940400C4490200FD
:10FDD0004CE803002464FFFF98340A00D1F840E0A7
:10FDE000DBF80051DBF85C014FF000730022C5FB2B
:10FDF0000E324FF000764C6C4FF00009C5FB0469E1
:10FE0000C4F1000CC0FB0C32C0FB0E69DBF8DC0156
:10FE1000DBF8804115904FF000774FF0000AC4FBEB
:10FE20000E7A4FF00075486C4FF00008C4FB005884
:10FE30001598C0FB0C7AC0FB0E58D1F848E0DBF8EF
:10FE400004C1DBF85801CCFB0E32CC6CCCFB04694E
:10FE5000C4F1000CC0FB0C32C0FB0E69DBF8D8010A
:10FE6000DBF884411590C4FB0E7AC86CC4FB0058C3
:10FE70001598C0FB0C7AC0FB0E58D1F850E0DBF8A7
:10FE800008C1DBF85401CCFB0E324C6DCCFB04698D
:10FE9000C4F1000CC0FB0C32C0FB0E69DBF8D401CE
:10FEA000DBF888411590C4FB0E7A486DC4FB0058FE
:10FEB0001598C0FB0C7AC0FB0E58D1F858E0DBF85F
:10FEC0000CC1DBF85001CCFB0E32CC6DCCFB0469CD
:10FED000C4F1000CC0FB0C32C0FB0E69DBF8D00192
:10FEE000DBF88C411590C4FB0E7AC86DC4FB00583A
:10FEF0001598C0FB0C7AC0FB0E58D1F860E0DBF817
:10FF000010C1DBF84C01CCFB0E324C6ECCFB04690B
:10FF1000C4F1000CC0FB0C32C0FB0E69DBF8CC0155
:10FF2000DBF890411590C4FB0E7A486EC4FB005874
:10FF30001598C0FB0C7AC0FB0E58D1F868E0DBF8CE
:10FF400014C1DBF84801CCFB0E32CC6ECCFB04694B
:10FF5000C4F1000CC0FB0C32C0FB0E69DBF8C80119
:10FF6000DBF894411590C4FB0E7AC86EC4FB0058B0
:10FF70001598C0FB0C7AC0FB0E58D1F870E0DBF886
:10FF800018C1DBF84401CCFB0E324C6FCCFB04698A
:10FF9000C4F1000CC0FB0C32C0FB0E69DBF8C401DD
:10FFA000DBF898411590C4FB0E7A486FC4FB0058EB
:10FFB0001598C0FB0C7AC0FB0E58D1F878E0DBF83E
:10FFC0001CC1DBF84001CCFB0E32CC6FCCFB0469CA
:10FFD000C4F1000CC0FB0C32C0FB0E69DBF8C001A1
:10FFE000DBF89C411590C4FB0E7AC86F1691C4FBD8
:10FFF00000581599C1FB0C7AC1FB0E580C24184609
:020000023000CC
:10000000142102FA04F342FA01F220FA01F040EA64
:10001000030045F0B1FF129B23F8040C3846142767
:100020000AFA04F34AFA07FA20FA07F040EA030052
:1000300045F0A2FF129B23F8020C304609FA04F3A4
:1000400049FA07F920FA07F040EA030045F094FF67
:10005000139BA3F87C00284608FA04F348FA07F833
:1000600020FA07F040EA030045F086FF139B16993B
:10007000A3F87E00129B04331293139B043B13934B
:10008000DE4B40318B420BF5807B7FF4A7AE0D9B9E
:100090000F9AD3F800329B1A0D9A03F00703C2F8A7
:1000A00000320E9B01330E93119B80331193089BFA
:1000B000803308930E9B122B7FF42BAD059B0133ED
:1000C00005931A9B08331A93FEF785BE0025F4E4C6
:1000D000079B4036002703F5005807F001030E93F5
:1000E0000B9B0B98079903F5805300EBC710D3F8CF
:1000F000183B0093D8F8002207F0010344F09AFB64
:1001000007F00103D8F800225B4203F4886313442C
:10011000079A02EB8309002052F82310D9F85C20DB
:100120004FF000730446C1FB04306FF07301C2FB53
:1001300001304FF4557ED9F80420D9F85810C2FB8D
:100140000E30AF4AC1FB023041F6D47CD9F808200A
:10015000D9F85410C2FB0C30AA4AC1FB023046F257
:10016000B865D9F80C20D9F85010C2FB0530A64A62
:10017000C1FB0230A54AD9F81010C1FB0230A44AD5
:10018000D9F84C10C1FB0230D9F81410D9F8482026
:10019000C1FB053045F28401C2FB0130D9F81810CB
:1001A000D9F84420C1FB0C3040F22C71C2FB013065
:1001B000D9F81C10D9F84020C1FB0E307421C2FBC5
:1001C00001300C2402464FF0140A184602FA04F3D8
:1001D00042FA0AF220FA0AF040EA030045F0CCFEA7
:1001E00009F5805126F8400C0A684FF00070002392
:1001F0004FF4D075C2FB050341F67C054A68C2FB8B
:10020000050349F2FC758A68C2FB0503814DCA6883
:10021000C2FB0503804A0D69C5FB02036FF0B305FD
:100220004A69C2FB05034FF412758A69C2FB0503D4
:10023000CA696FF01301C2FB010303FA04F243FA27
:100240000AF320FA0AF040EA020045F095FEDFF8D2
:10025000CCA126F8200CA6F140030D930896DAE90C
:1002600010ECD9F80021D9F85C114FF00070002390
:10027000C2FB0E034FF000754FF0000BC2FB0C5B8E
:10028000CCF10002C1FB0203C1FB0E5BDAE912EC08
:10029000D9F80411D9F85821C1FB0E03C1FB0C5B3E
:1002A000CCF10001C2FB0103C2FB0E5BDAE914ECE6
:1002B000D9F80811D9F85421C1FB0E03C1FB0C5B1E
:1002C000CCF10001C2FB0103C2FB0E5BDAE916ECC4
:1002D000D9F80C11D9F85021C1FB0E03C1FB0C5BFE
:1002E000CCF10001C2FB0103C2FB0E5BDAE918ECA2
:1002F000D9F81011D9F84C21C1FB0E03C1FB0C5BDE
:10030000CCF10001C2FB0103C2FB0E5BDAE91AEC7F
:10031000D9F81411D9F84821C1FB0E03C1FB0C5BBD
:10032000CCF10001C2FB0103C2FB0E5BDAE91CEC5D
:10033000D9F81811D9F84421C1FB0E03C1FB0C5B9D
:10034000CCF10001C2FB0103C2FB0E5BDAE91EEC3B
:10035000D9F81C11D9F84021C1FB0E03C1FB0C5B7D
:10036000CCF10001C2FB0103C2FB0E5B0C24142183
:1003700003FA04F243FA01F320FA01F040EA020022
:1003800045F0FAFD0D9B23F8020F14210D9328462A
:100390000BFA04F34BFA01FB20FA01F040EA0300E8
:1003A00045F0EAFD089B23F8020D0893134B0AF170
:1003B000400A9A4509F580797FF451AFD8F80032A8
:1003C0000E9A01379B1A03F00703122FC8F8003268
:1003D00006F140067FF481AE70E60699039846F078
:1003E000D8F86FF00B04FEF73FBC6FF00404FEF783
:1003F0003BBC6FF00504FEF737BC00BF58380A005D
:10040000D4F8FFFF7CAFFFFF3CB6FDFF78940400FB
:10041000C44902004CE803002464FFFF98340A003A
:100420000024FEF721BC00BF2DE9FF411C460D460C
:1004300028461146424A1FF067FA2768414B3B4065
:10044000062B05D0BA070AD13A683F4B9A4206D12B
:1004500039463E4845F2461250F064FF07460121F6
:10046000384623F05FF8067C16F0010602D03848C3
:100470003FF074FF012D2BD96068062201A922F0FC
:10048000FFFFDDE9015633495C2052F078F9EB07B4
:1004900004461FD50135013EB6F5305F1CD905F580
:1004A00090536563A6F5105605F51055A363656274
:1004B000A6620023C4E90B335DF0D9F8206100285F
:1004C00035D1204649F04EF9234924485CF0F3F930
:1004D0003546D8E7002DDFD14FF40068C4F82880F6
:1004E000404650F0B9FB606228B9204649F03AF91D
:1004F00040463FF0B1FEB6F5105F04D3656305F5E5
:100500009055A563D5E74FF4905050F0A5FB60637C
:1005100028B9204649F026F94FF49050E9E74FF406
:10052000905050F099FBA0630028C2D1F1E720461B
:10053000394609F0EFF9204604B0BDE8F08100BF6C
:10054000040002000F0080FF58290900B85209007A
:10055000D0350900CCC2090029450900DC28090072
:1005600010B50446407B47F033FEA3689FED107A38
:100570005A0800EE102A94F8442004EB820423F079
:100580000103626B13449A4209D1F1EEC77ABDE8C8
:100590001040B8EEC00A87EE800A26F0C1B832F9E2
:1005A000021B07EE901AF8EEE77AA7EEA77AEAE7C1
:1005B0000000000038B504460D46407B47F008FEB9
:1005C00045F246122946044850F0ACFE014620464A
:1005D00009F0A0F90E2038BDB852090038B50D4613
:1005E0000446407B47F0F4FD0121284622F09AFFA3
:1005F000037CDB0702D504483FF0B0FE20462946C5
:1006000009F088F90E2038BDD0350900F0B587B063
:10061000084611461A4603AB0193274B0093032368
:1006200050F041FD40F24241039842F093F840F20D
:100630004D510746049842F099F820490646242077
:1006400052F09DF8BDF814501D49044600220B6875
:10065000D3F80005C0070AD50132042A01F10401CC
:10066000F5D10023A36033B916483FF059FE16496F
:100670008A5C2277F6E70022C3F80C25A3680122E2
:10068000C3F81025A2683B792376C2F86035387923
:1006900008F0CEFD3EB1A26833796376C2F86835C2
:1006A000307908F0C5FDA3682D0A01222046A582F5
:1006B000C3F8002507B0F0BDC4200A00B0C209008D
:1006C0009C180A009047090096180A00F0B50D46DC
:1006D00085B055F8044B0646A068174648F077FDEC
:1006E00002AB0193504B0093701E294602233A46F9
:1006F0001FF042F92046029E9DF80C5049F043F845
:1007000010B1204649F04AF8666084F82050337BE7
:100710007568DB08E376F37B84F82230B37B003B1B
:1007200018BF012384F82130B768737BA37638465D
:1007300040F2E3224FF6FF71BF001FF0CDF93846BB
:1007400050F08AFA94F82230E0601BB9384650F035
:1007500083FA206105F574432333B3FBF5F36B4350
:10076000590801F5740101F51051B1FBF3F14B0883
:10077000A26803F5740303F51053B3FBF1F303EB25
:100780005503B3FBF5F3013BC2F84835A268C2F844
:1007900028354B1EE382A368C3F80815A36801221D
:1007A000C3F81425606847F05DFD204A0023114618
:1007B000106890BB41F823403BF03EF9A368002548
:1007C0000422A5772046C3F8002229464EF053FDA7
:1007D000A368D3F82025C3F84025A368D3F82425BF
:1007E000C3F84425A368C3F80851A368C3F80C51A3
:1007F000A368C3F81051A368C3F81451A368C3F8E1
:100800000451A3680C22C3F80423A26801230E201C
:1008100093606377E57705B0F0BD0133042B02F1F7
:100820000402C5D1CAE700BFB4200A00505001201D
:1008300010B50C4C206890B10B4B1B6883B95AF073
:10084000B7FD236898422368A0EB030038BF00F18E
:10085000FF3040F2EE23984294BF0020012010BDEB
:100860000020FCE72059012070500120024A136843
:1008700023EA00031360704770500120024A136896
:1008800003431360704700BF7050012038B50C4B14
:100890001B78A3B10B4B1B688BB90B4C25685AF026
:1008A00087FD2060236813B923680133236035B9BD
:1008B000064B01221A70064B03F174029A6238BD8E
:1008C00061680120705001202059012060670120DB
:1008D000F85C012010B504460BF03CF9E3681BB945
:1008E0000A4A1168A14203D1BDE810400BF044B997
:1008F000A360074B1968E160196809B119688C6039
:10090000116801B914601C60EEE700BF805001203F
:100910008850012008B50BF01DF9044A1368013B0B
:100920001360BDE808400BF027B900BF74500120E8
:1009300008B50BF00FF9044A136801331360BDE8E2
:1009400008400BF019B900BF745001202DE9F041A7
:10095000134E33680BB3134D0BF0FCF82C681CB12D
:10096000BDE8F0410BF008B90F4A01232B60336852
:10097000346014601BB92B68013B2B60F0E7D3E9AE
:1009800000689F68C3E902440BF0F6F80EB14046D8
:10099000B0470BF0DFF83B46ECE7BDE8F08100BF65
:1009A00080500120745001208850012008B524F0A7
:1009B000B3FEC1880348972914BF972242223FF013
:1009C000D5FC00BFB438090010B5064A002352F820
:1009D0003340844202EBC30101D90133F7E7486891
:1009E00010BD00BF58190A00F0B595B0054601A822
:1009F0000E4617461C4657F09DFB10B1002015B05F
:100A0000F0BD3A46314628461FF05CFA2EF0C4FD90
:100A1000830703D10268034B9A42EFD02060012084
:100A2000EDE700BF30290900014A042333F09CBBE5
:100A3000B0300A00F0B587B0084611461A4602AB3E
:100A40000193254B0093042350F02DFB23491820DC
:100A500051F095FEDDE904230361214B9A428CBFDE
:100A60000123B3FBF2F3C3601E4BD3F8A431DDE9DD
:100A7000027604465BB317F07FF880F00105EDB213
:100A800004F11503009300222B4640F277513846BB
:100A900010F0FEFA04F1160360600022009340F2A9
:100AA0007A512B46304610F0F3FA01221146A0602D
:100AB000606810F071FB0122A068114610F06CFB19
:100AC000204659F046FF20B905203FF013FC0125D0
:100AD000D6E7204607B0F0BD94200A0094C2090072
:100AE00020A10700F85C0120F0B50C4687B054F84F
:100AF000045B06462846174648F084FB284648F023
:100B00008EFB02AB0193094B00933A462146701EBF
:100B100004231EF031FF059B00932846DDE90323E3
:100B2000029958F084FC0E2007B0F0BD74200A0032
:100B3000F0B50C4687B054F8045B064628461746C5
:100B400048F060FB284648F06AFB02AB01930A4B71
:100B500000933A462146701E04231EF00DFF012328
:100B60000193059B00932846DDE9032302995CF07D
:100B70000FFD0E2007B0F0BD54200A00F0B50C4662
:100B80008BB054F8045B06462846174648F03AFBFB
:100B9000284648F044FB03AB01930E4B00933A46C2
:100BA0002146701E07231EF0E7FE00230193079BDA
:100BB0000093DDE90312069B28465CF0E9FC099BE3
:100BC00000932846089B059A039958F030FC0E20A4
:100BD0000BB0F0BD1C200A00F0B50D4687B055F8EB
:100BE000044B06462046174648F00CFB204648F0CA
:100BF0001CFB02AB0193204B00933A462946701E22
:100C000004231EF0B9FE40F2E943012200210398BB
:100C100050F07CFA40F2D943012200210646C5B2C9
:100C2000049850F073FA40F2CA23092208210746BB
:100C3000059850F06BFA0299104AB2FBF1F301FBF0
:100C4000132202B101332361237DC3F38002AA4240
:100C50000AD066F3820323756B1E594260684FF019
:100C60000002594110F098FA237D0E2067F3C30368
:100C7000237507B0F0BD00BFE41F0A0020A10700E4
:100C80002DE9F04186B0084611461A4603AB0193A0
:100C90002D4B0093032350F006FA2C49182051F0F5
:100CA00067FD2B4B059ED3F8A431DDE9038704468D
:100CB000002B47D016F060FF80F00105EDB204F183
:100CC0001503009300222B4640F20331404610F0FA
:100CD000DFF9217D60600022C1F3800110F05CFA31
:100CE00004F11603009301222B4640F2914138464D
:100CF00010F0CEF9227DA060B0F10E0318BF0123E1
:100D000063F341029307227503D50022114610F0C8
:100D100043FA04F11703009301222B4640F282416B
:100D2000304610F0B5F905232361237DE06023F000
:100D30000D030E2818BF43F001032046237506B0AB
:100D4000BDE8F0810125BAE704200A0078C2090055
:100D5000F85C01202DE9F04F0D468DB055F8044B9D
:100D600006462046174648F04DFA204648F05DFA00
:100D700008AB01934A4B009329460423701E3A4660
:100D80001EF0FAFD062205A9089822F079FB9DF8CD
:100D90001C10002240201EF033FF099B04930546DF
:100DA000069B0A99B3FBF0F303AA04A8039357F038
:100DB000D9F9049E039B6E435D4304960395002D71
:100DC0004BD0237DDF0704D4364840F282413FF008
:100DD000E1FA9807DDF814A0DDF82C90276940D4DB
:100DE000554406EB0A0835445FFA89F64FF0080BC4
:100DF0004FF0000A237D990703D5A068F1094BF055
:100E00008BFB217D0A0735D438462EF061FD217D0C
:100E1000606881F00401C1F380014BF07DFB0DF1AE
:100E20000B01E0684BF05FFB9DF80B30217D43EA3E
:100E30004A0A0B072BD438462EF04AFD217D606804
:100E4000C1F380014BF068FB7600BBF1010BF6B2F9
:100E5000D0D108F801AB4545C6D10E200DB0BDE894
:100E6000F08FA06800214BF057FB0028B8D1052077
:100E70003FF040FAC1F3800181F00101606801F0A8
:100E800001014BF049FB38462EF022FDC7E76068B0
:100E9000C1F380014BF040FB38462EF019FDD3E73B
:100EA000AC1F0A00AC4109002DE9F04F0D468BB094
:100EB00055F8044B06462046174648F0A3F920464D
:100EC00048F0B3F907AB0193444B00932946032341
:100ED0003A46701E1EF050FD052204A9079822F024
:100EE000CFFA9DF81810002240201EF089FE089BC2
:100EF00003930546059B0999B3FBF0F302AA03A8E7
:100F0000029357F02FF9039B029A6B4355430393C7
:100F10000295002D5AD0227D920704D4304840F229
:100F200091413FF037FA049AD4F8109002EB03088D
:100F3000002798F800604FBBA068F1094BF0ECFA6D
:100F4000002847D0BA46217D0B0708F1010B24D4B5
:100F500048462EF0BDFC217D606881F00401C1F39C
:100F600080014BF0D9FA48462EF0B2FC217D606832
:100F7000C1F380014BF0D0FA0AF1010ABAF1080F6F
:100F800021D07600F6B203E0D846D2E74FF0000A4F
:100F9000A068F1094BF0C0FAD5E7C1F3800181F0F8
:100FA000010101F0010160684BF0B6FA48462EF0ED
:100FB0008FFC217D6068C1F380014BF0ADFA48469B
:100FC0002EF086FCD8E70137BD42DDD10E200BB0F4
:100FD000BDE8F08F05203FF08DF900BFCC1F0A005F
:100FE000AC4109002DE9F04F0D4697B055F8044B80
:100FF00006462046174648F005F9204648F015F900
:1010000010AB0193614B009329460623701E3A46AC
:101010001EF0B2FC05220DA9109822F031FA9DF8BD
:101020003C10002240201EF0EBFD129B1399099307
:1010300005460E9BB3FBF0F308AA09A8089357F0E6
:1010400091F806220AA9119822F01AFA9DF8301098
:10105000002240201EF0D4FD149B159907930646EC
:101060000B9BB3FBF0F306AA07A8069357F07AF898
:10107000089A099B06996B435543079A0993724353
:101080004E43B54208950792069602D040483FF07D
:1010900079F9002D76D00D99C8180390207D860728
:1010A00006D4CE1826B140F291413A483FF072F989
:1010B0000A9EC00706EB020A05D4BAF1000F02D05F
:1010C00040F28241F1E7CE5CA068D4F810B0F1099B
:1010D0004BF022FA00283BD105203FF00BF97600B7
:1010E000F6B2A068F1094BF017FA217D0A0733D454
:1010F00058462EF0EDFB217D606881F00401C1F3BC
:1011000080014BF009FA0DF11701E0684BF0EBF9A3
:101110009DF81730217D43EA49090B0729D4584629
:101120002EF0D6FB217D6068C1F380014BF0F4F90D
:1011300008F10108B8F1080FD1D10AF8079001377A
:10114000BD421FD0039B4FF00008DE5DC146C8E7DB
:101150000027B846B946C8E7C1F3800181F0010114
:10116000606801F001014BF0D7F958462EF0B0FB52
:10117000C9E76068C1F380014BF0CEF958462EF004
:10118000A7FBD5E70E2017B0BDE8F08F1C210A00A1
:1011900048390900AC4109000E2AF7B506460D464C
:1011A000174602D133483FF06DF8806848F00FF8D9
:1011B000AA0706D12A68304B9A4202D12F483FF045
:1011C00085F8EB071FD5B288F3885343B3EB650F5F
:1011D0004FEA650405D8013B00225C2128483FF016
:1011E00069F894FBF2F502FB1544042F24B22DB2EA
:1011F0002AD12A462146304648F061FC400040F0A2
:10120000010003B0F0BD01AA0221284624F0BCF978
:10121000019B186850F0D9FE041EB38801DB9C4284
:1012200004DB013B002240F27761D7E7019B58685D
:1012300050F0CBFE051EF38801DB9D42D5DB013B60
:10124000002240F27D61C9E7384650F0BEFEB27B15
:101250004FF0FF31C2F1200221FA02F2A223002155
:101260004FF054FF2A4603462146304648F05DFCC5
:101270000E20C6E72146090034540900EF3E09005C
:10128000944909002DE9F04F93B00DAB0193684BE1
:10129000009305231EF070FB0D9D664940F253320A
:1012A00028461EF04FFCDDF83880624940F2C952F2
:1012B00040461EF047FCDDF83C905E4940F2CA52C1
:1012C00048461EF03FFC109C204624F0FFFF20B152
:1012D0002146594850F01AF80446012120464EF0A4
:1012E000EDFB824660B9204624F016FAC3880093CD
:1012F000524840F20E23432240F257413FF036F865
:10130000119F0E2F13D04B4940F2624238461EF017
:1013100019FC4146284607F0BFFD4946284607F01C
:10132000BBFDAB7B102B04D045483FF02BF80027CA
:10133000EFE7EB8804930026049BB34203DC0D988F
:1013400013B0BDE8F08FAB89AA68734302EB830347
:101350000593AB880693B8F80C30D8F8082073438F
:1013600002EB83030393B9F80C30D9F808207343D8
:1013700002EB8303089333B24FF0000B0B93069BF1
:101380005B4501DC0136D7E7039B33F8024B03933F
:101390003FB10B9A0FFA8BF1384648F090FB0028CA
:1013A0003FD163BAADF82430089B33F81B305ABAEA
:1013B000ADF82820C3F3C402C4F304210792C4F398
:1013C000002242EA4102C3F3042EC3F3002141EAA2
:1013D0004E014FF0400012FB001207991AF802204C
:1013E000C4F3C40CC3F3C003C4F3C00443EA410311
:1013F00044EA4C04402114FB0134099B1AF80440D0
:101400006408E40244EA52040A9AC3F34513C2F39F
:10141000451213FB01231AF8033044EA431464BA5B
:10142000A4B2059B23F81B400BF1010BA7E700BFFB
:101430005C210A0020BE0900CCC009003D4909001A
:10144000322C090070B586B003AB0193164B0093A4
:1014500003231EF091FA039E144940F2C72230463E
:101460001EF070FB049D124940F2CD4228461EF04A
:1014700069FBA86840F2CD424FF480711EF020FB5A
:10148000059C0E2C0DD0094940F2624220461EF008
:1014900059FB30466A68214637F0C4F9039806B014
:1014A00070BD0024F5E700BF94210A0020BE0900AA
:1014B0007CBD09002DE9F04FA7B003AB01934B4B66
:1014C000009303231EF058FA039D494940F2C722B6
:1014D00028461EF037FB049C204624F01DF9C37BF0
:1014E000002B40D000EB8300424B02699A423AD174
:1014F000606840F2574203211EF0E2FAD4E9037813
:10150000A4680DF118090026324621461F2058F024
:101510009EFA444509F8010B04D0324641461F208B
:1015200058F095FA0136202E89F85F00ECD10DF1C4
:1015300037060024224639463F2058F088FA013405
:10154000402C06F8010FF5D1059F0E2F0ED028492B
:1015500040F2624238461EF0F5FAAB7B102B07D002
:1015600025483EF00FFFA0462746CAE70027F4E7CC
:10157000B5F806900026B14503DC039827B0BDE816
:10158000F08FAB89AC68B5F804A0734304EB830417
:101590004FF000080FFA86FBC24501DC0136EAE78E
:1015A00037B15A460FFA88F1384648F088FAC8B978
:1015B000228853BAC3F3451398336B4413F8601C65
:1015C000C2F30423C2F3C402983398326B446A44D2
:1015D00013F8203C12F8802C43EAC22343EA41135B
:1015E0005BBA238008F101080234D5E7AC210A0078
:1015F00020BE0900917C0500322C09002DE9F04F36
:10160000ABB00FAB0193924B009303231EF0B4F9E0
:101610000F9C904940F2C72220461EF093FA3022D8
:10162000002112A84FF0F3FB109E16F0030566D1BF
:101630003368894A934224D112AF294630464EF08E
:1016400083F801353B46032D07F1140783ED000AAB
:10165000F3D1119F0E2F63D07E4940F2624238468B
:101660001EF070FA12AD0DF178080026731E0B2BD8
:1016700071D8DFE803F06D70686A706A57706D703A
:101680006873764A934217D10DF1480847462946B8
:1016900030464EF059F84346691C83ED000A304647
:1016A0004EF052F80235062D87ED030A08F11408B2
:1016B00007F11007EBD1CCE7694A934211D14FF003
:1016C0000308294630464EF03FF8B5FBF8F72AAB41
:1016D0002F44013503EB8707092D07ED180AF0D1D8
:1016E000B7E7604A93420AD112AF294630464EF01E
:1016F0002BF801350C2DA7EC010AF6D1A9E73046ED
:1017000024F00AF8C38801934FF487730093564876
:1017100040F20D1340F2272240F226213EF03AFE1D
:1017200000279FE7514BB5EC010A07EE903AF8EE1F
:10173000E77A013627EE800A35F03EFBBDEEC00A9F
:10174000A8EC010A92E74A4BEDE74FF40033EAE7D1
:101750004FF40043E7E74FF48033E4E7A37B102B1B
:1017600002D044483EF00EFE1E9B02931F9B039343
:10177000209B0493219B0593229B0793239B089313
:10178000249B0993259B0A93269B0B93279B0C93E1
:10179000B4F80690289BDDF8A4A00D930026B1456F
:1017A00003DC0F982BB0BDE8F08FA389A568B4F8CF
:1017B00004B0734305EB83054FF0000832B2C34514
:1017C00001DC0136EBE747B10FFA88F138460692A3
:1017D00048F075F9069A002835D1B5F800C0039B8A
:1017E0009CFA9CF1C1F3451103FB01F0029BCCF381
:1017F000C40E03FB0E00049BCCF3042C03FB0C0073
:10180000059BC3180693089B07984B4300FB0E33B8
:10181000099800FB0C330A9803440C9841430B9839
:1018200000FB0E110D9800FB0C110698A3F3064364
:101830005144A0F305405B0143EAC023A1F30541F5
:101840000B435BBA2B8008F101080235B7E700BFF4
:10185000DC210A0020BE0900F8C10900A8C1090066
:101860004CC10900E4C009009F2B0900C1FF3E00E4
:10187000E1FF1E00322C09002DE9F04F2DED028B07
:10188000A7B002AF07F1700301938F4B00930823B9
:101890001EF072F8D7F870B08C4940F2C722584653
:1018A0001EF050F9D7F88C303B660E2B1CD08749C0
:1018B00040F2624218461EF045F9F86F23F0A2FE8E
:1018C000D7F874804046F0EE408A24F0BFFDC4078C
:1018D0000DD4404623F020FF4FF40B72C3887C48A0
:1018E00040F265613EF056FD00233B66E5E744109B
:1018F00007EE904AB8EE677AF1EEC77AFDEEE77A26
:1019000017EE905AE90703D505FB05F39C4202D078
:1019100070483EF037FDA300073323F00703ADEB1B
:10192000030D02AB4FF000097B654E46A1451AD16D
:10193000B86F0E2828D023F065FEB0EE408A6B0801
:10194000FB6697F880307B6397F884303B6397F8A9
:101950008830FB62FB6E0133BB669BF80E30102BA8
:101960001FD05D48D5E74FEA4901042241F001014B
:10197000404626F0D5F850F028FB7B6D064443F82E
:10198000290009F10109D1E7B7EE007A36B107EE77
:10199000906AF8EEE77A87EE278AD0E7B0EE478ABA
:1019A000CDE7BBF804304D4D4D4CD5F800A00133C8
:1019B0005B10BB65BA6DBB6E02FB03F6B60040D18F
:1019C000BAF1000F02D0504631F0ECFE0023236044
:1019D0002B609A469FED430A28EE000A35F0ECF999
:1019E000FDEEC07A9FED400AC7ED127A28EE800A1C
:1019F00035F0E2F9FDEEC07ABBF806303B6217EE37
:101A0000903A5B007B61FB6EC7ED117A5B42FB6530
:101A1000FB6E5B003B614FF000093B6A4B4500F3F6
:101A2000D181BBF80650FB6EEC1A24EAE474A5429F
:101A300000F33383386F9437BD46BDEC028BBDE8AD
:101A4000F08FBAF1000F00F0B38123689E42C1D934
:101A5000264B1C6820465AF030FB864280F09F815E
:101A600055460C2E55F8043DB04623F0030938BF07
:101A70004FF00C08C14580F09B8005EB09004168E0
:101A8000CA0706D521F0030109F104030B444345BD
:101A90002ED2314620465AF017FB0546002800F0AA
:101AA0007E81B1454A46514628BF32464FF06EF915
:101AB000514620463CF0E6FFAA46084BC3F800A07A
:101AC000074B1E6086E700BFDC200A0020BE09002D
:101AD00025490900B32B0900322C09002C61012093
:101AE000306101200000804700007C4A50560120F0
:101AF000638AC3F3C7139942AAF1080980F00781EA
:101B00002269C2F38532B3FBF2F30022B1FBF3F397
:101B10007B66D0E902C1CCF80C10C1F808C021697D
:101B20007B6ED4F820E0C1F3853102FB01315EF811
:101B3000213098421AD1A4454EF821C016D1D4F8CC
:101B40001CE07B6E5EF822104FF0010C0CFA03F3E0
:101B500021EA03014EF82210E36953F822302BB931
:101B6000A3690CFA02FC23EA0C03A3615AF8043CB3
:101B70004268043322F0030213444AF8043C23F081
:101B8000030343F80590BA4B1BB101221021AFF3B8
:101B900000805AF8043C23F003032B445A6822F0D7
:101BA00002025A605AF8043C23F001034AF8043C4C
:101BB00023F0030308F110029342FFF47EAF454483
:101BC000A3EB08036A68043B02F0030213436B6053
:101BD0005AF8043C03F0030343EA08034AF8043CC0
:101BE0006B6805F1080E23F00303734443F8045CAB
:101BF00053F8042942F002025A60686820F0020398
:101C000020F0030043F0010370446B6050F80419A6
:101C1000CB074DD5638A21F00301C3F3C7138B4271
:101C200040F28E8022694FF0000CC2F38532B3FB84
:101C3000F2F3B1FBF3F37B66D0E90212CA60916064
:101C400022697B6ED4F82090C2F385320CFB0232FD
:101C500059F82230984219D1A14249F8221015D1E1
:101C6000D4F81C807B6E58F82C20012101FA03F374
:101C700022EA030248F82C20E36953F82C302BB9F0
:101C8000A36901FA0CF123EA0103A3616B684268BE
:101C9000043322F0030213446B6023F003039E44D9
:101CA000734B4EF8045C1BB101221021AFF300808E
:101CB0006968638A206921F00301C3F3C71399425D
:101CC000C0F3853053D2B3FBF0F3B1FBF3F3002242
:101CD000216A02FB003051F82010C5E90214CD60E2
:101CE0002169206AC1F3853102FB013140F821509E
:101CF0000125A16905FA02F00143E069A16150F8EC
:101D0000221005FA03F3194340F82210D5E6A9B1D1
:101D1000B1FA81F2C2F1200294F812C0531ECCF342
:101D2000021CA3EB0C0321FA03F3012101FA0CF1CD
:101D30004B40217C7B66A2EB5112EAE60A46EBE7B8
:101D400099B1B1FA81FCCCF1200CA27C0CF1FF33EB
:101D5000C2F302129B1A21FA03F301219140227C63
:101D60004B407B66ACEB521C66E78C46EDE7A1B1BD
:101D7000B1FA81F2C2F1200294F812C0531ECCF3E2
:101D8000021CA3EB0C0321FA03F3012101FA0CF16D
:101D90004B40217CA2EB51129AE70A46ECE75046F1
:101DA00031F000FD334B00221A6030463EF054FA09
:101DB000304631F0A7FD26608246286000287FF477
:101DC00009AEF2E7BBF80C30DBF8082009FB03F39F
:101DD00002EB8303BA6EFB63BB6EB9FBF3F302FB4A
:101DE0001393BA6D53430AEB8303FB61BBF80430D2
:101DF000BB613B690133BB63FB6EA9EB0303BB60B3
:101E00000FFA89F34FF000087B60BB6943451DDC86
:101E1000FB6E4B4517DCBBF80C00BD6EBC6EBBF80F
:101E20000420A9EB03014843B1FBF4F405FB1411B2
:101E3000BC6DDBF80830614352000AEB810103EB13
:101E400080004EF0A3FF09F10109E6E53B6E9BB16E
:101E50007A680FFA88F1184647F031FE60B1FB6BE3
:101E600033F81830FA6922F8183008F10108CCE785
:101E7000000000002C610120DBF808103964BBF879
:101E80000C103965F96EBBF80430BBF806204145EB
:101E900000F3BC80591A884580F2B880F96E494534
:101EA00000F3B480511A894580F2B080BB683A6D66
:101EB000D7F85CC002FB03F4A300FB643B6C00207A
:101EC00003EB4803BB620246786601467B6DFC6CFF
:101ED000FE6D03EB80033B64BB6A23447B627B6A39
:101EE00033F816503B6C53F804EB3B646CBAC5F303
:101EF000C4030EFB0311C4F345137C6E0EFB0343B6
:101F00007B66FB6E0136C5F30425B3420EFB05224A
:101F1000E5DABB6B1844D7E9134304EB8303FB6496
:101F2000FB6E0CF1010C6345D0DAD7E911307C6E01
:101F300001FB00317B6904FB0033D7E91104A3F3F3
:101F4000064302FB0402A1F305415B01A2F3054233
:101F500043EAC12313437A6B002A54D01D1205F0C3
:101F6000F8027A66DA1002F0FC01DB003965D9B2BA
:101F7000F964F96B31F8180041BAC1F3CC0606F0E8
:101F8000FC043C64FC6CC3F3421323437C6EC5F336
:101F9000421525433C6DC2F38112224302EB8202BB
:101FA000C2EB0212262415FB04254FF00F0413FB8D
:101FB00004533C6C3A6BC6F38116344300F0F80CC2
:101FC000C900C0F3421004EB840401F0F80E4CEA9F
:101FD0000000C1F34211C4EB04144FF02605C2EB1C
:101FE000E3134EEA01010F2210FB054011FB020131
:101FF000B3EBE11FF96AB4BF012200224FF6FF7371
:102000008A4208BF00235BBA9BB22BE70024013A47
:10201000013BFE6DBA627B6222467C662146BB6A4A
:10202000D7F85CC009EB060020EAE0709842A8BF30
:1020300018463B6D4343FB607B6D03EB8403FB64FD
:102040007B6A08EB0C0525EAE5759D42A8BF1D4695
:102050003B6C03EB4505FB6835F82350FB6C53F8EC
:1020600004EBFB6468BAC5F3C4030EFB0311C0F3B1
:102070004513786E0EFB03037B66FB6E0CF1010CBF
:10208000C5F3042563450EFB0522D9DABB6B1C445E
:10209000FB6E0136B342C2DA47E7BE6EBBF80C00F6
:1020A000B96EB4FBF1F106FB1141BE6DDBF80830EF
:1020B000BBF804206043714352000AEB810103EB3B
:1020C00080004EF063FE0134B1E400BF2DE9F04F13
:1020D0002DED028B89B005AB01935E4B009303237A
:1020E0001DF04AFC0698C8B123F08CFAB0EE408A85
:1020F000059C594940F2C72220461DF023FD079F49
:102100000E2F0ED0544940F2624238461DF01AFD9F
:10211000A37B102B07D051483EF034F9B6EE008A6D
:10212000E6E70027F4E79FED4E0A28EE000A34F0B8
:1021300043FEB4F806A0BDEEC08A00264FF0260B81
:102140004FF04009B24505DC059809B0BDEC028BA3
:10215000BDE8F08FA3880393A389A568734305EBBB
:1021600083054FF00008039B434501DC0136E9E796
:102170003FB132B20FFA88F1384647F0A0FC002890
:1021800064D129884BBA01F0F802C1F3421111431E
:10219000C3F3CC0202F0FC0CC2F3811242EA0C0041
:1021A000DB0000EB800203F0F80EC2EB0212C3F377
:1021B000421343EA0E034FF00F0C18EE10EA11FB26
:1021C0000B2213FB0C22BEEBE21F4FEAE21C3DDAAE
:1021D000CCEB4E024FF6D57C10FB0CFC4FF6EB7EA1
:1021E00011FB0ECC4FF6CA7E10FB0EF011FB09015D
:1021F0004FF6F67013FB09CC13FB0013DB114BF207
:10220000D2614FEAEC1C594345F61A0000FB0C1151
:10221000144882F30802A2EB2141434302EB23431B
:10222000114881F30801C90083F3080301F4FC613C
:1022300000EA03230B430D4901FB0CFC02EB2C428B
:1022400082F3080243EAD2035BBA2B8008F101084B
:10225000023588E7C4210A0020BE0900322C09009B
:1022600000008043E966010000F8FFFFA2C50100FD
:102270002DE9F04F2DED028B9BB011AB0193AE4BCE
:10228000009309231DF078FBAC4911984FF4557267
:102290001DF058FCA94940F2BB52054612981DF0AA
:1022A00051FCA649029040F2BC5213981DF04AFC22
:1022B000074615980E2835D023F0A4F9F0EE408A91
:1022C00016980E2831D1B7EE008A38EE688ADDF80C
:1022D00050909B494FF4447248461DF033FCDDF8A2
:1022E0005C80984940F2D52240461DF02BFC029AB2
:1022F000AB889188994212D1029BEA88DB8893428D
:102300000DD1029AA87B927B824208D1B88888427C
:1023100005D1F988994202D1BB7B93420AD08A4801
:102320003EF030F8F6EE008ACAE723F06BF9B0EE23
:10233000408ACCE799F80440092C0EDC0121A14029
:1023400011F0AA0F05D1092C07D1082B07D07F481F
:10235000E6E7102B03D07E48E2E77E48E0E71898D6
:1023600098F804300A930E283DD04FF02EFE00233B
:102370000390079319980E283AD04FF026FE0023B9
:1023800004900593AA88ADF83C200023EA880E93B8
:1023900028460EA9ADF83E2010930FF02FFEF0EE68
:1023A000687AFEEECC7A17EE90BAF0EE487AFEEE3E
:1023B000CC7A5B4617EE900A434348BFFF330BEBE2
:1023C0000002A2EB2323092C069340F08C809DF899
:1023D0000C300893C0F5807309939DF81030039377
:1023E0004FF0000C24E00123079300230393C1E77F
:1023F00000230122CDE90432C4E7AA89AB680CFBB3
:1024000002F203EB8208029BBA8999899B680CFB54
:1024100001F103EB8101BB680CFB02F203EB8202CA
:10242000C146AC88A9EB0803A3420ADB0CF1010CFE
:10243000EB889C45E1DB0E201BB0BDEC028BBDE8B8
:10244000F08F079B9BBB0B78089C1B1B18BF0123BD
:10245000059C002C40F0428192F800E0B3B30C469A
:10246000039E14F8013BB6450BFB03F328D00A9EEC
:1024700011F8014B12F8013B012E0BFB04F400FB99
:1024800003F316D103FB04FE0EF57F4A0AF1FF0A9F
:102490003EEA2E0E28BFD6462344A3EB2E43069CCD
:1024A00093FBF4F383F3080309F8013BB9E7012335
:1024B000CEE7099E744348BFFF3403EB2423EEE7C5
:1024C000002BB8BFFF331B122146EBE7039B9E4551
:1024D00006D012F8013B434348BFFF331B12E1E72C
:1024E00099F80030DEE704F0FB030B93C0F580732E
:1024F0004FF000080993EB8898459CDAAA89AB68ED
:1025000008FB02F203EB82030893029B9A899B6803
:1025100008FB02F203EB8203BA890C93BB6808FB49
:1025200002F203EB82030D934FF00009AB8899454B
:1025300012DB08F10108DEE70C220A0020BE0900C8
:10254000E8BD090020C00900EF4609009C430900CE
:1025500080430900093C09000C9B33F819200D9BAE
:1025600033F819100B9B032B079B01BF52BA49BAD2
:1025700092B289B2002B40F0B980059B002B40F04D
:10258000B180039B934200F08F80049B8B4276D0F6
:102590000A9E1412D3104FEA212E4FEAE10CD2000A
:1025A000C90004F0F80403F0FC03D2B20EF0F80EF8
:1025B0000CF0FC0CC9B2012E0BFB04F40BFB03F373
:1025C0000BFB02F200FB0EFE00FB0CFC00FB01F11A
:1025D00042D10EFB04FA0AF57F46FF363AEA2A0A90
:1025E00028BFB24674440CFB03FEA4EB2A440EF54C
:1025F0007F4A0AF1FF0A3EEA2E0E28BFD646634400
:1026000001FB02FCA3EB2E430CF57F4E0EF1FF0EF7
:102610003CEA2C0C28BFF4460A44A2EB2C42069953
:1026200094FBF1F493FBF1F32402DB0004F478440F
:1026300003F4FC63234392FBF1F2C2F3C40213439D
:102640000B9A032A01D15BBA9BB2089A22F8023B8B
:1026500009F10109089269E7099E7443099E48BF80
:10266000FF347343099E48BFFF33724348BFFF32B4
:102670000EEB24240CEB232301EB2222CFE702F400
:10268000784102F4FC635C4663430BFB01F102F00A
:102690001F0248BFFF330912624341EA232348BFA8
:1026A000FF3243EA2223CFE7049B8B4213D001F48D
:1026B000784201F4FC63434300FB02F201F01F0186
:1026C00048BFFF331212414342EA232348BFFF3180
:1026D00043EA2123B8E7089B1B88B6E7002B7FF469
:1026E000C6AEF6E6039B9342E1D051E7059B002B73
:1026F0007FF44EAF49E700BF2DE9F04F99B011AB21
:1027000001933F4B009307231DF036F93D49119883
:1027100040F2C7221DF016FA054605220BA91298B1
:1027200020F0AEFEEB88AA8813A909A801F0DEFA12
:10273000BDF92830BDF92690BDF924A0BDF92AB015
:102740000493A3EB0A049DF83410ABEB09030022B9
:1027500040205C431DF054FA0C9BB3FBF0F6179B32
:1027600005900E2B4F46039308D018464FF02DFCD2
:102770000690B44205D924483DF094FD0023069309
:10278000F7E7AB7B0B9C01269E40013EBB4534DC4A
:10279000049BADF83C30284600230EA9ADF838A0C4
:1027A000ADF83A90ADF83EB010930FF027FC0E2034
:1027B00019B0BDE8F08F059B022B18D0042B19D05F
:1027C00014F8013B03990E2902D00699994207D0CB
:1027D00033400FFA88F1284607920FF033FC079A2E
:1027E00008F10108049B4345E5DC0137CEE734F8E6
:1027F000023BE7E754F8043BE4E7D0463AB2F1E79E
:102800007C230A0020BE0900333409002DE9F04F73
:1028100097B002AF07F140030193B54B0093042337
:102820001DF0AAF8B349786C40F2BA521DF08AF94B
:10283000B04906464FF45572386C1DF083F9FC6CB4
:10284000AD49814640F28F2220461DF07BF9BD6CD8
:10285000AA4940F2BF5228461DF074F9B9F804A005
:10286000B388534509D1D9F80430BB60B9F80630B4
:10287000BB61BA69F388934202D0A1483DF06EFD76
:1028800099F80E30102B03D0012B01D09D48F5E7AD
:102890002A79092A06DC0121914011F0AA0F03D1FF
:1028A000092A06D09848E9E7B37B102B06D0974851
:1028B000E4E7B37B082B01D09548DFE7032AB4F99E
:1028C000043053D0072A4FD0052A52D1002242F0BB
:1028D000020B904ADBB252F8235069780AEB4103AD
:1028E00003EB43035B0007336A46DB08A2EBC30339
:1028F0009D460A2301EB41084B4302AC03EB8A03DC
:10290000D04404EB410204EB48081C440AF11F03C5
:1029100068465B09A0EB43139D46BA62C7F82C805A
:102920003C6343F8081B30467B62594600234CF059
:1029300043FD6B78009342460123594630464CF0E4
:102940003BFD6B78009322460223594630464CF0FB
:1029500033FD4FF000084446BB69434540F3DC803B
:10296000BB6A3B62002227E00122B0E74FF0010B77
:10297000AFE74FF0000BACE73B6A786A33F91230EF
:1029800023447F2BD4BF00210121802B8154B4BF6D
:102990000021FF215B1AFB61E81C4FF0000C297835
:1029A0008C4544DBAC78FB6914FB03F4002CB8BF06
:1029B000FF3444F30F2401329245DDDC7A6A41464C
:1029C00048465AF056FDFB6AFB61BB623B6B7B617C
:1029D000FB623B6A3B6308F101037B60BB6908F162
:1029E0000102934200F098806B7800933A6A08F1F4
:1029F0000303594630464CF0DFFC5246002A35D1DD
:102A00007A6A796848465AF034FD7B69BB623B6A52
:102A1000FB62FB693B636B780093FA6908F104037E
:102A2000594630464CF0C8FC08F1020894E790F98A
:102A3000011090F9004007F1500303EB8101FB699D
:102A400051F8281C796190F90210144411FB03F12C
:102A50007B69002933F814E0B8BFFF310EEB212E5B
:102A6000033023F814E00CF1010C98E7013AFB69FC
:102A700033F81230234419B27F29D4BF002001203B
:102A800080297C6AB4BF0021FF215B1AA0543B61FE
:102A9000E81C4FF0000C29788C4509DBAC783B69C9
:102AA00014FB03F4002CB8BFFF3444F30F24A5E754
:102AB00090F9011090F9004007F1500303EB8101F8
:102AC0003B6951F8281CF96090F90210141B11FBA6
:102AD00003F1FB68002933F814E0B8BFFF310EEBB7
:102AE000212E033023F814E00CF1010CD3E700BFD2
:102AF0005C240A0020BE090004C00900E8BD0900EA
:102B000086390900E22D0900222C0900D42D090084
:102B1000CB2D090054240A00BA68002307F13401C0
:102B20004846C7E90E237B630FF068FA0E2054373E
:102B3000BD46BDE8F08F00BF2DE9F04395B00AAB6C
:102B40000193304B00930A231CF016FF2E490A987C
:102B50004FF455721CF0F6FF40F27763828804460A
:102B600000210C984EF0D2FAE28840F27D630021F9
:102B700007460D984EF0CAFA234940F2BA528046F1
:102B80000B981CF0DFFF0546C38882880EA908A8B1
:102B900001F0ACF8A27BAB7B9A4202D21B483DF01D
:102BA000F1FB12980E2825D04FF00FFA4FF00009D4
:102BB000064613980E2821D04FF007FA0023CDE9DE
:102BC0000603BDF926300393BDF924300293BDF905
:102BD00022300193BDF9203000932046CDE90469ED
:102BE0000FFA88F33AB2294606F030FF0E2015B0EE
:102BF000BDE8F0834FF001090026DAE70123002049
:102C0000DDE700BFDC230A0020BE0900F22D090029
:102C10002DE9F04F91B00BAB0193974B0093052337
:102C20001CF0AAFE4FF4557294490B981CF08AFFD1
:102C30000E9B827B029301239340029A9A4206469E
:102C400002D38F483DF09EFB0F9F6FF000429742EA
:102C500003D0BB4201D88B48F4E7BDF93090B9F1FD
:102C6000000F02DBB388994501DB8748EAE7BDF92D
:102C70003480B8F1000FF8DBF3889845F5DA029B51
:102C8000BB4200F0F58000201AF032F805464846B5
:102C90004FF0B6FD069040464FF0B2FD06A90790F2
:102CA000022023F0D1FE014628464FF0D4FC6FF0FD
:102CB00000439F420CD106984FF087F904460798CD
:102CC0004FF083F921B202B2304646F0F8FE0746D3
:102CD000002304AA05A928460593CA464FF0F1FC33
:102CE000CDF80C80059A8AB9039BADF820900AF1C3
:102CF000010A013308A93046ADF82280ADF824A0BE
:102D0000ADF826300A920FF079F9B1E004AA05A9CE
:102D100028464FF0D6FC0021284623F0E1FB04466C
:102D200080684FF052F98346E0684FF04EF90FFA91
:102D30008BF102B2304646F0C2FEB84205D004AA7A
:102D400005A928464FF0BDFCCCE7A0684FF0DEFA9D
:102D50008346E0684FF0DAFACB45039BB8BF0FFA21
:102D60008BF9D345C8BF0FFA8BFA4045B8BF0FFAAD
:102D700080F89842C8BF03B2A068C8BF03934FF061
:102D800024F98346E0684FF020F9029B02B20FFA63
:102D90008BF130460FF056F9E0684FF0B7FA002893
:102DA00011DDA3680893E0684FF0B0FA01384000E5
:102DB00040F00100099008A9022023F045FE0146D9
:102DC00028464FF048FCA0684FF0A0FA002811DD1B
:102DD000A0684FF09BFA0138400040F001000890D5
:102DE000E368099308A9022023F02EFE0146284635
:102DF0004FF031FCA0684FF089FAB3880130984257
:102E000011DAA0684FF082FA0130400040F0010072
:102E10000890E368099308A9022023F015FE0146F3
:102E200028464FF018FCE0684FF070FAF388013044
:102E3000984211DAA3680893E0684FF067FA01300E
:102E4000400040F00100099008A9022023F0FCFD99
:102E5000014628464FF0FFFB04AA05A928464FF07B
:102E600030FCFDF773FD094B9B6A002B3FF43AAF32
:102E70000E2011B0BDE8F08FEC220A0020BE090040
:102E8000D32B0900B6390900462F0900F85C012050
:102E90002DE9F04F93B00DAB0193714B00930523D7
:102EA0001CF06AFD4FF455726E490D981CF04AFEF5
:102EB000827BDDF84480012393409845044602D389
:102EC00069483DF05FFABDF938A08288BDF94060DD
:102ED00040F27763002150464EF018F9BDF93C905E
:102EE000E28840F27D63002148464EF00FF940F23F
:102EF0000B52002130464EF001F90EAA8CCA002573
:102F0000D11BCDE909553A44ADF81C10D91B3B44FF
:102F1000ADF82020ADF82230A388ADF81E1007AA26
:102F20001046ADF82C300AA9E388ADF82E300C9588
:102F300049F095FC07A920460FF060F84B4940F294
:102F4000776347F6FF7250464EF0E0F840F27D633B
:102F500047F6FF72454948464EF0D8F8A088E28807
:102F600050454FEA4703A8BF5046C3F103034A4503
:102F70001BB200B2A8BF4A4612B2039320EAE07324
:102F8000049322EAE277B54203DD0E2013B0BDE8D8
:102F9000F08F049B06EB070B05EB03090FFA8BF28E
:102FA0000FFA89F1434620460FF04CF8049BA7EB3B
:102FB000060A591B09B20FFA8AF2434620460591C8
:102FC0000FF040F80FFA8BF20599434620460FF0B8
:102FD00039F80FFA8AF20FFA89F1434620460FF0CA
:102FE00031F8049B05EB070B03EB06090FFA8BF294
:102FF00043460FFA89F120460FF024F8049BA3EB17
:10300000060A0FFA8BF24346A7EB050B0FFA8AF17B
:1030100020460FF017F843460FFA8BF20FFA8AF1A9
:1030200020460FF00FF80FFA8BF243460FFA89F1A2
:1030300020460FF007F8039B002BC5BF039BAA1B7C
:1030400006330A33D2BF03EB850303EB820306F199
:10305000FF361BB2C8BF36B20393013593E700BFFA
:103060002C240A0020BE0900462F09000080FFFF23
:103070002DE9F0438FB008AB01932A4B0093062350
:103080001CF07AFC4FF45572274908981CF05AFD41
:10309000827BDDF83490012393409945044602D3A6
:1030A00022483DF06FF90B98099A0C990A9B15B2CA
:1030B00007B21EB20FFA81F8BD42B5BF421C3846B6
:1030C000284601324645B4BF4B1C0133ADF80E30E3
:1030D0004FF00003CDE90433ADF80C20A288ADF821
:1030E0001820E288ADF81A20B4BF3146414602AA42
:1030F000ADF80800ADF80A10104605A9079349F08D
:10310000AEFB02A920460EF079FF2046CDE90089EA
:103110003B46324629464AF089FC0E200FB0BDE8F6
:10312000F08300BFBC220A0020BE0900462F090020
:103130002DE9F04F9FB019AB01935B4B0093052332
:103140001CF01AFC594919984FF455721CF0FAFCFE
:10315000052210A906461A9820F092F905220DA919
:103160001B9820F08DF99DF84810002240201CF09B
:1031700047FD9DF83C100546002240201CF040FD14
:10318000854202D04A483DF0FDF8119BB3FBF5F3B0
:103190000993099A0E9BB3FBF5F39A4201D0454877
:1031A000F1E71C9B0293B37B029A012404FA03F318
:1031B0009A4201D34048E6E79DF874300A93109B89
:1031C00007932A460D9B0798089300214DF09AF922
:1031D0002A4607B2002108984DF094F90FFA80F8BA
:1031E000CDE90378C246CDF81880BB460597099B08
:1031F000A3422BD80A9B43B1029BDDE90312CDE920
:10320000008330463B464AF011FC059BADF84C303C
:10321000069BADF84E300023CDE91533ADF852A032
:10322000ADF850B0B288ADF85C20F288ADF85E2001
:1032300013AA16A91046189349F011FB304613A99A
:103240000EF0DCFE0E201FB0BDE8F08F214607987F
:103250002A464DF057F9214603B22A4608980B93A7
:103260004DF050F9029B0FFA80F9CDE90093DDE9AA
:1032700003120B9B30464AF0D9FB0B9B059A9A42EE
:10328000D4BF059205939B45069AB8BF9B464A4515
:10329000D4BF0692CDF81890CA45CDE90339B8BF1E
:1032A000CA460134A3E700BFB4230A0020BE0900C8
:1032B0003D45090052450900462F0900F0B591B07F
:1032C0000AAB0193274B009306231CF055FB4FF4E8
:1032D000557225490A981CF035FC827B0F9F01230B
:1032E00093409F42044602D320483DF04BF8828829
:1032F000C3880BA902A800F0F9FC029B04930025E7
:10330000039B059304A8069549F098FAA388ADF8A5
:10331000203004AAE388079507A91046ADF82230AB
:10332000099549F09CFA04A920460EF067FEBDF904
:103330001050BDF91430AB4202DC0E2011B0F0BDCC
:10334000BDF91260BDF91630B34202DC01352DB271
:10335000EFE732463B462946204601360EF072FE24
:1033600036B2EFE714230A0020BE0900462F0900F9
:103370002DE9F04786B003AB01931F4B0093032365
:103380001CF0FAFA40F2C7221C4903981CF0DAFB41
:10339000827BDDF81090012393409945044603D2C7
:1033A000DDF814A09A4524D3154840F20B313CF0C7
:1033B000F1FF3A462946204646F081FB814505D17A
:1033C00053463A46294620460EF03CFE08F10108D5
:1033D000E3880FFA88F79F42EBDB0136A38835B20A
:1033E0009D4203DB0E2006B0BDE8F0874FF00008D9
:1033F000EEE70026F2E700BFF4210A0020BE090034
:103400000A4909002DE9F04F2DED0C8B99B00BAB5B
:1034100001930D4B00930D231CF0AEFA0B490B9852
:103420004FF455721CF08EFB40F2BA5280460749A9
:103430000C981CF087FB98F80E20837B9A42074675
:1034400008D203483CF09EFF54220A0020BE090027
:10345000F22D0900B8F804100D98490859F01CFC29
:10346000B8F806100DEE100A49080E9859F014FC31
:10347000B9880CEE100A4908119859F00DFCF9882A
:103480000BEE900A4908129859F006FC0023109C94
:10349000009307AA0DF11E010BEE100A0F9811F010
:1034A00043F9B8F90620B8F904300092204606AA7C
:1034B0000DF11A0111F038F9BDF91E20BDF91A00FD
:1034C000824206DD1346ADF81E00ADF81A20024612
:1034D0001846BDF91C30BDF918108B4206DD1C469C
:1034E000ADF81C10ADF818300B462146002ABCBFC1
:1034F0000022ADF81E20B8F80440002BBCBF00230A
:10350000ADF81C30A242B8F80620C8BFADF81E4086
:103510009342C8BFADF81C2000284FF0000380F292
:103520001B829942ADF81A3002DAADF8183019460C
:103530008A424FF00003B8BFADF81820149C1398CE
:10354000009305AA0DF1160111F0EEF8B7F9062067
:10355000B7F904300092204604AA0DF1120111F0CF
:10356000E3F8BDF91620BDF91200824206DD1346CC
:10357000ADF81600ADF8122002461846BDF9143019
:10358000BDF910108B4206DD1C46ADF81410ADF8E5
:1035900010300B462146002ABCBF0022ADF8162091
:1035A000BC88002BBCBF0023ADF81430A242FA88BF
:1035B000C8BFADF816409342C8BFADF8142000282C
:1035C0004FF0000380F2D2819942ADF8123002DA56
:1035D000ADF81030194615988A42B8BFADF81020E2
:1035E0000E2800F0CD8122F00DF8F0EE40CA1698BA
:1035F0000E2840F0C881B7EE00AA17980E2800F0F8
:10360000CD814EF0E2FC002383460293BDF91630D3
:10361000BDF91C20039208EE103ABDF91430BDF933
:103620001A60BDF91E90BDF918A008EE903ABDF9D8
:10363000123009EE103ABDF91030B0EE6C0A09EE06
:10364000903A35F01BFCF0EE40AAB0EE6C0A0CF09C
:1036500065FAF8EEEB4AB8EECB4A20EE647A2AEE31
:10366000843A27EE0A7A23EE0A3AF8EECD3A77EE5C
:10367000035A6AEEE47A60EE046A02EE906A75EE2E
:10368000A35A67EE8A7A66EE8A6AF8EEE22AB8EE04
:10369000CC5A37EEE66AF4EEE25AF1EE10FA36EE64
:1036A000056A039A40F17F81FDEEE52A12EE903A19
:1036B0000FFA83FC02EE909AF8EEE22AF4EEE25A58
:1036C000F1EE10FA40F37181FDEEE55A15EE903AF5
:1036D0001DB205EE90AAF8EEE55AB4EEE56AF1EEF9
:1036E00010FA40F16481FDEEC65A15EE903A19B217
:1036F00005EE902AF8EEE55AB4EEE56AF1EE10FA1E
:1037000040F35781BDEEC66A16EE103A1CB2BB8874
:103710001BEE900A1B1A06EE103AB8EEC66A02EECD
:1037200090CA60EE065A2AEE866A65EE8A5A26EE3E
:103730000A6A33EE253AF8EEE22A33EE233A76EEC1
:10374000666AB4EEE23AF1EE10FA76EE856A05D5D5
:10375000FDEEC32A12EE903A0FFA83FC02EE905A65
:10376000F8EEE22AB4EEE23AF1EE10FA04DDBDEE34
:10377000C33A13EE103A1DB203EE101AB8EEC33A74
:10378000F4EEC36AF1EE10FA04D5BDEEE63A13EE9C
:10379000103A19B203EE104AB8EEC33AF4EEC36A17
:1037A000F1EE10FA04DDFDEEE66A16EE903A1CB278
:1037B000FB881BEE100A1B1A06EE903AF8EEE66A3A
:1037C00002EE90CA2AEEA63A60EE266A23EE0A3A84
:1037D00066EE8A6A75EEC35AF8EEE22A75EEA35ACF
:1037E00036EE266AF4EEE25AF1EE10FA36EE056A8B
:1037F00005D5FDEEE52A12EE903A0FFA83FC02EEB3
:10380000905AF8EEE22AF4EEE25AF1EE10FA04DDF4
:10381000FDEEE55A15EE903A1DB205EE901AF8EE5F
:10382000E55AB4EEE56AF1EE10FA04D5FDEEC65A9B
:1038300015EE903A19B205EE904AF8EEE55AB4EE5C
:10384000E56AF1EE10FA04DDBDEEC66A16EE103A36
:103850001CB277EEA67A37EE437A06EE90CA37EEC0
:10386000237AF8EEE66A77EE857AB4EEE67AF1EE40
:1038700010FA05D5FDEEC76A16EE903A0FFA83FCF2
:1038800006EE905AF8EEE66AB4EEE67AF1EE10FA39
:1038900004DDBDEEC77A17EE103A1DB207EE101A1E
:1038A000B8EEC77AF4EEC77AF1EE10FA04D5BDEEA1
:1038B000E77A17EE103A19B207EE104AB8EEC77A57
:1038C000F4EEC77AF1EE10FA04DDFDEEE77A17EEBA
:1038D000903A1CB2CAEE8ABA731EE1451BB2B8BF59
:1038E000E146AE42D8BF1D468A42B8BF0A460AF139
:1038F000FF331BB2A245D8BF1C466B1CADF8243069
:10390000631C80EE0ABAADF8263008A900234046B1
:103910001646ADF82090ADF822200A9365EE2B7A7A
:1039200025EE0B5AE3EE8B7AABEEE35A74EEE7AA80
:1039300007EE902A34EE45AAF8EEE77AEBEEA7AA56
:10394000ABEE27AA0EF05AFBB44234DA0E2019B0BF
:10395000BDEC0C8BBDE8F08F0029BCBFADF8183072
:1039600019468442B8BFADF81A40E1E50029BCBF52
:10397000ADF8103019468442B8BFADF812402AE6BF
:10398000DFED37CA33E621F03DFEB5EEC00AF1EEB9
:1039900010FAB0EE40AA7FF530AE2CE60123029378
:1039A0004FF0000B32E6B44684E64D4691E65146B0
:1039B0009EE61446ABE607EE909AF8EEE77AB0EE94
:1039C0006ACAF0EE4ACAABEE27CACA46EBEEE7CAAD
:1039D000554506DA01367AEEABAA3AEE0BAA36B2B4
:1039E000B2E7F8EEC87AF4EECC7AF1EE10FA2DD800
:1039F000F8EEC97AB4EEE7CAF1EE10FA26D5F8EE81
:103A0000E87AF4EEEC7AF1EE10FA1FD8F8EEE97AE3
:103A1000F4EEE7CAF1EE10FA18D5FDEEEC7A38466E
:103A2000CDED037AFDEECC7ABDF90C20CDED037A15
:103A3000BDF90C1046F043F8029A03460AB98345D3
:103A400004D03246514640460EF0FCFA0AF1010A13
:103A50003CEE0BCA7CEEEBCA0FFA8AFAB8E700BF5D
:103A6000000000002DE9F04F9DB002AF07F14C03BC
:103A70000193974B009307231BF07EFF9549F86C49
:103A800040F2C7221CF05EF8BE6D731E012B824609
:103A900005D9042E03D0904831463CF07BFCD7F882
:103AA0005480B8F1020F05DCB8F1000F14DC8B482C
:103AB0004146F2E7A8F104031C2BF8D8884A0121FB
:103AC00099400A4042B9142BF1D1012E04D0854807
:103AD000182231463CF05EFC3B6DBB6297F85C30CF
:103AE000FB6297F860303B6297F86430FB619AF8AC
:103AF0000E30B86A012101FA03F3013B7B611FF02C
:103B000011FDBAF8043078600024A7F8443007F1BA
:103B10004001BAF80630A7F8463050463C64BC6411
:103B20000EF06CFABAF804307C6308FB03F303EB85
:103B3000C603F200013BB3FBF2F373433B63033371
:103B400023F003037B623B6B013323F00103BB6172
:103B50007B6A073323F00703BB60BAF806907B6BE0
:103B6000994504DC0E206C37BD46BDE8F08FBB687C
:103B7000C7F810D0ADEB030DFB6902AD9BB17B6BB9
:103B800009F1FF39A9EB03090023FB637B683A6B5A
:103B90005C68B86A294607F13C03A047F96B29B174
:103BA00008463CF0A7FBD7F83490EDE73B6B834227
:103BB00002D04D4858F07FFE3B6A93B1022E0BD0E5
:103BC000042E0ED17A6A2B46A918994209D01A6898
:103BD00012BA43F8042BF8E7BA692B4651199942F7
:103BE00010D108F1FF33AB460024FB600FFA89F9CE
:103BF000BAF804309C420ADB7B6BD7F810D0013353
:103C00007B63AAE71A8852BA23F8022BE7E7B8F1D8
:103C1000080F08DCFA68072A0ED8DFE802F00F2741
:103C20000D360D0D0D45B8F1180F42D0B8F1200F2B
:103C30004AD0B8F1100F39D0002309E0FA6AE31036
:103C40008AB1E24302F00702EB5C134103F0010387
:103C50007A6921B2134050464A460EF0F3F9013416
:103C60000BF1030BC4E704F00702EDE7FA6AA310B7
:103C700042B1E24302F00302EB5C5200134103F055
:103C80000303E5E704F00302F6E7FA6A631042B1C2
:103C9000E24302F00102EB5C9200134103F00F03D8
:103CA000D6E704F00102F6E72B5DD1E735F81430D2
:103CB000CEE79BF801309BF800201B0243EA024349
:103CC0009BF802201343C3E755F82430C0E700BF38
:103CD00044230A0020BE09002033090040330900B4
:103CE0001110001032330900DC51090073B504468D
:103CF0000D461E466846084B44F065FC291D0DF133
:103D00000200064B324644F05EFC6B4603CB20605B
:103D10002046616002B070BD54210A004C210A00A7
:103D20002DE9F04F0D4687B00021924629F0E0F8CA
:103D300004460021284629F0DBF82379662B02D0BF
:103D40000379662B02D1C8483CF01CFB002303908A
:103D500008208DF817304CF061FF074608204CF022
:103D60005DFF064608204CF059FF0399CDE900603D
:103D700005463B460DF11702204653F035FF0399E7
:103D800050B9384613F03CFD304613F039FD284653
:103D900013F036FDB548D7E70AF1FF3A9DF8170052
:103DA000D4F81C90D1F81C802279BAF1030F05D801
:103DB000DFE81AF0E901BD0398053B08AA46B346BF
:103DC0002379D4F81C90D1F81C80422B40F0C1809C
:103DD0000A79422A3DD1394654F0B3F8C269044603
:103DE0000020134698F800C099F8001001EA0C0171
:103DF00003F8011BDAF80410D4F810C0DBF804E073
:103E000003918844991A8C45F144EBD8DBF80010F3
:103E1000DAF800200CFB1E11894403990CFB1122D7
:103E20009044E2680130904211D3384613F0E8FC28
:103E3000304613F0E5FC284613F0E2FC204607B0BC
:103E4000BDE8F08F5A461C46D3469246B8E71A465C
:103E5000C7E7622A28D13946682254F072F8C1694E
:103E600004460023002298F900C099F8000000EAF7
:103E70000C0021F8020B2069DBF804E0DAF804C03A
:103E800001328242F144E044EDD3DBF8002000FB34
:103E90001E229144DAF8002000FB1C229044E268C4
:103EA00001339342DED3C0E7482A27D1394654F084
:103EB00048F8C169044600230022B8F800C099F808
:103EC000000000EA0C0021F8020B2069DBF804E096
:103ED000DAF804C001328242F144E044EDD3DBF869
:103EE000002000FB1E229144DAF8002000FB1C2277
:103EF0009044E26801339342DED396E7682A41F0AA
:103F00003782394654F01DF8C16904460023002267
:103F1000B8F800C099F8000000EA0C0021F8020B84
:103F20002069DBF804E0DAF804C001328242F1448F
:103F3000E044EDD3DBF8002000FB1E229144DAF8C8
:103F4000002000FB1C229044E26801339342DED340
:103F50006BE7622B40F08C800A79622A2CD13946BB
:103F600053F0EFFFC26904460020134698F800C0E2
:103F700099F8001001EA0C0103F8011BDAF80410AB
:103F8000D4F810C0DBF804E003918844991A614525
:103F9000F144EBD3DBF80010DAF800200CFB1E1123
:103FA000894403990CFB11229044E268013090424D
:103FB000BFF43BAF1A46D8E7482A27D1394653F019
:103FC000C0FFC169044600230022B8F800C099F977
:103FD000000000EA0C0021F8020B2069DBF804E085
:103FE000DAF804C001328242F144E044EDD3DBF858
:103FF000002000FB1E229144DAF8002000FB1C2266
:104000009044E26801339342DED30EE7682A0B4600
:1040100021467FF417AF394653F093FFC169044638
:1040200000230022B8F800C099F9000000EA0C0053
:1040300021F8020B2069DBF804E0DAF804C0013251
:104040008242F144E044EDD3DBF8002000FB1E2265
:104050009144DAF8002000FB1C229044E26801330E
:104060009342DED3E1E600BF9E300900E32F090052
:10407000482B57D10A79482A27D1394653F061FF96
:10408000C169044600230022B8F800C0B9F8000056
:1040900000EA0C0021F8020B2069DBF804E0DAF8F2
:1040A00004C001328242F144E044EDD3DBF8002049
:1040B00000FB1E229144DAF8002000FB1C229044F1
:1040C000E26801339342DED3AFE6682A0B4621460D
:1040D0007FF4B8AE394653F034FFC169044600237B
:1040E0000022B8F800C0B9F8000000EA0C0021F87E
:1040F000020B2069DBF804E0DAF804C001328242E6
:10410000F144E044EDD3DBF8002000FB1E22914493
:10411000DAF8002000FB1C229044E268013393424D
:10412000DED382E6682B41F023810A79682A0B46A8
:1041300021467FF487AE394653F003FFC169044638
:1041400000230022B8F800C0B9F8000000EA0C0013
:1041500021F8020B2069DBF804E0DAF804C0013230
:104160008242F144E044EDD3DBF8002000FB1E2244
:104170009144DAF8002000FB1C229044E2680133ED
:104180009342DED351E6AA46B3462379D4F81C9075
:10419000D1F81C80422B40F0B5800A79422A31D1F7
:1041A000394653F0CEFEC26904460020134698F803
:1041B00000C099F8001041EA0C0103F8011BDAF87D
:1041C0000410D4F810C0DBF804E003918844991A75
:1041D0006145F144EBD3DBF80010DAF800200CFB6A
:1041E0001E11894403990CFB11229044E2680130AE
:1041F0009042BFF41AAE1A46D8E75A461C46D34638
:104200009246C2E7622A28D13946682253F099FEC5
:10421000C16904460023002298F900C099F8000003
:1042200040EA0C0021F8020B2069DBF804E0DAF820
:1042300004C001328242F144E044EDD3DBF80020B7
:1042400000FB1E229144DAF8002000FB1C2290445F
:10425000E26801339342DED3E7E5482A27D13946A5
:1042600053F06FFEC169044600230022B8F800C075
:1042700099F8000040EA0C0021F8020B2069DBF8F5
:1042800004E0DAF804C001328242F144E044EDD3A4
:10429000DBF8002000FB1E229144DAF8002000FB2E
:1042A0001C229044E26801339342DED3BDE5682AC4
:1042B00041F05E80394653F044FEC1690446002354
:1042C0000022B8F800C099F8000040EA0C0021F87C
:1042D000020B2069DBF804E0DAF804C00132824204
:1042E000F144E044EDD3DBF8002000FB1E229144B2
:1042F000DAF8002000FB1C229044E268013393426C
:10430000DED392E5622B40F087800A79622A2CD1B5
:10431000394653F016FEC26904460020134698F849
:1043200000C099F8001041EA0C0103F8011BDAF80B
:104330000410D4F810C0DBF804E003918844991A03
:104340006145F144EBD3DBF80010DAF800200CFBF8
:104350001E11894403990CFB11229044E26801303C
:104360009042BFF462AD1A46D8E7482A27D13946B1
:1043700053F0E7FDC169044600230022B8F800C0ED
:1043800099F9000040EA0C0021F8020B2069DBF8E3
:1043900004E0DAF804C001328242F144E044EDD393
:1043A000DBF8002000FB1E229144DAF8002000FB1D
:1043B0001C229044E26801339342DED335E5682A3B
:1043C0000B4621467FF419AF394653F0BAFDC16957
:1043D000044600230022B8F800C099F9000040EA22
:1043E0000C0021F8020B2069DBF804E0DAF804C0C5
:1043F00001328242F144E044EDD3DBF8002000FBBF
:104400001E229144DAF8002000FB1C229044E2684E
:1044100001339342DED308E5482B57D10A79482A65
:1044200027D1394653F08DFDC1690446002300228F
:10443000B8F800C0B9F8000040EA0C0021F8020BFF
:104440002069DBF804E0DAF804C001328242F1446A
:10445000E044EDD3DBF8002000FB1E229144DAF8A3
:10446000002000FB1C229044E26801339342DED31B
:10447000DBE4682A0B4621467FF4BFAE394653F091
:1044800060FDC169044600230022B8F800C0B9F8F5
:10449000000040EA0C0021F8020B2069DBF804E080
:1044A000DAF804C001328242F144E044EDD3DBF893
:1044B000002000FB1E229144DAF8002000FB1C22A1
:1044C0009044E26801339342DED3AEE4682B40F0BF
:1044D0004F870A79682A0B4621467FF48EAE39460B
:1044E00053F02FFDC169044600230022B8F800C034
:1044F000B9F8000040EA0C0021F8020B2069DBF853
:1045000004E0DAF804C001328242F144E044EDD321
:10451000DBF8002000FB1E229144DAF8002000FBAB
:104520001C229044E26801339342DED37DE4AA4624
:10453000B3462379D4F81C90D1F81C80422B40F06C
:10454000B7800A79422A31D1394653F0FAFCC26960
:1045500004460020134698F800C099F8001081EA3C
:104560000C0103F8011BDAF80410D4F810C0DBF8D2
:1045700004E003918844991A6145F144EBD3DBF8D8
:104580000010DAF800200CFB1E11894403990CFB83
:1045900011229044E26801309042BFF446AC1A46C2
:1045A000D8E75A461C46D3469246C2E7622A28D12B
:1045B0003946682253F0C5FCC16904460023002235
:1045C00098F900C099F8000080EA0C0021F8020B6D
:1045D0002069DBF804E0DAF804C001328242F144D9
:1045E000E044EDD3DBF8002000FB1E229144DAF812
:1045F000002000FB1C229044E26801339342DED38A
:1046000013E4482A28D1394653F09BFCC16904467B
:1046100000230022B8F800C099F8000080EA0C00DE
:1046200021F8020B2069DBF804E0DAF804C001325B
:104630008242F144E044EDD3DBF8002000FB1E226F
:104640009144DAF8002000FB1C229044E268013318
:104650009342DED3FFF7E9BB682A40F089863946EA
:1046600053F06FFCC169044600230022B8F800C073
:1046700099F8000080EA0C0021F8020B2069DBF8B1
:1046800004E0DAF804C001328242F144E044EDD3A0
:10469000DBF8002000FB1E229144DAF8002000FB2A
:1046A0001C229044E26801339342DED3FFF7BDBB86
:1046B000622B40F089800A79622A2CD1394653F066
:1046C00040FCC26904460020134698F800C099F8DF
:1046D000001081EA0C0103F8011BDAF80410D4F889
:1046E00010C0DBF804E003918844991A6145F14455
:1046F000EBD3DBF80010DAF800200CFB1E11894424
:1047000003990CFB11229044E26801309042BFF4FF
:104710008CAB1A46D8E7482A28D1394653F011FC09
:10472000C169044600230022B8F800C099F90000CE
:1047300080EA0C0021F8020B2069DBF804E0DAF8CB
:1047400004C001328242F144E044EDD3DBF80020A2
:1047500000FB1E229144DAF8002000FB1C2290444A
:10476000E26801339342DED3FFF75FBB682A0B4652
:1047700021467FF416AF394653F0E3FBC169044686
:1047800000230022B8F800C099F9000080EA0C006C
:1047900021F8020B2069DBF804E0DAF804C00132EA
:1047A0008242F144E044EDD3DBF8002000FB1E22FE
:1047B0009144DAF8002000FB1C229044E2680133A7
:1047C0009342DED3FFF731BB482B59D10A79482AEF
:1047D00028D1394653F0B5FBC169044600230022B5
:1047E000B8F800C0B9F8000080EA0C0021F8020B0C
:1047F0002069DBF804E0DAF804C001328242F144B7
:10480000E044EDD3DBF8002000FB1E229144DAF8EF
:10481000002000FB1C229044E26801339342DED367
:10482000FFF703BB682A0B4621467FF4BAAE394630
:1048300053F087FBC169044600230022B8F800C08A
:10484000B9F8000080EA0C0021F8020B2069DBF8BF
:1048500004E0DAF804C001328242F144E044EDD3CE
:10486000DBF8002000FB1E229144DAF8002000FB58
:104870001C229044E26801339342DED3FFF7D5BA9D
:10488000682B40F075850A79682A0B4621467FF42B
:1048900088AE394653F055FBC16904460023002217
:1048A000B8F800C0B9F8000080EA0C0021F8020B4B
:1048B0002069DBF804E0DAF804C001328242F144F6
:1048C000E044EDD3DBF8002000FB1E229144DAF82F
:1048D000002000FB1C229044E26801339342DED3A7
:1048E000FFF7A3BA422A40F0A8800B79422B28D1C7
:1048F000394653F026FBC26904460020134698F857
:1049000000C099F8001001FA0CF103F8011BD4F86B
:1049100010C0D6F804A0D5F804E0991A6145D14436
:10492000F044ECD32A6831680CFB1E229044E26804
:1049300001300CFB1A1190428944BFF476AA1A4642
:10494000DCE7622B27D16822394653F0FAFA044695
:10495000C0690023002298F900C099F8001001FAFC
:104960000CF120F8021B2169D6F804E0D5F804C048
:1049700001328A42F144E044EDD3326801FB1E2249
:1049800091442A6801FB1C229044E268013393425F
:10499000E0D3FFF74ABA482B27D11A46394653F0DD
:1049A000D0FA0446C06900230022B8F800C099F884
:1049B000001001FA0CF120F8021B2169D6F804E07E
:1049C000D5F804C001328A42F144E044EDD33268A4
:1049D00001FB1E2291442A6801FB1C229044E268DC
:1049E00001339342E0D3FFF720BA6822394653F0EF
:1049F000A8FA0446C06900230022B8F900C099F85B
:104A0000001001FA0CF120F8021B2169D6F804E02D
:104A1000D5F804C001328A42F144E044EDD3326853
:104A200001FB1E2291442A6801FB1C229044E2688B
:104A300001339342E0D3FFF7F8B9622A40F0A8802F
:104A40000B79422B27D16822394653F07AFA044673
:104A5000C0690023002298F800C099F9001001FAFB
:104A60000CF120F8021B2169D6F804E0D5F804C047
:104A700001328A42F144E044EDD3326801FB1E2248
:104A800091442A6801FB1C229044E268013393425E
:104A9000E0D3FFF7CAB9622B28D1394653F051FA57
:104AA000C26904460020134698F900C099F9001025
:104AB00001FA0CF103F8011BD4F810C0D6F804A0D9
:104AC000D5F804E0991A6145D144F044ECD32A6842
:104AD00031680CFB1E229044E26801300CFB1A1175
:104AE00090428944BFF4A1A91A46DCE7482B27D19C
:104AF0001A46394653F025FA0446C06900230022BD
:104B0000B8F800C099F9001001FA0CF120F8021B66
:104B10002169D6F804E0D5F804C001328A42F14494
:104B2000E044EDD3326801FB1E2291442A6801FB68
:104B30001C229044E26801339342E0D3FFF775B939
:104B40006822394653F0FDF90446C069002300226B
:104B5000B8F900C099F9001001FA0CF120F8021B15
:104B60002169D6F804E0D5F804C001328A42F14444
:104B7000E044EDD3326801FB1E2291442A6801FB18
:104B80001C229044E26801339342E0D3FFF74DB911
:104B9000482A40F0A7800B79422B26D1394653F0A2
:104BA000D0F90446C0690023002298F800C0B9F883
:104BB000001001FA0CF120F8021B2169D6F804E07C
:104BC000D5F804C001328A42F144E044EDD33268A2
:104BD00001FB1E2291442A6801FB1C229044E268DA
:104BE00001339342E0D3FFF720B9622B29D11A4653
:104BF000394653F0A6F9C26904460020134698F9D5
:104C000000C099F9001001FA0CF103F8011BD4F867
:104C100010C0D6F804A0D5F804E0991A6145D14433
:104C2000F044ECD32A6831680CFB1E229044E26801
:104C300001300CFB1A1190428944BFF4F6A81A46C1
:104C4000DCE7482B26D1394653F07BF90446C0698E
:104C500000230022B8F800C0B9F8001001FA0CF1E6
:104C600020F8021B2169D6F804E0D5F804C001320F
:104C70008A42F144E044EDD3326801FB1E229144A4
:104C80002A6801FB1C229044E26801339342E0D37E
:104C9000FFF7CBB86822394653F053F90446C06990
:104CA00000230022B8F900C0B9F8001001FA0CF195
:104CB00020F8021B2169D6F804E0D5F804C00132BF
:104CC0008A42F144E044EDD3326801FB1E22914454
:104CD0002A6801FB1C229044E26801339342E0D32E
:104CE000FFF7A3B8682A40F043830B79422B39467B
:104CF00025D153F026F90446C0690023002298F814
:104D000000C0B9F9001001FA0CF120F8021B21696A
:104D1000D6F804E0D5F804C001328A42F144E044F8
:104D2000EDD3326801FB1E2291442A6801FB1C224C
:104D30009044E26801339342E0D3FFF776B8622BE8
:104D400025D153F0FEF80446C0690023002298F9EB
:104D500000C0B9F9001001FA0CF120F8021B21691A
:104D6000D6F804E0D5F804C001328A42F144E044A8
:104D7000EDD3326801FB1E2291442A6801FB1C22FC
:104D80009044E26801339342E0D3FFF74EB8482BDA
:104D900025D153F0D6F80446C06900230022B8F9A3
:104DA00000C0B9F8001001FA0CF120F8021B2169CB
:104DB000D6F804E0D5F804C001328A42F144E04458
:104DC000EDD3326801FB1E2291442A6801FB1C22AC
:104DD0009044E26801339342E0D3FFF726B853F0E2
:104DE000B0F80446C06900230022B8F900C0B9F940
:104DF000001001FA0CF120F8021B2169D6F804E03A
:104E0000D5F804C001328A42F144E044EDD332685F
:104E100001FB1E2291442A6801FB1C229044E26897
:104E200001339342E0D3FFF700B8422A40F0A88054
:104E30000B79422B28D1394653F083F8C2690446D6
:104E40000020134698F800C099F8001041FA0CF1C0
:104E500003F8011BD4F810C0D6F804A0D5F804E07C
:104E6000991A8C45D144F044ECD82A6831680CFB7F
:104E70001E229044E26801300CFB1A1190428944D2
:104E8000BEF4D3AF1A46DCE7622B27D1682239463D
:104E900053F057F80446C0690023002298F900C077
:104EA00099F8001041FA0CF120F8021B2169D6F89C
:104EB00004E0D5F804C001328A42F144E044EDD365
:104EC000326801FB1E2291442A6801FB1C22904497
:104ED000E26801339342E0D3FEF7A7BF482B27D106
:104EE0001A46394653F02DF80446C06900230022C3
:104EF000B8F800C099F8001041FA0CF120F8021B34
:104F00002169D6F804E0D5F804C001328A42F144A0
:104F1000E044EDD3326801FB1E2291442A6801FB74
:104F20001C229044E26801339342E0D3FEF77DBF38
:104F30006822394653F005F80446C0690023002270
:104F4000B8F900C099F8001041FA0CF120F8021BE2
:104F50002169D6F804E0D5F804C001328A42F14450
:104F6000E044EDD3326801FB1E2291442A6801FB24
:104F70001C229044E26801339342E0D3FEF755BF10
:104F8000622A40F0A8800B79422B27D1682239464B
:104F900052F0D7FF0446C0690023002298F800C0F1
:104FA00099F9001041FA0CF120F8021B2169D6F89A
:104FB00004E0D5F804C001328A42F144E044EDD364
:104FC000326801FB1E2291442A6801FB1C22904496
:104FD000E26801339342E0D3FEF727BF622B28D16A
:104FE000394652F0AEFFC26904460020134698F9D4
:104FF00000C099F9001041FA0CF103F8011BD4F834
:1050000010C0D6F804A0D5F804E0991A8C45D14414
:10501000F044ECD82A6831680CFB1E229044E26808
:1050200001300CFB1A1190428944BEF4FEAE1A46C0
:10503000DCE7482B27D11A46394652F082FF044656
:10504000C06900230022B8F800C099F9001041FAA5
:105050000CF120F8021B2169D6F804E0D5F804C051
:1050600001328A42F144E044EDD3326801FB1E2252
:1050700091442A6801FB1C229044E2680133934268
:10508000E0D3FEF7D2BE6822394652F05AFF0446FA
:10509000C06900230022B8F900C099F9001041FA54
:1050A0000CF120F8021B2169D6F804E0D5F804C001
:1050B00001328A42F144E044EDD3326801FB1E2202
:1050C00091442A6801FB1C229044E2680133934218
:1050D000E0D3FEF7AABE482A40F0A7800B79422B06
:1050E00026D1394652F02DFF0446C0690023002224
:1050F00098F800C0B9F8001041FA0CF120F8021B32
:105100002169D6F804E0D5F804C001328A42F1449E
:10511000E044EDD3326801FB1E2291442A6801FB72
:105120001C229044E26801339342E0D3FEF77DBE37
:10513000622B29D11A46394652F003FFC269044650
:105140000020134698F900C099F9001041FA0CF1BB
:1051500003F8011BD4F810C0D6F804A0D5F804E079
:10516000991A8C45D144F044ECD82A6831680CFB7C
:105170001E229044E26801300CFB1A1190428944CF
:10518000BEF453AE1A46DCE7482B26D1394652F01E
:10519000D8FE0446C06900230022B8F800C0B9F860
:1051A000001041FA0CF120F8021B2169D6F804E046
:1051B000D5F804C001328A42F144E044EDD33268AC
:1051C00001FB1E2291442A6801FB1C229044E268E4
:1051D00001339342E0D3FEF728BE6822394652F0ED
:1051E000B0FE0446C06900230022B8F900C0B9F837
:1051F000001041FA0CF120F8021B2169D6F804E0F6
:10520000D5F804C001328A42F144E044EDD332685B
:1052100001FB1E2291442A6801FB1C229044E26893
:1052200001339342E0D3FEF700BE682A40F0A0802D
:105230000B79422B394625D152F083FE0446C069D2
:105240000023002298F800C0B9F9001041FA0CF1CF
:1052500020F8021B2169D6F804E0D5F804C0013219
:105260008A42F144E044EDD3326801FB1E229144AE
:105270002A6801FB1C229044E26801339342E0D388
:10528000FEF7D3BD622B25D152F05BFE0446C06908
:105290000023002298F900C0B9F9001041FA0CF17E
:1052A00020F8021B2169D6F804E0D5F804C00132C9
:1052B0008A42F144E044EDD3326801FB1E2291445E
:1052C0002A6801FB1C229044E26801339342E0D338
:1052D000FEF7ABBD482B25D152F033FE0446C06922
:1052E00000230022B8F900C0B9F8001041FA0CF10F
:1052F00020F8021B2169D6F804E0D5F804C0013279
:105300008A42F144E044EDD3326801FB1E2291440D
:105310002A6801FB1C229044E26801339342E0D3E7
:10532000FEF783BD52F00DFE0446C0690023002243
:10533000B8F900C0B9F9001041FA0CF120F8021BCD
:105340002169D6F804E0D5F804C001328A42F1445C
:10535000E044EDD3326801FB1E2291442A6801FB30
:105360001C229044E26801339342E0D3FEF75DBD16
:105370000024FEF75ABD00BF38B50C4BD3F8B0304F
:1053800004460D4643B90C204BF048FC2A46214602
:10539000BDE8384000F00CB89A68A24202D15A68C1
:1053A000AA4201D01B68EDE738BD00BFF85C0120C0
:1053B00070B5094CD4F8B0502B462BB9C0E9005257
:1053C0008160C4F8B00070BD9E688E4202D15E68F4
:1053D0009642F8D01B68F0E7F85C012030B5094A26
:1053E00052F8B03F4BB19C6884421C6806D15D689E
:1053F0008D4203D1146000221A6030BD1A46234644
:10540000F0E700BFF85C0120044B1B7823B104488F
:1054100043680BB144F005BA18467047596701203C
:10542000C44F012008B50348012104F0C9FB0E2038
:1054300008BD00BF0C51012070B52DED028B8EB060
:1054400006AB0193574B00930431022301381AF045
:1054500093FA40F28622544906981AF073FB40F200
:10546000076104469FED510A07981AF059FB204640
:1054700004A9B0EE408A41F09DFE0E2200210AA848
:105480004BF0C5FCDFED4A7A9FED4A7A4A4B4B4A16
:105490000A9328EE278AA023C8EE077AADF82C30AD
:1054A00010685168B6EE007A77EE877AFCEEE77AFC
:1054B00017EE903AADF82E3008AB03C3404803A96D
:1054C000FFF75AFF00238DF80E3008AA01230AA91E
:1054D00004A854F0C0FB044630B1394803A9FFF7D3
:1054E0007DFF204643F0AEFE9DF80E3063B1344898
:1054F00003A9FFF773FFBDF80C604FF6FF739E42E0
:1055000005D1304823F04EFBFBF720FAECE70020F2
:1055100029F0F8FF0446B8B16378012B36D123781F
:10552000DB0733D506220DF1110104F151004BF0D8
:1055300019FC58BB04F1240204F13601304654F042
:1055400098FBB0FA80F46409002502A93046ADF852
:10555000085054F092FB4FF40071304654F0A3FB16
:1055600043F070FE29462A46304654F078FB43F05B
:1055700069FE154B882101FB05F2D0189A5AB242F8
:1055800006D00135052DF6D11048BBE72046BFE710
:105590000123837080F85A4000F0B4FD0EB0BDECDA
:1055A000028B70BDD41A0A0060AC09000000000034
:1055B0000024744900401C460001A000F8D80800EF
:1055C0005BBD0700DE430900A0090120E643090096
:1055D00037B5012104F0F4FA684654F02AFB43F091
:1055E00031FE09490C204DF0C3F8062104460DF1A7
:1055F00001009DF8005020F0E7FFC5F34605A060CC
:105600002046257103B030BD60AC09002DE9F041A2
:105610000746806986B0F0B9104D044606464FF63D
:10562000FF782B8843450CD0E86D0E2803D128461F
:1056300000F068FDE86506AB03EB8403013443F832
:10564000140C0136052E05F18805EAD101A9204682
:1056500021F0F2F9B86106B0BDE8F081A00901209F
:1056600008B501483AF032FE2846090010B50C464C
:1056700086B0A068012203A91DF002FF88B19DF841
:105680000430227962F347038DF80430039B1A68D3
:10569000CDF805209B88ADF8093001A854F0CBFA6D
:1056A00010B1034823F07EFA0E2006B010BD00BFF3
:1056B000354509002DE9F04F2DED028B95B00CAB6F
:1056C00051F8044B01935F4B0093013808231AF003
:1056D00053F90C98052209A91DF0D2FE0D9800235C
:1056E0000E28CDE90633089303D0052206A91DF044
:1056F000C7FE119808B9544811904FF484611AF00C
:1057000037FADFED527AB4EEE70AF1EE10FAB0EEB6
:10571000408A06D4DFED4E7AB4EEE70AF1EE10FAD5
:1057200004DD4C4A4C494D483AF034FEDDF840A0C7
:10573000BAF1000F04DA40F2076100201AF0AEF966
:105740000A9B9DF838601F2B05D926B1079B13B122
:10575000434823F027FA13980E280DD00EB941487C
:10576000F7E7414940F263321AF0ECF9074694F842
:1057700044301BB13D48ECE70027F8E7E3689DF8AB
:105780003C80DDF8489013B1204604F077FB0A9D79
:105790003146284603F0DEFADDF81CB031465846A3
:1057A00003F0D8FA1F2D04D9BBF1000F02D0304806
:1057B000CFE715B10FB12F48CBE7B8F1000F09D1F2
:1057C0002D4B2E4A03FB0AF3934205D92C48B421F2
:1057D00023F0E8F94FF0B40A616819B9FF2011F01D
:1057E00045FC6060A16819B9FF2011F03FFCA06082
:1057F000DDE9091260684BF0C9FADDE90612A0681C
:105800004BF0C4FACDE90497BDF81C300393A368AC
:105810000293BDF82830019363680093B0EE480A04
:105820005346424631462046F4F7D6FE43F00AFD81
:1058300001230E2084F8443015B0BDEC028BBDE886
:10584000F08F00BFD4190A00CECC4CBE0AD7A33CBF
:105850000AD72341251909002B1909005C330900D7
:10586000F24509007740090060AC0900874709004C
:105870001B440900FA44090040420F000FBCBA0A59
:10588000A43D09002DE9F04F2DED068B93B00AAB36
:1058900051F8044B0193834B0093013808231AF00D
:1058A0006BF80D980E2828D09FED7F0A40F2076113
:1058B0001AF036F9F0EE408A0E9808B97B480E903F
:1058C0000F9B0BB9794B0F934FF484611AF050F989
:1058D000DFED777AB4EEE70AF1EE10FAB0EE408A27
:1058E00006D4DFED747AB4EEE70AF1EE10FA07DDC4
:1058F000714A724972483AF04DFDDFED6B8ADBE781
:10590000F5EE408AF1EE10FA07D0F4EEC08AF1EE1F
:1059100010FA02D56B483AF035FD0F984FF4CD617F
:105920001AF026F9B4EEC08AF1EE10FAB0EE409A01
:1059300001D56548EFE70A980023049358B1052282
:1059400003A91DF09DFD049B2BB1039812F014F9DF
:1059500008B95E48DFE70B9F002F04DC4FF4397174
:1059600001201AF09BF823699DF83050DDF8409033
:105970009DF84480DDE903BA3BB193F8293013B9AF
:10598000534823F00FF900232361E36843B16268B1
:10599000934202D1112003F0A9FA204604F06EFAD6
:1059A0004C499FED4DAA2C204CF0E2FE39460646AC
:1059B000083053F0AFFF002DC6E907BAC6F82490AF
:1059C00026610CBF1F26FF2606F108004BF044F9A4
:1059D0002369586000F108030360868007460120B0
:1059E00041F02CFF43F02EFC21693C48FFF7C4FC3A
:1059F00068EE8A6A9FED3A7AC6EE877AF6EE009AEA
:105A000077EEA97AFCEEE77A17EE906AB6F5803F5A
:105A100001D334487FE736B9F5EEC08AF1EE10FACB
:105A200001DD314877E70E22002106A84BF0EFF99F
:105A300028EE0A8A9FED2D7AADF81E60C8EE077A2F
:105A400045F4807545EA880525F0FA05394606A82B
:105A5000ADF8185029EE0A9A77EEA97AFCEEE77AAB
:105A600017EE903AC9EE077AADF81A3077EEA97AB8
:105A7000FCEEE77A17EE903AADF81C3054F005F9D9
:105A8000054640B115482169FFF7A8FC00232361B2
:105A9000284643F0D7FB206913B0BDEC068BBDE868
:105AA000F08F00BF141A0A0000000000CECC4CBEDC
:105AB0000AD7233B66D62342301909003A19090058
:105AC0005C330900BD300900952B0900E43F090053
:105AD000083F090088AB090000247449C976060014
:105AE00000401C464D2D0900CD30090000401C44EB
:105AF000022838B50D46144610D193070CD1126810
:105B0000084B9A4208D1A168A8684CF0FAF918B17C
:105B10002A7923799A4203D01E2038BD0020FCE761
:105B20003E20FAE760AC090030B589B0084611465E
:105B30001A4603AB0193134B009302234BF0B3FAC5
:105B400005A9039805221DF09BFC069840F28622C9
:105B5000062119F0B5FF40F28923032204980021A1
:105B60004BF0D4FA084905460C204CF001FE062102
:105B70000446059820F028FDA0602046257109B054
:105B800030BD00BFC41A0A0060AC090010B50B4656
:105B900088B0044605A9986805221DF071FC059996
:105BA00008780B794A7903904878029088780190B8
:105BB000C9780091204602494CF0F2FF08B010BDB0
:105BC00041190900062837B50D4618D18C680D4BD0
:105BD0002340062B11D1200953F0F8F930B901A95F
:105BE000204621F051FE019953F0C7F92B79584016
:105BF000400040F0010003B030BD6068EEE70020D7
:105C0000F9E700BF0F0080FF2DE9F04F97B00DAB13
:105C10000193344B009304310923013819F0ACFE91
:105C200031490D9840F28A5219F08CFF2F490890A3
:105C300040F24A620E9819F085FF9DF83C603F2EB5
:105C4000834603D94FF49F6019F088FE9DF8407099
:105C5000384643F0D4FD9DF84480404643F0CFFDE4
:105C6000129C002C04DA40F26B41002019F016FF60
:105C700014989DF84C500E2804D15DB354B32046BF
:105C80004CF0A1FD0DF12809052249461DF0F8FB55
:105C90000B9840F214422146F5B119F011FF159806
:105CA0000E281CD021F018FE8246114928204CF005
:105CB0005FFDCDE9059ACDE90345CDE90178089965
:105CC00000965B460022099004F040F9099817B04D
:105CD000BDE8F08F0748D5E719F0FEFEDFE74FF08B
:105CE000000AE2E77C1A0A0068AB090040AB090031
:105CF00014AC0900505A090010B54368044653B16A
:105D000001460648FFF76AFB0023C4E90333C4E9F0
:105D10000633636063610E2010BD00BFF39007007F
:105D200070B52DED028B86B0084611461A4603ABBE
:105D300001931F4B009303234BF0B5F91D490398C2
:105D400040F2FA2219F0FEFE40F207610646B7EE75
:105D5000000A049819F0E4FE059D002DB0EE408A7B
:105D600004DC4FF43971012019F098FE1249242007
:105D70004CF0FEFC044628464AF06EFFDFED0F7A39
:105D8000666028EE278A0023BCEEC88AC4E90305B2
:105D9000C4E905330A4884ED028A84F82030E361BF
:105DA0002146FFF7E9FA204606B0BDEC028B70BD34
:105DB000541A0A0014AC0900F0AB090000007A4440
:105DC000F390070008B501483AF080FAA0450900B1
:105DD00010B50446808A43F010FAE3692BB1BDE8A0
:105DE0001040D3E9020120F027BE014810BD00BFDA
:105DF000A029090070B58B6804460D4616466BB1A4
:105E000007494CF0CDFEA9682046324600F03EFE20
:105E100004492046BDE870404CF0C2BE0249F9E793
:105E200069190900531A090079190900F0B50C46DF
:105E300085B054F8045B0646A88A174643F0DDF99E
:105E400002AB0193084B00933A4602232146701E91
:105E500019F092FD28469DF80C209DF8081004F0DA
:105E6000A7F90E2005B0F0BD6C1A0A0008B501486C
:105E70003AF010FAE4400900084930B500228825BC
:105E800005FB02F463180C5B844204D00132052A3E
:105E9000F6D1002030BD1846FCE700BFA009012064
:105EA0002DE9F04F8BB004AB51F8048B0193784B84
:105EB00000930138012319F05FFDD8F80440204613
:105EC00000F0F6F87348049D2146FFF755FA0020CC
:105ED00016F00EFF0E2D606030D101210AE06268DD
:105EE0009368D26803F18043013B52F82330D98A8A
:105EF000013189B2002220460BF01CFE0028EED1B1
:105F0000654F002663689A68964236D321466148F9
:105F1000FFF764FAD8F80440204600F0C9F8636837
:105F2000D3E9020120F088FDD8F80430044658680F
:105F30004CF0B4FB20460BB0BDE8F08F284606A914
:105F40001DF00AFB554E054628461DF0C7FC0028EB
:105F5000D6D0830702D10368B34202D050483AF04A
:105F6000FDF98388ADF8143005AA83798DF81630D1
:105F7000012120460BF0DEFDE6E7DB6853F82650F2
:105F8000AB680BB90136BDE7AB8ADFF81C91EA8A32
:105F90009A4212D3ADF81830DFF810A1C9F80050BA
:105FA0000023ADF81A203B702088012306A98AF847
:105FB000003053F074FE00283DD02B699B6802939B
:105FC0000023029A9A42DDD02A69D1685A1C0392B2
:105FD000029A51F823B0501E834216BF01EB830191
:105FE00000234B68DBF8081009B3BBF8141001312B
:105FF00089B2002B32D09B8A013B1FFA83F9E88AD1
:10600000884214D3494512D8264BADF81810DFF852
:106010009CA0C3F800B000213970ADF81A9001219E
:106020008AF80010208806A953F03BFED8B1039BE4
:10603000C7E7FAF78BFC9AF80030002BF9D13B78D0
:10604000002BBAD02A699368D26803F18043013BE0
:1060500052F823309B8A01339BB298E7B5F816902B
:10606000CDE7FAF773FC9AF800100029F9D13978D6
:106070000029DCD0DBF81C008168C06801F1804198
:10608000013950F82110898A013189B2B7E700BF80
:106090001C1B0A00751B04001A69012040AB090093
:1060A000F6300900D85C0120D45C01201969012078
:1060B00008B543F0C6FB10B901483AF0EBF808BD4B
:1060C0006445090038B544680D4D2046FFF7F0FFE0
:1060D00094F874306BB9B4F86C3000EE103AB8EE46
:1060E000C00AF7EE047ABDE8384020EE270A20F017
:1060F00017BBAB6A002BEED1FAF728FCE8E700BF2C
:10610000F85C012010B50446C06D0E2805D1034986
:106110000C204CF02DFB4460E06510BD30AC090054
:1061200030B585B003AB51F8044B0193224B00937B
:106130000138012319F020FC9DF80C3033B91F48B9
:106140004FF4A67240F2DB213AF0C8F864681C4DA7
:106150002046FFF7ADFF94F85A30012B01D1AB6A0E
:10616000EBB194F85A30022B22D00123154984F860
:106170005A302088124D53F068FD43F063F894F8CC
:106180005A30012B01D1AB6A63B1AB6A83B994F881
:106190005B1069B1882908D10B4822F011FDFAF78C
:1061A000D5FBD8E7FAF7D2FBE9E7084822F008FD6B
:1061B0000E2005B030BD00BF241B0A00DD480900D9
:1061C000F85C012074180A00253C09007F3C090096
:1061D0002DE9F04796B00FAB0193544B0093043177
:1061E0000723013819F0C8FB51490F9840F2FA22F1
:1061F00019F0A8FC4F4940F24A620746109819F07E
:10620000A1FC9DF844908246484643F0F8FA9DF878
:106210004880404643F0F3FA139E002E04DA40F221
:106220006B41002019F03AFC15989DF850500E284B
:1062300004D14DB346B330464CF0C5FA052204A94B
:106240001DF01EF9059840F214423146F5B119F0DF
:1062500037FC394918204CF08BFAC0E9017A002349
:106260000446838280F8169080F81780DDE90401E7
:1062700020F0AAF9E060002D4FD1B6F5007F08DDCF
:106280002E4A4FF400714EE02D48D7E719F024FC58
:10629000DFE72682A574FB69002B3AD0A368A17DB5
:1062A0009A889B798DF80E3085F001050DF108086C
:1062B00045F002050026404605F00705ADF80C2024
:1062C000ADF808608DF80A5042F002FAE17D0DF158
:1062D000090042F0FDF9052207A9E0681DF0D0F899
:1062E00003ABCDE90A38089BADF83030238AADF80E
:1062F00034300AA9079BB88A0E9304F11402ADF852
:10630000326053F0E0FC42F09DFFF86921464CF00A
:10631000A2F9204616B0BDE8F087B6F5FF7FB8DDDC
:10632000084A4FF4FF7108483AF034F8E41A0A00BA
:1063300014AC090040AB0900D4AB09009DD908009A
:10634000505A0900A8D908003C32090070B58B6882
:1063500004460D4616466BB107494CF021FCA9686E
:106360002046324600F092FB04492046BDE87040CA
:106370004CF016BC0249F9E7A1190900531A0900AB
:10638000AD1909007FB504460522084601A91DF094
:1063900077F8A58A65B163685E68F06842F06BFAC9
:1063A000B37901463BB1002301AA284642F0E7FA3F
:1063B0000E2004B070BDA07C029B228A20B19A42BC
:1063C00006D0064839F0DEFF9A4201D20448F9E7C8
:1063D00001AA284642F0FAFAEAE700BFE53B0900C5
:1063E000DA3B0900022A70B504460E4615460BD169
:1063F0004FF41C7052F0FEFD014620464CF0C1FBEC
:10640000054920464CF0BDFB2A4631462046BDE8F2
:1064100070401EF013BE00BF92D9080070B506464A
:1064200086B008460D46144642F015FA00234FF494
:1064300000722048019401A9CDE90223ADF8105063
:106440008DF81430FEF798FF00223146284653F0AD
:1064500030FC11280446F7D030B1164801A9FEF7E8
:10646000BDFF204642F0EEFE9DF81430B3B1BDF8FA
:10647000100042F0F0F901A90E48FEF7AFFFBDF899
:10648000121089B291B140F20513994209D040F23D
:106490000F13994208D0084822F084FBFAF756FA05
:1064A000E2E7064822F08CFB0548FBE7039806B0BC
:1064B00070BD00BF017207009A3C09001943090032
:1064C0001043090008B5014839F05CFF7F4109001D
:1064D0002DE9F04788B0084611461A4605AB0193EE
:1064E0002D4B009303234AF0DEFD2C49059840F222
:1064F000FA2219F027FB069D002D074604DC4FF415
:106500003971012019F0CAFA07980E2836D17E8A0F
:10651000234930204CF02CF940F2FD139E4228BF55
:106520001E467B68BA7D9B7902F03004804602F0FB
:10653000060213B9134622461C4642B306F102096D
:1065400005FB09F948464AF087FB054614B3304677
:106550004AF082FB824630464AF07EFB0446002326
:10656000CDE902634046CDE900A44B462A463946B0
:10657000F4F712F9404608B0BDE8F08740F26D41EB
:1065800019F00EFB061EC3DC40F26D41B9E715465B
:106590009146DBE7A246E2E75C1B0A0014AC090067
:1065A000B8AB090030B50D4685B00446406842F0EE
:1065B0001FFE062201A928461CF062FFDDE9011238
:1065C000204643F08AF9002803DA4142034839F0B3
:1065D000E1FE400040F0010005B030BDAE460900CC
:1065E00010B58AB002AB0C460193144B00930431F2
:1065F0000223013819F0C0F92468606842F0F8FD00
:106600000298052207A91CF03BFF039800230E28DF
:10661000059303D0052204A91CF032FF059B0093CB
:10662000DDE90712049B204603F0A0FE20EAE0709B
:10663000400040F001000AB010BD00BF4C1B0A0032
:10664000F8B5354C354B236043F0BAF8002861D0DB
:10665000334B1A781AB9334A1278012A28D13248B2
:1066600000251D7003F058FE304B9A8A02B19D82BE
:106670002F4B9A8A0AB100229A822E4D6B68BBB1C9
:106680002D4B1B78A3B1284603F058FE284603F093
:1066900043FE2A4B9A8A0AB100229A82284B9A8A90
:1066A0000AB100229A82274B9A8A0AB100229A8262
:1066B000194803F001FCE36813B1174803F0DEFB4F
:1066C0000023214DA3614FF6FF7705240E2628886D
:1066D000B84202D0132153F0CAFA013CEE6505F12D
:1066E0008805F4D154F068FE0B48214603F068FA9F
:1066F0004FF42A23154A1B68934205D14FF43122E7
:10670000D2F8FC2F9A4201D000F072FBBDE8F840AD
:1067100035F04EBCF8BD00BF0C51012088AC09001B
:10672000626801204B690120EC4F012020620120AA
:10673000506201201C500120596701205061012046
:10674000A0610120D0610120A00901203130444224
:1067500030B589B003AB51F8045B01930E4B009345
:106760000138022319F008F99DF81040039805A993
:1067700005221CF085FE84F00104E8680094DDE940
:106780000523D0E9021042F065F900280CBF1E2055
:106790003E2009B030BD00BF3C1B0A007FB5084653
:1067A00011461A4602AB0193104B009302234AF0A4
:1067B0007AFC40F24A6202980D4919F0C3F90D497A
:1067C0009DF80C60054618204BF0D9FF04460020C8
:1067D00016F08EFA324603462946204640F0AEFABD
:1067E00042F030FD204604B070BD00BF2C1B0A00F3
:1067F00040AB090068AB090070B58B6804460D46D4
:1068000016466BB107494CF0CBF9A96820463246D1
:1068100000F03CF904492046BDE870404CF0C0B996
:106820000249F9E7D1190900531A0900DA190900D8
:1068300008B5014839F04AFD773F090010B5022834
:1068400088B00B46144624D1A20720D12168124AF1
:1068500091421CD19A79012A09D1A279012A06D143
:106860009A88A3889A4212D13E2008B010BD1846DB
:10687000694643F079F804A9204643F075F81022E0
:106880000DEB020168464AF06DFA0028ECD01E209C
:10689000EBE70020E9E700BF40AB090008B58B78C3
:1068A00013B9044822F07EF90B8883808B788371BA
:1068B00008BD00BFA73C09001FB58379012B02D199
:1068C000054839F0DFFC694643F04EF81021684670
:1068D0001FF07AFE05B000BDB0300900F0B51C46CF
:1068E00008468FB011464FF0021219F00DF82068DB
:1068F000C20706D410F0030317D10168414A914240
:1069000013D14BF062FBA2234FF6FF7200214AF035
:10691000FDFB3D49054608204BF02AFF01230446B4
:106920008580837120460FB0F0BD384A0240062AA8
:1069300005D0002B4DD10268354B9A4249D101A9AF
:1069400020F0A2FF019B242B02D0324839F01AFD1F
:10695000037A2D2BF9D1437B2D2BF6D1837C2D2B64
:10696000F3D1C37D2D2BF0D1461E00F12304002569
:1069700016F8017F384639F065FC28B105F1380377
:106980006B44013503F8207CB442F1D1202DDCD1D9
:1069900006AD0F2402AE287855F085FF07466878CB
:1069A00055F081FF40EA0710A055013C631C05F13A
:1069B0000205F0D100231449BDF81450ADF814308D
:1069C00008204BF0D5FE02A98580044642F0B6FFB0
:1069D000A8E7012206A91CF053FD08B90E48B5E747
:1069E0000798A222102119F06BF8069B02AC03F164
:1069F000100518685968224603C20833AB42144692
:106A0000F7D1D7E7E42A090040AB09000F0080FF67
:106A1000582909000E3D0900FF3C0900F0B589B076
:106A200003AB51F8044B0193174B00930138022339
:106A300018F0A2FF062205A903981CF021FD069F6D
:106A40000498002140F2B1433A464AF05FFBA67930
:106A5000012E14BF802110210546C90840F2E3220F
:106A6000381A4AF05FFB059B012E03EB050107D1A5
:106A7000A2885A55A3881B0A4B700E2009B0F0BD9E
:106A8000204642F071FFF8E7FC1B0A0010B58A7936
:106A9000012A92B0044606D18A881F4912B0BDE887
:106AA00010404CF07DB808460EA942F05DFF9DF8FD
:106AB00038300D939DF839300C939DF83A300B9394
:106AC0009DF83B300A939DF83C3009939DF83D308A
:106AD00008939DF83E3007939DF83F3006939DF84C
:106AE000403005939DF8413004939DF84230039364
:106AF0009DF8433002939DF8443001939DF8453052
:106B000000939DF847209DF84630044920464CF0FC
:106B100047F812B010BD00BFFB190900081A0900A0
:106B20002DE9F0472DED048B84B002AB0193344B7B
:106B30000093022318F020FF039C0E2C04D14FF485
:106B400080504BF032FE04460221204648F0B6FF4A
:106B5000074660B920461EF0DFFDC3880093294830
:106B600040F257232E2240F2F45139F0FFFBDDF8BA
:106B700008809FED258ADFED258A002507EE905AD3
:106B8000B8EEE70A07EB851920EE080A1FF0C8FDEA
:106B900000268246B7EE009A07EE906AB8EEE70A42
:106BA00020EE080A1FF0BCFD5146024640464AF05E
:106BB000B9FB1EF027FDB5EEC00AF1EE10FA1AD4AB
:106BC000B4EEC90AF1EE10FA17DC20EE280A30F014
:106BD000F3F8FCEEC07A17EE903A09F80630013669
:106BE000402ED9D10135402DC8D1204604B0BDEC8E
:106BF000048BBDE8F0870023EFE70123EDE700BF3A
:106C000084210A003D4909002108823C00007C42A1
:106C10002DE9F04F754C85B0002600AFA4F10808AF
:106C20004FF0880909FB068393F87830002B65D074
:106C300054F0C2FBD4E91E23801A61EB0301B0F5C6
:106C40007A7F71F1000159D3002134F8080CF980E2
:106C50000323BA1D6D4653F044F8002847D1FB8842
:106C600034F8080C0733DB08A5EBC3039D46BA1DB7
:106C700003236946EA4653F034F8002837D1B4F8C4
:106C8000502014F8060C022148F03BFC834660B10A
:106C9000FB88C2889A4205D100F1080168464AF093
:106CA00061F820B3584649F07BFB00233B7214F88F
:106CB000063C3A89F888F88143F4007302F0FE023A
:106CC00023F0FE0313433B81B4F850307B8134F84A
:106CD000083CBB810FF07CF90222834607F10801D2
:106CE00030F05CFEFA885146584656F033FB882354
:106CF00003FB06830022AD4683F8782009FB068358
:106D000093F87930002B41D014F8060C002847D0B6
:106D1000B4F82EA05246012148F0F3FB054650B1CD
:106D2000C288502A04D1214608304AF01BF840B3EB
:106D3000284649F035FB002028F0E4FB054690BBCF
:106D4000387214F8063C3A89A7F80AA043F4807315
:106D500002F0FE0223F0FE03134350253B81284638
:106D600034F8083CBB81FD810FF032F902228246E3
:106D700007F1080130F012FE2A462146504656F02F
:106D8000E9FA09FB0683002283F879200136052EF3
:106D900004F188047FF446AF1437BD46BDE8F08F98
:106DA000B4F812A0B6E76B78012B1DD12B7814F83C
:106DB000062C03F001039A4216D1B5F806B0BBF1D8
:106DC000500F11D1062204F1490105F1510049F09B
:106DD000C9FF48B95A46214605F1080049F0C2FFEB
:106DE00010B1284649F0DCFA2846A5E7A809012099
:106DF00073B5104D4FF42A244FF00106200B2E706E
:106E000052F08BFF08B930F0B9FD04F58054B4F5A9
:106E1000322FF3D1084B019301A901224FF42A200C
:106E200030F0BCFD0548012201A930F0B7FD02B0E9
:106E300070BD00BF3069012031304442FC1F0B009F
:106E4000032A05D11E2914BF044905494BF099BEF8
:106E50001E2914BF03490449F8E700BF41D90800BF
:106E600046D90800A8D908009DD9080030B587B0D8
:106E70000C460592D1E90123174904935528CDE921
:106E80000212236809D054F8042C02A9184620F0F5
:106E900047FEA4F1080007B030BD184600931EF06D
:106EA0003BFC827B009B82B100EB820002A905695A
:106EB000019318460422A8470090F6F7E9F9DDE9A6
:106EC000000310B120602046E5E718464BF089F832
:106ED0000146024839F04AFA34540900734809005F
:106EE0002DE9F04F2DED028BB9B00AAF08461146DF
:106EF0001A4607F150030193BA4B00931A234AF044
:106F0000D2F83B6D786D3B60052207F144011CF01F
:106F1000B7FA4FF42E71D7F890003BF027FCF863D6
:106F2000D7F898001EF06EFBD7F868B05A229BFB8A
:106F3000F2F302FB13B3B0EE408A13B1AA4839F062
:106F400021FA97F8B0A0FE6EBAF1000F08D0012E1A
:106F500006D0A64840F21A2240F20E3139F01AFA51
:106F6000F5F746FBA24B036097F88450B7F9603001
:106F70007D6297F888503B633D62B7F9643097F8BB
:106F80008C50FB62FD6197F870307D6C7B63BD6156
:106F900097F8A030BD6C7D610446B7F8945097F81F
:106FA0007400FB6097F8A43097F87CC097F880E0F5
:106FB000B7F85810B7F85C20D7F8A890B8623D61D0
:106FC00097F8780097F89C50BB6397F8AC30BB609B
:106FD0004FF00008D7F8B4307B6084F8B380CDE977
:106FE00004CE0390BB6A02937B6BB6B2CDE900631B
:106FF00004F108001FFA8BF346F0B3F804F15003D4
:107000007B63012E14BF00230AF00103CDE907833F
:10701000CDF82480FB6806934FF48073CDE90433E8
:107020003B6A03937B6A0293FB6A01933B6B009379
:10703000C5F58075ABB21A46396804F150000BF003
:10704000B3F8FB6984F8B2303B69A4F8AC30BB6B91
:10705000A4F8AE9083F0010384F8B430BB6884F8E0
:10706000B5301FFA89F94FF47A73B3FBF9F3A4F83A
:10707000B030BB8AFB62C346FB6A9B4537D35D4B8E
:10708000C4F88430FB6BD3B1187942F092FFB0B1F1
:1070900000220092BB88F96B04F1840005F084F8AB
:1070A000002800F08B80544BC4F88430F96B04F155
:1070B000840042F0BBFCFB6B187942F08FFFB0EE0E
:1070C000480A204603F0D0F94C4991F82A309B0732
:1070D00002D4204642F067FCB96B204642F04FFCD8
:1070E0002046BC37BD46BDEC028BBDE8F08FBB69C6
:1070F00003EB0B0898F80150786B0BF047F8002869
:107100003AD094F880906BB23B6305F07F05B9F1FB
:10711000000F3CD005F1080303F0F803E946ADEB9E
:10712000030D98F800208DF828200AAB6E1C2A4623
:1071300008F102010DF12900BB6249F027FE00961B
:10714000266EBB6A206D01220021B047CD46786BC8
:1071500045F082FE3B6B002B2DDA6E1C023518F8D1
:107160000500FF2808BF4FF4FA701CF045FA0BF138
:10717000020306EB030B7FE7F9F7E8FB204B9B6A62
:10718000002BB9D01F4840F26D3139F0D1F80123FE
:107190000093B5EB0902206D266E434618BF01220D
:1071A0004946B0470095206D266E08F102034A4615
:1071B0000121B047CBE72E460A20D6E7124BD4F880
:1071C0008800C4F884302DF0B9FD94F88C200F4964
:1071D00002F07F02012393400A5C13430B54D4F85E
:1071E000903069E78C240A009A4409008A49090012
:1071F00058BF0900085C090098BE09004001012041
:10720000F85C0120BE490900FCB709001D69012096
:10721000F0B58DB002AF07F108030C460193264B81
:10722000009304310223013818F0A6FB206823F0F4
:1072300067F9D7E902650446062207F11C012846D2
:107240001CF01EF994F83A30102B02D01B4839F08C
:1072500099F8A28E386ABA8202F00103002103EB8A
:1072600052033961B0EB830F7E8206F10106B961EA
:10727000FE821ED3520901327A607A68FB6992005D
:10728000073222F00702ADEB020D02AA8C467E689F
:1072900088B2864209D807F1100104F1080045F0D0
:1072A00096FF28462C37BD46F0BD42F820C001317C
:1072B000EDE70348CBE700BFF4250A00AC44090022
:1072C000A746090008B5014839F02AF8CF46090059
:1072D0007FB502AB0C4601932B4B00930431022384
:1072E000013818F049FB206823F00AF9039B044693
:1072F0000298002BCABF4FF47A764FF0FF3696FB08
:10730000F3F60E2811D04AF060FE4FF47A7595FB23
:10731000F0F594F8B3305BB10023204684F8B43024
:107320003FF0E1FF3E2004B070BD4FF0FF35F0E7C5
:1073300094F8B430002BEFD16B1CEDD054F03CF836
:107340002369C31A9E4202D2104838F0E9FFD4F8EC
:10735000A020821A9542C4E9280112D3B3FBF5F2AA
:1073600005FB1233ED1A54F027F8D4E92832C01A7D
:1073700061EB0201A84271F10001CDD2F9F7E6FA02
:10738000F1E71E20CFE700BF7C240A00FF4609007A
:1073900038B50D4623F0B4F8044628461EF032F9FD
:1073A000B5EEC00AF1EE10FA06D4B7EE007AB4EEEC
:1073B000C70AF1EE10FA01DD00F00CF8204603F0E8
:1073C00053F810B9024838F0ABFF0E2038BD00BFAB
:1073D000CF46090008B503480123002240F2E1210D
:1073E00038F0D8FF9449090008B5014838F04AFF41
:1073F000F34709002DE9F04786B0084611461A46C2
:1074000002AB0193674B0093042349F04CFE40F21A
:10741000775102983BF09EF940F27A510546039865
:107420003BF098F9604906460C204BF0A8F9FF2381
:10743000DDF8108083722A7933799A42044603D1A9
:107440004FF49C6018F08AFA00234360574B1A7A75
:1074500022B11A7E002A40F0A280012203EB02131F
:1074600063602879012128F0D5F80121307928F0CE
:10747000D1F80A2028F02CFA2879002128F0CAF83F
:107480003079002128F0C6F8032028F021FA30795D
:1074900028F012F940B930792EF054FD28792EF0F9
:1074A00051FD434838F03CFF287928F005F90028C1
:1074B000F1D0404B96F804902F79984522D83E4B56
:1074C00098458CBF4FF080684FF0CC786772307968
:1074D000A07201F0ADFE2879384D01F0A9FE636875
:1074E00001221A72666896F804A0342101FB0AF1A1
:1074F0006B1893F82D2042B1204603F063F8052065
:1075000038F0F8FE4FF0C868E0E71F2F9A6083F864
:10751000302083F82F2083F832205E608ABF07F086
:107520001F033B46264A2748685098BF4FF0A042A9
:1075300003F5E073B9F11F0F40F20C6142F823101C
:107540008CBF09F01F034B4603F5E0738CBF1C4A48
:107550004FF0A04240F20C6142F823103368C3F8A8
:107560000875C3F80C95C3F82485342303FB0AF38C
:10757000EB5853B13068072140F30730F1F7DEFDD7
:10758000306840F307303FF02BF8342303FB0A55F3
:107590002046012385F82D3006B0BDE8F0870A4863
:1075A00038F0F0FED4250A003CBF09005404012045
:1075B000514109007F1A06008FD003001C5C012096
:1075C0000003005099C60800C2470900F0B50C46F8
:1075D0008DB054F8045B0646A87A174641F0F1FDD9
:1075E000284641F029FE08AB01931D4B009321462C
:1075F0000423701E3A4618F0BFF9062205A909981F
:107600001BF03EFF9DF81C100022402018F0F8FAF5
:10761000069B0B99B3FBF0F30446049304AA0A9B60
:10762000039303A850F09EFD049E40F2E322012143
:10763000304649F077FD039A06FB04F36243039258
:10764000049353B1059928460A44BDF8201003F06D
:107650003BF810B1404238F04DFE0E200DB0F0BDA9
:10766000B4250A00F0B50C468DB054F8045B06460C
:10767000A87A174641F0A5FD284641F0DDFD08AB8C
:1076800001931A4B0093214604233A46701E18F0CA
:1076900073F9052205A909981BF0F2FE9DF81C104C
:1076A0000022402018F0ACFA069B0B99B3FBF0F3D4
:1076B0000446049304AA0A9B039303A850F052FDC6
:1076C000039A049B0121009105996243039263434D
:1076D0000A442846BDF820100493F3F7C3F810B10C
:1076E000404238F007FE0E200DB0F0BD94250A0090
:1076F0002DE9F0410C4694B054F8046B0546B07A7D
:10770000174641F05EFD304641F096FD0DAB01930A
:10771000314B00933A4607232146681E18F02CF996
:1077200005220AA90E981BF0ABFE9DF8301000222E
:10773000402018F065FA0B9B1199B3FBF0F3054656
:10774000069306AA109B059305A850F00BFD062290
:1077500007A90F981BF094FE9DF8241000224020EA
:1077600018F04EFA089B1399B3FBF0F30446049308
:1077700004AA129B039303A850F0F4FC049F40F268
:10778000BD420121384649F0CDFC0598069BBDF865
:107790003480002268436B430092039D0A9A05904F
:1077A000654302447C4341463046079F0693039558
:1077B0000494F3F757F838B94CB123467A19414687
:1077C000304602F081FF10B1404238F093FD0E20A8
:1077D00014B0BDE8F08100BF5C250A00F0B50C468E
:1077E00087B054F8045B0646687A174641F0E3FC1C
:1077F000284641F021FD02AB0193184B009321462E
:10780000701E04233A4618F0B7F840F2E94301220B
:107810000021039849F07AFC40F2D943012200216B
:107820000446049849F072FC40F2CA230646092235
:107830000598082149F06AFCC0B2082802D005204A
:1078400038F058FD0299F3B2E2B2284642F0B4F89B
:107850000028F4D00E2007B0F0BD00BF6C260A004F
:107860002DE9F04F89B0084611461A4604AB019342
:10787000744B0093042349F016FC40F20331049842
:107880003AF068FF40F29141074605983AF06EFFE2
:1078900040F28241044606983AF068FF064618B95D
:1078A00014B9694838F06EFD68490C204AF067FF4A
:1078B0009DF81C30FF220546427223B164484FF404
:1078C0007D7138F00BFD4360624BD3F8003513F047
:1078D0000F0305D0604BD3F800351B0711D10123EE
:1078E0005E4A02EB03136B6097F80480D3F808A09C
:1078F00085F80980404601F09BFC24B9FF24AC7256
:1079000006E05748CEE72479AC72204601F090FC9F
:107910000EB33679EE72304601F08AFCD5F804B029
:10792000504F9BF80490242303FB09731B7F63B91A
:107930005046F9F749F80290B9F1000F0ED1B0F1B5
:10794000206F02D0B0F1A05F0BD1284602F000FFFB
:10795000052038F0CFFCFF26EE72DFE7B9F1010F0A
:10796000F3D1242202FB09F2B8180021DBF800A0B1
:1079700041604046B95027F081FEB8F11F0F8BBF20
:1079800008F01F02424638494FF0A04102F5E0726C
:107990000120FF2C41F822004AD0204627F06EFE3D
:1079A000204627F047FEFF2E45D0002130460396A3
:1079B00027F030FE039A242101FB09F3F918039301
:1079C00081F82160FF2681F820600221CAF8601545
:1079D000029BCAF80885CAF80C45CAF8102500228F
:1079E0001146CAF82435504650F0FCFB039BCAF8F8
:1079F000C065FA5807210AB34022CAF80423CAF81E
:107A00000015DBF8000040F30730F1F797FBDBF8D7
:107A1000000040F307303EF0E3FD242303FB097729
:107A200000237B77284601233B7709B0BDE8F08F20
:107A30004FF0FF34B7E74FF0FF32BCE7CAF800154C
:107A4000EBE700BF8C260A00EC41090020BF0900CB
:107A5000184A090000F0024000300240A0190A0054
:107A6000B1470900BC5B01200003005010B504467B
:107A7000407A41F0A0FB63681B68D3F82435B3F16A
:107A8000805F23D013D8B3F1006F21D00BD8B3F1AE
:107A9000007F1FD01248B3F1806F18BF0020400054
:107AA00040F0010010BD0F48B3F1206FF5E7B3F1CE
:107AB000804F11D006D8B3F1A05F0FD00A48B3F1C0
:107AC000005FEAE70948B3F1004FE6E70848E6E758
:107AD0000848E4E70848E2E70848E0E70848DEE746
:107AE00090D003000024F40080841E0000127A006D
:107AF00040420F0020A1070048E8010000093D00B6
:107B00000048E801F0B50C468DB054F8045B064619
:107B1000687A174641F04FFB284641F08DFB08ABD1
:107B200001931A4B0093214604233A46701E17F026
:107B300023FF062205A908981BF0A2FC9DF81C1043
:107B40000022402018F05CF8099B0A99049304462F
:107B5000069BB3FBF0F303AA04A8039350F002FBC7
:107B60000499039B614303FB04F20491039252B115
:107B700005989DF82C300144284641F03CFF10B98F
:107B8000052038F0B7FB0E200DB0F0BD34260A00FA
:107B9000F0B50C468BB054F8045B0646687A17467D
:107BA00041F009FB284641F047FB07AB0193194B15
:107BB0000093214603233A46701E17F0DDFE05228E
:107BC00004A907981BF05CFC9DF8181000224020C7
:107BD00018F016F8089B03930446059B0999B3FB1C
:107BE000F0F302AA03A8029350F0BCFA039B029A96
:107BF000634362430393029242B1049928461944B5
:107C000002F04AFE10B9052038F074FB0E200BB0CC
:107C1000F0BD00BF54260A00F0B50C4693B054F8EE
:107C2000046B0546707A174641F0C5FA304641F0BC
:107C300003FB0CAB01932B4B009321460623681EDC
:107C40003A4617F099FE052209A90C981BF018FC7A
:107C50009DF82C100022402017F0D2FF0E9B0F99A8
:107C6000059304460A9BB3FBF0F304AA05A804930A
:107C700050F078FA062206A90D981BF001FC9DF839
:107C800020100022402017F0BBFF109B1199039396
:107C90000546079BB3FBF0F302AA03A8029350F03A
:107CA00061FA049B039A0298059963436A4345432A
:107CB0006143AB42059104930392029502D00A48B6
:107CC00038F060FB53B106980244099801443046ED
:107CD00002F0AAFD10B9052038F00CFB0E2013B0FD
:107CE000F0BD00BF04260A00483909002DE9F04F15
:107CF0002DED028B97B0084611461A460AAB019348
:107D00005A4B00930C2349F0CEF940F26B510B987B
:107D10003AF02CFD40F2226181460A983AF026FDA5
:107D200040F26751824612983AF020FD4FF44D71AF
:107D3000804613983AF01AFD40F2625107461498B3
:107D40003AF014FD0546BAF1000F05D1B9F1000F64
:107D50000DD1474838F016FBD14518D0C24516D092
:107D6000BA4514D0824512D0B9F1000F05D0C145F3
:107D70000DD0B9450BD0A94509D0B8F1000F03D0FB
:107D8000B84504D0A84502D02FB1AF4203D14FF47B
:107D90009C6017F0E3FD40F2CA23092205210D98EB
:107DA00049F0B4F940F21D534FF6FF720646012127
:107DB000119849F0ABF90E9B2E4A9342834629D085
:107DC0002D4AA3EB020CDCF1000343EB0C035B0038
:107DD000022201210F980293962349F097F91098F7
:107DE0001DF010FCB0EE408A54F05EFF9DF8543058
:107DF000224903932C204AF0C2FCF6B20C9B079355
:107E0000082E039B044607D01D48082240F2CA21D1
:107E100038F0C0FA0123DBE705B913B1194838F08F
:107E200055FA4560184D2B68D3F8003513F00F0351
:107E300005D0AB68D3F800351E0714D10123DE004E
:107E400005EBC303636003931FFA8BF3184640F2FC
:107E50001D520121069349F051F9029B022B039B0D
:107E600018D10A4876E70A4874E700BFAC260A0032
:107E7000C42C0900E85F0900EC5F0900FCBE0900A2
:107E80009A4909007E3F090064020120AC400900C4
:107E9000A2470900BAF1000F00F0E0809AF804B0A0
:107EA000B9F1000F00F0DD8099F804200492002F52
:107EB00000F0DA803A790592B8F1000F00F0D7802F
:107EC00098F804200392029A1B790893002A18BF9D
:107ED0000E2208990292794A242303FB012393F886
:107EE0002030002B40F0C68047EA0803079809932A
:107EF00010F07AF9BBF1FF3F099005D0584627F002
:107F0000EBFB584627F096FB049B581C03D000213E
:107F1000184627F07FFBAB59099AC3F82425029B2A
:107F2000AA5947EA0801002918BF43F00103DBB250
:107F3000C2F86C35AB59049AC3F80CB5C3F81425D4
:107F4000B1B1059B591C03D00021184627F062FBF4
:107F5000039B5A1C05D0184627F0BEFB039827F058
:107F600069FBAB59039AC3F80825059AC3F8102595
:107F7000089A5249A8592423534301EB030B504A52
:107F8000CC504FF48871CBF8042050F008F9A85970
:107F90004FF4907150F003F9A8594FF4927150F0DA
:107FA000FEF8A8594FF4A27150F0F9F8A8594FF40F
:107FB000AC7150F0F4F8AB59424AC3F80423A85905
:107FC000032140F30730F1F7B9F8A85940F307301F
:107FD0003EF006FBAB590822C3F800250023CBE98D
:107FE0000633CBF8143001238BF82030B9F1000FA1
:107FF00045D1BAF1000F55D09AF8040084F8260054
:1080000001F016F9B8F1000F50D098F8040084F888
:10801000290001F00DF9002F4CD0387984F82800A0
:1080200001F006F9DFED287A079BA36028EE278A86
:108030000023BCEEC88A84F82530606884ED038A8A
:1080400004F1240127F098FE204B9842024612D1F9
:10805000204617B0BDEC028BBDE8F08F4FF0FF3B20
:108060001EE74FF0FF3221E74FF0FF3223E74FF0DA
:10807000FF3227E7164A1749174854F027FC06999C
:1080800004F1100051F046FC28B9606827F0FAFEB0
:10809000069838F0E1F899F8040084F8270001F018
:1080A000C7F8A6E7FF2384F82630ABE7FF2384F860
:1080B0002930B0E7FF2384F82830B3E7845C01203F
:1080C000A3C608001003420000007A440000AD0B74
:1080D0000500AD0B333609006C4A090010B522F0DB
:1080E00077FA90F82730FF2B044628D0406827F015
:1080F000C9FE94F826002DF025FF94F827002DF0F6
:1081000021FF94F829002DF01DFF94F828002DF090
:1081100019FF61680B4A4FF6FF73E3842385914290
:108120004FF00003C4E90433C4E90733A36103D06B
:108130000832914203D10123034A0021D1540E2079
:1081400010BD00BF640201201B69012010B522F0A0
:108150003FFA044690F8270041F027F894ED030A0F
:10816000DFED047AB8EE400ABDE8104080EE270A41
:108170001EF0D6BA00007A4410B522F029FA04465F
:1081800090F8270041F011F86368186840F3073051
:10819000002801DBF0F7C2FF0023C4E90733A36125
:1081A00063681B6843F30733002B08DB590901227E
:1081B00003F01F0302FA03F3024A42F821300E20B3
:1081C00010BD00BF00E100E038B52DED028B0D467B
:1081D00022F0FEF9044690F8270040F0E6FF28461A
:1081E0001DF010FAB0EE408A54F05EFDDFED057A26
:1081F00028EE278A0E20BCEEC88A84ED038ABDECE7
:10820000028B38BD00007A4407B50A4A40F2931346
:10821000914208BF4FF4A173019340F2ED13009314
:10822000054940F242234FF43A724AF0B9FC03B0D8
:1082300000BD00BFE85F0900631A09002DE9F0479F
:1082400015460E461F4622F0C3F9044690F8270053
:1082500040F0ABFF1DB900252846BDE8F0876368F4
:108260001B68D3F81435013304D12E4840F26B510A
:1082700038F090F853F0A0F8DFF8B0A080468946B7
:10828000A3699D4238D86368186840F30730002816
:1082900044DA2A46314604F1100051F05EFB94F8AE
:1082A0002530054693B1012204F1240104F11000A8
:1082B00051F07AFB04F12401606827F05DFD94F829
:1082C000290027F0DBF9002384F8253063681B6858
:1082D00043F30733002B08DB5909012203F01F0386
:1082E00002FA03F3104A42F82130002DB4D10B23D7
:1082F0003B604FF0FF35AFE753F05EF8E368B0EB5B
:10830000080061EB0901984271F10001BBD2F8F756
:108310001DFBDAF82830002BB2D09CE7F0F7FEFE08
:10832000B7E700BFAC41090000E100E0F85C0120C4
:1083300038B50C462046114606221D4617F0E4FAD1
:108340002CB921460120BDE83840F4F769BD296801
:10835000CB0706D411F0030308D10868144A9042F1
:1083600004D1012C14D0134837F0F8FF124A0A4008
:10837000062A04D03BB90A68104B9A4203D1012C5B
:1083800001D10F48F0E7BDE838400120F4F7A8BC60
:10839000084649F01AFE054601462046F4F740FD1E
:1083A0002A4604460021C06848F031FD204638BD09
:1083B000E42A09005B2B09000F0080FF58290900FF
:1083C0009C2D0900012807B50B4606D10B680093C8
:1083D00040F61623019302206B4601460022024814
:1083E0001FF096FA03B000BD582909000146014864
:1083F0001CF076B9B0590900014A1CF0B7B900BFAA
:10840000B0590900014A1CF0B1B900BF5829090050
:1084100008B508460AB117F0A9FA21B11946BDE816
:10842000084000F005B8014808BD00BF505A0900D7
:1084300070B50646086810F003038EB00D4603D1F0
:108440000168454A91422AD0444C00EA0402062AB7
:1084500004D043BB0268424B9A4224D1023E012E13
:1084600002D9404837F07AFF0AA91FF00DFA0646F4
:10847000286800EA0403062B13D1000950F0A6FD7A
:1084800004460A9D24B92946304650F076FD04463C
:10849000314910204AF06CF9C0E9025644600EB030
:1084A00070BD4468EDE7012E01D02F48DAE710F0E7
:1084B000010411D0441002D5002037F063FF21469B
:1084C0000AA854F087FE0C982246002148F09FFC31
:1084D0000AA81EF081F8E2E701AA40F25F211BF032
:1084E00051FE019B2BB101AA2146204648F024FFF2
:1084F000D5E72868324603A91AF0C2FF20B1DDE9AA
:1085000003011EF061F8CAE728681DF0AFFF0446BA
:10851000B8B91020CDE90A0448F080FB8DF834404A
:108520000C90286806A91BF017F8044620461BF09B
:10853000D5F90028CCD049F048FDFF2806D90B48D2
:10854000BBE741100AA854F037FEEAE7C1B20AA817
:1085500054F07EFDEAE700BFB05909000F0080FF2C
:10856000582909009C2D09005B2B090025390900B9
:10857000F0B585B0054617460C461DF0CDF86946A6
:10858000064628461FF080F9042F054622D1A3078E
:10859000009814D12268104B9A4210D101AA2146AA
:1085A0004AF048FC10B90D4837F090FEDDE90112A1
:1085B0003046521A29441EF0E5F905B0F0BD0146D7
:1085C0000023224630461AF079FF285C400040F034
:1085D0000100F2E70020F0E734540900FD2F090004
:1085E0002DE9F14F8F0705460C46164613D001F0D2
:1085F0000F03022B19D102F0FD06012E4FEA1111D3
:1086000004D001B0BDE8F04F06F0E4BD01B0BDE814
:10861000F04F06F0EDBA4968CBB22D2B00F0878001
:108620000BD8062B0ED02C2B13D0554A21462846AA
:1086300001B0BDE8F04F06F0DBBD2E2B00F08C80C2
:108640009D2BF2D1002EF0D104F10802090A284630
:1086500087E0022A02D0A16806F020FBE768002F1D
:10866000E3D017F00309E0D17B68DAB28E2AB8466E
:108670000DD1022E4FEA132805D007F1040A08F1A4
:10868000FF3BD94515DB08F1010857F8288098F819
:108690000430312B2BD1022E13D1686A48F0E0FF51
:1086A000686A56226FF0020101B0BDE8F04F45F054
:1086B0008FBA5AF8041F284606F0F0FA09F10109AA
:1086C000DFE72846D8F8081006F0E8FA012E686AB5
:1086D00009D15822022145F07BFA686A01B0BDE851
:1086E000F04F48F0E7BF56226FF00201DCE7322B73
:1086F0009BD1012E686A0AD148F000FFD8F8081013
:10870000686A090901B0BDE8F04F48F0A8BE022E22
:1087100001D148F0A9FFD8F80830686A1B0918226F
:108720006FF0010101B0BDE8F04F45F0D1BAA26889
:10873000002A3FF47AAF002E7FF477AF5168090A20
:10874000022907D1D3682BB1980703D11B79AC2B31
:108750003FF46BAF08327AE7002A7FF466AFA16876
:1087600021B901B0BDE8F04F00F00CB88E0703D17D
:108770000B79922B0A46E1D004F10802012166E749
:10878000ED3809002DE9F04701F1FF3A054688462A
:1087900091464FEA0A2700244FF0FF3617F5807FF5
:1087A0000CD1731C05D1686A4346302251460AF049
:1087B000A3FF002444451DD1BDE8F08759F82410DB
:1087C00071B18A070CD10A79222A09D101360BD15D
:1087D000686A47EA0403312251460AF08DFF2646B3
:1087E0000134A7F58077D9E72846084ABDE8F04765
:1087F00006F0FEBC59F82410A64208BF8968002282
:108800002846FFF7EDFE0134D4E700BFA43109008C
:1088100001F00F03022B2DE9F04707460C4604D167
:10882000BDE8F047090906F081B800295BD011F0D6
:10883000030558D10B792C2B3FD1896806F02EFA0D
:10884000E568002D4FD015F003084CD16E68F2B2E8
:108850008E2A2B4609D1360A05F1040906F1FF3AA2
:10886000C24518DC013655F826301A79312A1AD15A
:108870009968384606F012FA7C6A204648F0CAFE2B
:10888000204648F0EDFE20465622BDE8F0476FF046
:10889000020145F09DB959F8041F384606F0FEF96B
:1088A00008F10108DCE7322A1DD19968786A0222B2
:1088B000BDE8F047090948F0BABD2D2B13D18C68EB
:1088C0008CB163681B0A022B01D1E36833B9261D02
:1088D0006368B5EB132F0DD3BDE8F0879A07F6D187
:1088E0001B79AC2BF3D121463846064ABDE8F04748
:1088F00006F07EBC56F8041F3846FFF789FF0135A5
:10890000E6E700BF8F38090070B5137803F0600305
:10891000202B104660D19388304A54789C420ED068
:1089200092F829489C4257D102F628030125447841
:10893000203C032C50D8DFE804F005050E37134621
:108940000025F4E7012904D1072203F1080136F0DC
:108950006DFF012070BD012902D136F057FFF8E705
:108960000329F6D14188597101F0010093F82310D1
:1089700080F00104B4EBD11F1CBF64F3C71183F86E
:10898000231050B99368B3F5966FE2D14FF080434E
:108990004E22C3F81C252DF0ABFA114B11480122D1
:1089A0001A70F7F797FFD4E70129D6D00329D0D161
:1089B0000D4B1B78002BCCD00C4B1B680133C8D05F
:1089C000002DC6D14388002BC3D0094B094A5A66F3
:1089D00003F15C029A62BCE70020BBE75C10012057
:1089E0005B67012040610120466901201C020120D3
:1089F000F85C0120145F09002DE9F04700211B48B5
:108A000041F2500248F003FA184B00209C464FF008
:108A1000FF0A4FF4E13901464FF008084FF4806433
:108A200040F6280E012748F2010503F128021A61D9
:108A30000EFB00C203F5856683F806A0C3F8089014
:108A40001973597383F80E809C825183D7821183E6
:108A5000DE611C84D18455849184421C022A03F671
:108A600028034FF00100E0D1BDE8F0875C10012041
:108A70002DE9F3414B79022B12D18B79022B0FD1C7
:108A8000274D95F80280B8F1000F12D095F82A38DA
:108A90005BB14FF0E023D3F8F03DDB0700D500BE1B
:108AA0000026304602B0BDE8F0814FF0010805F61F
:108AB000280528708B786B700B780926CC186378A2
:108AC000242B1ED1964217D96378042B10D16379D9
:108AD0000A2B0DD12778AB1C022200931146EB1C08
:108AE000E01953F0ABFF0028D3D00E363744BEB2A6
:108AF0004046F2F7B7F9D4E723781E44B6B21C44D7
:108B0000DDE7052BE0D1204639F0ACFA0028C0D0D3
